:10800000BC5200200DEB010025EB010027EB010025
:1080100029EB010029EB010029EB01000000000021
:1080200000000000000000000000000029EB01003B
:1080300029EB01000000000029EB01002BAC00003F
:1080400029EB010029EB010029EB010029EB0100DC
:1080500029EB010029EB0100A987000029EB0100B1
:1080600029EB010029EB010029EB010029EB0100BC
:1080700029EB010029EB010029EB010029EB0100AC
:1080800029EB010029EB010029EB010029EB01009C
:1080900029EB010029EB010029EB010029EB01008C
:1080A00029EB010029EB010029EB010029EB01007C
:1080B00029EB010029EB010029EB010029EB01006C
:1080C00029EB010029EB010029EB010029EB01005C
:1080D00029EB010029EB010029EB010029EB01004C
:1080E00029EB010029EB01000000000029EB010051
:1080F00029EB010029EB010029EB010029EB01002C
:1081000029EB010029EB010029EB010029EB01001B
:10811000000000000000000029EB010029EB010035
:1081200029EB010029EB010029EB010029EB0100FB
:1081300029EB010029EB010029EB010029EB0100EB
:10814000000000000000000000000000000000002F
:1081500029EB010029EB010029EB010029EB0100CB
:10816000000000000000000000000000000000000F
:1081700000000000000000000000000000000000FF
:1081800000000000000000000000000000000000EF
:1081900000000000000000000000000000000000DF
:1081A00000000000000000000000000000000000CF
:1081B00029EB010029EB010029EB010029EB01006B
:1081C00029EB010029EB010029EB010029EB01005B
:1081D00029EB010029EB010029EB010029EB01004B
:1081E00029EB010029EB010029EB01000000000050
:1081F0000000000029EB010029EB010029EB010040
:1082000029EB010029EB0100000000000000000044
:1082100029EB010029EB010029EB010029EB01000A
:1082200029EB010029EB010029EB010029EB0100FA
:1082300029EB010029EB010029EB010029EB0100EA
:1082400029EB010029EB010029EB010029EB0100DA
:1082500029EB010029EB010029EB010029EB0100CA
:1082600029EB010029EB010029EB010080B5DFF8C3
:10827000380B01F02BFFDFF8340B01F027FF02F081
:108280009DF8DFF82C0B02F0AEF80121DFF8240B8B
:1082900002F0E4F90120DFF8201B0860DFF81C0B76
:1082A000DFF81C1B0860FF20DFF8181B0860802126
:1082B000DFF8140B02F0D2F98020DFF8101B086001
:1082C000DFF80C0B02F0F4F9DFF8080B02F0F0F91C
:1082D0003021DFF8040B02F0DDF901F08DFF60239F
:1082E0004FF461420100DFF8F40A02F04DFA102267
:1082F0000221DFF8E80A02F043FADFF8E40A006836
:1083000030F01000DFF8D81A08601021DFF8CC0A2E
:1083100002F08DFADFF8C40A02F065FA0321DFF8F3
:10832000BC0A02F092FA162002F0CEF8172002F0F2
:10833000CBF8C021162002F096FA162002F0A4FA1B
:108340000F21162002F052F8DFF85C1C162002F014
:1083500060F80F21172002F049F8DFF8501C1720B1
:1083600002F057F801200021DFF8442CC2E9000197
:1083700001F0F0FDDFF83C0C006850F00100DFF880
:10838000341C086001BD80B5DFF8280C0078C007F8
:1083900040F1EE81DFF81C0C0068C0F3800000287B
:1083A00040F0E381DFF8080CD0E90001012200234E
:1083B000994204D1904202D100F018FAD5E1DFF8D9
:1083C000F00BD0E90001002904D1022802D100F00D
:1083D000F6FACAE1DFF8D80BD0E90001B1F5807FE9
:1083E00004D1002802D100F0B8FBBEE1DFF8C00BD9
:1083F000D0E90001B1F5007F04D1002802D100F0DE
:108400000CFCB2E1DFF8A80BD0E900010022012347
:10841000994204D1904202D100F045FBA5E1DFF87A
:10842000900BD0E90001002904D1042802D100F00A
:1084300054FC9AE1DFF8780BD0E90001002904D15F
:10844000082802D100F0CEFC8FE1DFF8640BD0E900
:108450000001002905D1B0F5807F02D100F019FE9E
:1084600083E1DFF84C0BD0E90001802904D100281A
:1084700002D100F0A1FD78E1DFF8340BD0E9000172
:10848000002905D1102803D1012000F057FE6CE12E
:10849000DFF81C0BD0E90001022905D1002803D127
:1084A000012000F0F6FE60E1DFF8040BD0E90001E6
:1084B000002905D1202803D1022000F03FFE54E11D
:1084C000DFF8EC0AD0E90001042905D1002803D126
:1084D000022000F0DEFE48E1DFF8D40AD0E9000116
:1084E000002905D1402803D1032000F027FE3CE1FC
:1084F000DFF8BC0AD0E90001082905D1002803D122
:10850000032000F0C6FE30E1DFF8A40AD0E9000144
:10851000002905D1B0F5806F02D100F02FFF24E1D2
:10852000DFF88C0AD0E90001002905D1B0F5801FE1
:1085300002D100F0D5FF18E1DFF8740AD0E900019C
:10854000202904D1002802D101F016F80DE1DFF84E
:10855000600AD0E9000100225FF08073994205D1E2
:10856000904203D1002001F0BBF8FEE0DFF8400AA2
:10857000D0E9000100225FF00073994205D19042DA
:1085800003D1012001F0ACF8EFE0DFF8240AD0E9D4
:10859000000100225FF08063994205D1904203D12F
:1085A000022001F09DF8E0E0DFF8040AD0E90001C4
:1085B00000225FF00063994205D1904203D103206D
:1085C00001F08EF8D1E0DFF8E809D0E900010022DF
:1085D0005FF08053994205D1904203D1042001F00D
:1085E0007FF8C2E0DFF8C809D0E9000100225FF09F
:1085F0000053994205D1904203D1052001F070F853
:10860000B3E0DFF8AC09D0E9000100225FF080435D
:10861000994205D1904203D1062001F061F8A4E00F
:10862000DFF88C09D0E9000100225FF00043994295
:1086300005D1904203D1072001F052F895E0DFF810
:108640007009D0E90001002906D1B0F5805F03D19F
:10865000002001F0CEF888E0DFF85409D0E90001ED
:10866000002906D1B0F5005F03D1012001F0C1F867
:108670007BE0DFF83C09D0E90001002906D1B0F524
:10868000804F03D1022001F0B4F86EE0DFF820093A
:10869000D0E90001002906D1B0F5004F03D1032035
:1086A00001F0A7F861E0DFF80809D0E9000100292E
:1086B00006D1B0F5803F03D1042001F09AF854E0D0
:1086C000DFF8EC08D0E90001002906D1B0F5003F41
:1086D00003D1052001F08DF847E0DFF8D408D0E998
:1086E0000001002906D1B0F5802F03D1062001F04A
:1086F00080F83AE0DFF8B808D0E90001002906D197
:10870000B0F5002F03D1072001F073F82DE0DFF85A
:10871000A008D0E90001002905D1B0F5807F02D181
:1087200000F0B7FC21E0DFF88808D0E9000140291B
:1087300004D1002802D100F082FF16E0DFF87008B3
:10874000D0E90001002905D1B0F5007F02D101F088
:1087500007F90AE0DFF85808D0E90001002904D140
:10876000B0F5006F01D101F0ABF8082002F0B3F9C9
:1087700001BD10B4DFF8F02BD2E9002302430B4314
:10878000DFF8E44BC4E90023DFF8E02BD2E9002353
:1087900010431943DFF8D42BC2E9000110BC704725
:1087A000DFF8CC1B0860704780B50121DFF82C068C
:1087B00002F042F80100DFF8240602F043F8DFF887
:1087C000F4070068C0F38000002807D1162001F0EC
:1087D00067FE002809D101F0AFF906E0DFF8940B3D
:1087E0000068800601D501F0A7F901BD10B5DFF8DA
:1087F000C4070068C0F3400000287AD12920DFF8C0
:10880000DC1C08700020DFF8D41C48708820DFF8DA
:10881000CC1C88705320DFF8C41CC8704420DFF8DB
:10882000BC1C08714B20DFF8B41C48714520DFF8F0
:10883000AC1C88715620DFF8A41CC8714F20DFF8EB
:108840009C1C08720020DFF8941C48720020DFF89E
:108850008C1C88720020DFF8841CC8720020DFF8AE
:108860007C1C08730020DFF8741C48730020DFF8BC
:108870006C1C88730020DFF8641CC8730020DFF8CC
:108880005C1C08740E2002F003F9DFF8501C4874D9
:108890000F2002F0FDF8DFF8441C8874FF20DFF899
:1088A0003C1CC874FF20DFF8341C0875FF20DFF87B
:1088B0002C1C48758420DFF8241C88757B20DFF889
:1088C0001C1CC875002005E00021DFF8102C0244B4
:1088D0001176401C1328F7D33320DFF8001C81F8F1
:1088E00022003020DFF8F41B81F8230001F051F959
:1088F00064E001F0B8F901285ED1DFF8780C407827
:10890000BB2802D102F0EEF858E0DFF8680C80785E
:1089100088284ED1002407E0DFF8580C2044C178A5
:10892000200002F09EFA641C0E2CF5D3DFF8440CF4
:1089300090F82210002002F008FADFF8380C90F8C6
:108940002310012002F001FADFF8280C817D0220BB
:1089500002F0FBF9DFF81C0CC17D032002F0F5F9F1
:10896000DFF8100C417C042002F0EFF9DFF8040C72
:10897000817C052002F0E9F9DFF8F80B90F8270078
:108980000006DFF8F01B91F8281010EB0140DFF82B
:10899000E41B91F8291010EB0120DFF8D81B91F8A7
:1089A0002A10401802F0F6FB01F097F801F0FCFAEB
:1089B00004E001F01CF801E001F050F810BD80B5B2
:1089C000DFF8F0050068C0F34000002810D1052052
:1089D000DFF8081B08700020DFF8001B48702F200C
:1089E000DFF8F81A887001F0DBF901F0D2F859E0ED
:1089F00001F039F9012853D1DFF8780B4078BB2812
:108A000002D102F06FF84DE0DFF8680B8078A12802
:108A10003CD1DFF85809D0E9000110F0000011F452
:108A200080710022002399420FD190420DD1DFF8CE
:108A3000440B8379DFF83C0B4279DFF8380B01797E
:108A4000DFF8300BC07802F034FCDFF82009D0E901
:108A5000000110F0000011F400710022002399427F
:108A60000FD190420DD1DFF80C0B837ADFF8040BA5
:108A7000427ADFF8000B017ADFF8F80AC07902F0D9
:108A800023FC01F02AF801F08FFA0BE0F92804D159
:108A900001F023F801F05EFA04E000F0A8FF01E025
:108AA00000F0DCFF01BD80B5DFF808050068C0F309
:108AB000400000281DD10720DFF8201A0870002090
:108AC000DFF8181A48705220DFF8101A887001F089
:108AD00067F97F2002F0A2FADFF8001AC871DFF808
:108AE000FC09C079C043DFF8F419087201F051F8AD
:108AF00032E001F0B8F801282CD1DFF8780A40788C
:108B0000BB2802D101F0EEFF26E0DFF8680A80788A
:108B1000862806D101F051F900F0DFFF01F044FA98
:108B20001AE0F0280CD1DFF84C0AC078522804D1A2
:108B300000F0D3FF01F038FA0EE000F058FF0BE030
:108B4000F92804D100F0C9FF01F004FA04E000F0B4
:108B50004EFF01E000F082FF01BD80B5DFF8540454
:108B60000068C0F3400000282CD10A20DFF86C19FF
:108B700008700020DFF8641948708720DFF85C195E
:108B8000887001F00DF90120DFF85019C87100203C
:108B900002F0A5FBDFF844190872012002F09FFBE8
:108BA000DFF838194872022002F099FBDFF82C191F
:108BB0008872032002F093FBDFF82019C87200F0DE
:108BC000E8FF29E001F04FF8012823D1DFF8A409DC
:108BD0004078BB2802D101F085FF1DE0DFF8940941
:108BE0008078F0280CD1DFF88C09C078872804D170
:108BF00000F073FF01F0D8F90EE000F0F8FE0BE092
:108C0000F92804D100F069FF01F0A4F904E000F0B4
:108C1000EEFE01E000F022FF01BD80B5DFF8940315
:108C20000068C0F3400000282CD10A20DFF8AC18FF
:108C300008700020DFF8A41848708720DFF89C181F
:108C4000887001F0ADF80220DFF89018C87100209C
:108C500002F04CFBDFF884180872012002F046FB9A
:108C6000DFF878184872022002F040FBDFF86C1839
:108C70008872032002F03AFBDFF86018C87200F037
:108C800088FF29E000F0EFFF012823D1DFF8E40896
:108C90004078BB2802D101F025FF1DE0DFF8D408A1
:108CA0008078F0280CD1DFF8CC08C078872804D170
:108CB00000F013FF01F078F90EE000F098FE0BE0F1
:108CC000F92804D100F009FF01F044F904E000F0B4
:108CD0008EFE01E000F0C2FE01BD80B5B54800681F
:108CE000C0F3400000283AD10E20DFF8F0170870DA
:108CF0000020DFF8E81748700620DFF8E0178870DA
:108D000001F04EF80020DFF8D417C8715FF0FF3093
:108D100002F009FC0100090EDFF8C0271172010002
:108D2000090CDFF8B82751720100090ADFF8AC27F7
:108D30009172DFF8A817C8720020DFF8A017087337
:108D40000020DFF8981748730020DFF89017887329
:108D50000020DFF88817C87300F01BFF23E000F045
:108D600082FF01281DD1DFF80C084078BB2802D112
:108D700001F0B8FE17E0DFF8FC078078862806D1FE
:108D800001F01BF800F0A9FE01F00EF90BE0F92844
:108D900004D100F0A2FE01F0DDF804E000F027FEAF
:108DA00001E000F05BFE01BD011800F0000C00F0D6
:108DB0000008002000400240044002404B434F4C5A
:108DC0002075004024750040007000400072004093
:108DD00002100200021402000060004000D00040B7
:108DE0002CD0004080B573480068C0F340000028D4
:108DF0003AD10E20DFF8E41608700020DFF8DC1608
:108E000048700720DFF8D416887000F0C9FF0020F2
:108E1000DFF8C816C8715FF0FF3002F084FB010074
:108E2000090EDFF8B82611720100090CDFF8AC2634
:108E300051720100090ADFF8A4269172DFF89C162E
:108E4000C8720020DFF8941608730020DFF88C1633
:108E500048730020DFF8841688730020DFF87C1642
:108E6000C87300F096FE9EE000F0FDFE012840F081
:108E70009880DFF800074078BB2802D101F032FE6D
:108E800091E0DFF8F0068078772840F08080DFF806
:108E9000E406C078DFF8DC16097910EB012002F057
:108EA00022F9DFF8D0064079DFF8C816897910EB8F
:108EB000012002F02CF9DFF8BC06407ADFF8B41686
:108EC000897A10EB012002F02AF9DFF8A806407B2E
:108ED000DFF8A016897B10EB012002F010F9DFF813
:108EE0009406C07BDFF88C16097C10EB012002F0A1
:108EF0001EF9DFF88006C07D00F0FF00DFF8741671
:108F0000097E10EB012002F0F2F8DFF86806C07E5F
:108F1000DFF86016097F10EB012002F01DFADFF880
:108F20005406407FDFF84C16897F10EB012002F0D9
:108F300010FADFF84006C07FDFF8381691F82010ED
:108F400010EB012002F00BFADFF82004D0E9000159
:108F5000C00217D4DFF81C0690F82100DFF81416C1
:108F600091F8221050EA012002F052FADFF80406CC
:108F700090F82300DFF8FC1591F8241050EA012046
:108F800002F04CFA00F0A9FD01F00EF80BE0F92810
:108F900004D100F0A2FD00F0DDFF04E000F027FDA9
:108FA00001E000F05BFD01BD0080000C008000C00E
:108FB00088110020E011002080B5DFF8BC030068B4
:108FC000C0F34000002837D10D20DFF810150870DD
:108FD0000020DFF8081548708520DFF8001588703C
:108FE00000F0DEFE02F0C9F80100090EDFF8EC2403
:108FF000D1710100090CDFF8E42411720100090AA3
:10900000DFF8D8245172DFF8D4148872C04301000D
:10901000090EDFF8C824D1720100090CDFF8BC2466
:1090200011730100090ADFF8B4245173DFF8AC149E
:10903000887300F0AEFD2BE000F015FE012825D16D
:10904000DFF830054078BB2802D101F04BFD1FE06E
:10905000DFF820058078F0280ED1DFF81805C078F9
:10906000852806D102F08DF800F037FD00F09CFF56
:109070000EE000F0BCFC0BE0F92804D100F02DFD5F
:1090800000F068FF04E000F0B2FC01E000F0E6FC54
:1090900001BD10B5DFF8E0020068C0F34000002811
:1090A00010D10520DFF8341408700020DFF82C14EC
:1090B00048700D20DFF82414887000F071FE00F075
:1090C00068FD3AE000F0CFFD012834D1DFF8A404B8
:1090D0004078BB2802D101F005FD2EE0DFF89404B2
:1090E00080789D281DD1A148D0E9000110F0000032
:1090F00011F040010022002399420DD190420BD182
:10910000002407E0DFF86C042044C178200002F05E
:1091100057F8641C1F2CF5D300F0DFFC00F044FF6F
:109120000BE0F92804D100F0D8FC00F013FF04E0B4
:1091300000F05DFC01E000F091FC10BD10B50400F2
:109140008D480068C0F3400000281ED10520DFF8DC
:109150008C1308700020DFF884134870012C04D1B0
:109160000120DFF8781388700AE0022C04D1022075
:10917000DFF86813887003E00320DFF8601388705D
:1091800000F00EFE00F005FD82E000F06CFD01280D
:109190007CD1DFF8E0034078BB2802D101F0A2FCCB
:1091A00076E0DFF8D0038078832820D1032C1ED10D
:1091B0006E48D0E9000110F0000011F00801002213
:1091C000002399420ED190420CD1002408E0DFF830
:1091D000A4032044C17814F1400002F0F5F9641CA6
:1091E0001F2CF4D300F079FC00F0DEFE50E0822862
:1091F00020D1022C1ED15D48D0E9000110F0000002
:1092000011F004010022002399420ED190420CD1AA
:10921000002408E0DFF85C032044C17814F120004A
:1092200002F0D2F9641C1F2CF4D300F056FC00F0BD
:10923000BBFE2DE081281FD1012C1DD14B48D0E968
:10924000000110F0000011F00201002200239942F9
:109250000DD190420BD1002407E0DFF81803204421
:10926000C178200002F0B0F9641C1F2CF5D300F087
:1092700034FC00F099FE0BE0F92804D100F02DFC3D
:1092800000F068FE04E000F0B2FB01E000F0E6FB55
:1092900010BD38B5040038480068C0F3400000280D
:1092A0002DD124208D49087000208C494870012C54
:1092B00003D181208949887008E0022C03D18220E3
:1092C0008649887002E083208449887000F068FD38
:1092D000012C01D1002404E0022C01D1202400E063
:1092E0004024002506E0281902F06BF97B49294447
:1092F000C8716D1C1F2DF6D300F04BFC33E000F05D
:10930000B2FC01282DD19B484078BB2802D101F046
:10931000E9FB28E0974880789649C978F02816D16B
:10932000012C02D1C9B2812909D0022C02D1C9B2C3
:10933000822904D0032C07D1C9B2832904D100F0BB
:10934000CCFB00F031FE0EE000F051FB0BE0F92801
:1093500004D100F0C2FB00F0FDFD04E000F047FB8B
:1093600001E000F07BFB31BD90110020981100203E
:10937000F01100203CD00040E011002080B5DFF863
:10938000200C0068C0F34000002810D1022053498F
:1093900008700020514948700B2050498870DFF850
:1093A000040C00684D49C87000F0F3FB94E000F035
:1093B0005AFC012840F08E806E484078BB2802D1CC
:1093C00001F090FB88E06B4880788B2840F07F802C
:1093D0006848C078DFF8CC1B0968884274D16548BA
:1093E0000179DFF8C00B006802F028F86148417984
:1093F0006048807951EA00215E48C07951EA004115
:109400005C48007A51EA0061DFF8980B006801F0CF
:10941000CDFF5848427A00235648807A002109023D
:1094200041EA1061000202430B435248C07A002116
:10943000090441EA1041000402430B434D48007BFC
:109440000021090641EA1021000602430B43494866
:10945000407C00210100002002430B434548807CF2
:1094600000210102002002430B434248C07C00213E
:109470000104002002430B433E48007D0021010609
:10948000002002430B43DFF81C0B006801F0A3FF30
:109490003848417B3748807B51EA00213548C07B02
:1094A00051EA00413348007C51EA0061DFF8F40AD8
:1094B000006801F0A4FF0020DFF8E81A086000F05F
:1094C0000CFB00F071FD07E000F091FA04E000F001
:1094D0008EFA01E000F0C2FA01BD0000200E00206B
:1094E00080B5DFF8BC0A0068C0F34000002820D136
:1094F0000520DFF8601B08700020DFF8581B48705B
:109500000A20DFF8501B887001F085FFDFF8441B4C
:10951000C870000ADFF83C1B087101F082FFDFF819
:10952000341B4871000ADFF82C1B887100F031FBF6
:109530001FE000F098FB012819D10E484078BB28A5
:1095400002D101F0CFFA14E00A488078F0280BD15C
:109550000848C0780A2804D100F0BFFA00F024FDC2
:1095600007E000F044FA04E000F041FA01E000F006
:1095700075FA01BDA00D002080B5DFF8240A00684F
:10958000C0F3400000282ED10B20DFF8C81A087065
:109590000020DFF8C01A48708F20DFF8B81A8870F2
:1095A00000F0FEFB002001F006FEDFF8A81AC871EB
:1095B000012001F000FEDFF89C1A0872022001F081
:1095C000FAFDDFF8901A4872042001F0F4FDDFF88C
:1095D000841AC872052001F0EEFDDFF8781A0873CE
:1095E00000F0D7FA2AE000F03EFB012824D1DFF892
:1095F000680A4078BB2802D101F074FA1EE0DFF857
:10960000580A8078DFF8501AC978F0280AD1C9B210
:109610008F2904D100F061FA00F0C6FC0EE000F0E2
:10962000E6F90BE0F92804D100F057FA00F092FCBB
:1096300004E000F0DCF901E000F010FA01BD10B523
:10964000DFF85C090068C0F3400000281CD1252029
:10965000DFF8001A08700020DFF8F81948709D2024
:10966000DFF8F019887000F09BFB002407E0200071
:1096700001F0B1FDDFF8DC192144C871641C202C15
:10968000F5D300F086FA2AE000F0EDFA012824D1A3
:10969000DFF8C4094078BB2802D101F023FA1EE0AC
:1096A000DFF8B4098078DFF8B019C978F0280AD15A
:1096B000C9B29D2904D100F010FA00F075FC0EE04B
:1096C00000F095F90BE0F92804D100F006FA00F05B
:1096D00041FC04E000F08BF901E000F0BFF910BD9F
:1096E00038B50400DFF8B8080068C0F3400000286F
:1096F00052D12620DFF85C1908700020DFF85419D9
:1097000048709020DFF84C19887000F049FB012C5C
:1097100004D10120DFF83C19C8712DE0022C04D1DE
:109720000220DFF83019C87126E0032C04D1032091
:10973000DFF82019C8711FE0042C04D10420DFF8E1
:109740001419C87118E0052C04D10520DFF804199C
:10975000C87111E0062C04D10620DFF8F818C87192
:109760000AE0072C04D10720DFF8E818C87103E0ED
:109770000020DFF8E018C871002508E0290020006B
:1097800001F0C9FDDFF8CC18294408726D1C1F2DAB
:10979000F4D300F0FEF92BE000F065FA012825D1A2
:1097A000DFF8B4084078BB2802D101F09BF91FE034
:1097B000DFF8A4088278DFF8A008C078DFF89818EE
:1097C0000979F02A08D1902806D1A14204D100F0ED
:1097D00084F900F0E9FB0BE0F92804D100F07DF9F1
:1097E00000F0B8FB04E000F002F901E000F036F907
:1097F00031BD38B50400DFF8A8070068C0F34000A9
:10980000002813D10620DFF84C1808700020DFF87C
:10981000441848701020DFF83C18887000F0C0FA37
:10982000DFF83008C47100F0B4F948E000F01BFA2A
:10983000012842D1DFF820084078BB2802D101F08E
:1098400051F93CE0DFF81008807890282BD10020F7
:109850005FF08071220001F0E5FEDFF80028D2E918
:1098600000231040194000220023994218D1904251
:1098700016D1DFF8E407C078844211D1002508E052
:10988000DFF8D407284402792900200001F035FDD3
:109890006D1C202DF4D300F020F900F085FB0EE0C4
:1098A00000F0A5F80BE0F92804D100F016F900F05B
:1098B00051FB04E000F09BF801E000F0CFF831BD6F
:1098C00080B5DFF8DC060068C0F34000002810D146
:1098D0000520DFF8801708700020DFF8781748703F
:1098E0000E20DFF87017887000F05AFA00F051F976
:1098F00035E000F0B8F901282FD1DFF85C07407897
:10990000BB2802D101F0EEF829E0DFF84C0780789F
:10991000912818D1DFF840070079DFF83C17497922
:1099200050EA0120DFF83017897950EA0140DFF86A
:109930002817C97950EA016001F01BFB00F0CDF84F
:1099400000F032FB0BE0F92804D100F0C6F800F07B
:1099500001FB04E000F04BF801E000F07FF801BDEE
:1099600080B5DFF83C060068C0F34000002810D145
:109970000520DFF8E01608700020DFF8D8164870E0
:109980000F20DFF8D016887000F00AFA00F001F915
:109990002CE000F068F9012826D1DFF8BC064078F9
:1099A000BB2802D101F09EF820E0DFF8AC068078F9
:1099B00078280FD1DFF8A0064279DFF89C060179FC
:1099C000DFF89406C07801F0BAFC00F086F800F0E9
:1099D000EBFA0BE0F92804D100F07FF800F0BAFAB6
:1099E00004E000F004F801E000F038F801BD80B5B3
:1099F000DFF86C060068401CDFF864160860DFF8CA
:109A0000A005006830F00200DFF894150860DFF868
:109A10005406D0E90001DFF85026D2E900231043B4
:109A20001943DFF84026C2E90001DFF83006D0E92B
:109A30000001DFF83426D2E9002310431943DFF890
:109A40001C26C2E90001DFF8180600680B2804D3C1
:109A5000102001F062FD00F07DFA01BD80B501F03B
:109A600037F8DFF808160968401A652834D3DFF89C
:109A70003005006830F00200DFF824150860DFF8D8
:109A8000E405D0E90001DFF8E025D2E90023104326
:109A90001943DFF8D025C2E90001DFF8C005D0E99D
:109AA0000001DFF8C425D2E9002310431943DFF891
:109AB000AC25C2E90001DFF8B8050068401CDFF8FA
:109AC000B0150860DFF8A80500680A2804D3102044
:109AD00001F023FD00F03EFA01BD80B50020DFF863
:109AE00080150860DFF8B804006830F00200DFF885
:109AF000B0140860102001F009FD01BD80B5DFF849
:109B0000A014096851F00401DFF894241160802149
:109B1000DFF8602511600121DFF85C2511600090FD
:109B2000DFF85835DFF858250121172000F07DFCBB
:109B3000172000F048FC01BD80B5DFF86404006820
:109B400030F00400DFF8581408600020DFF8281512
:109B500008600020DFF81C150860162000F03BFCB0
:109B6000002004E00021DFF81C251154401CB0F552
:109B7000807FF7D34FF480700090DFF80835DFF86E
:109B8000FC240121162000F050FC162000F01BFCE4
:109B900001BD38B501250220DFF8E4140870002467
:109BA0001FE0DFF8B004005DC0B20009C0B201F0F0
:109BB0009AFDDFF8CC1401EB44014870DFF89404FF
:109BC000005D10F00F0001F08EFDDFF8B41401EB22
:109BD00044018870002C03D0DFF87804005D2D1854
:109BE000641CDFF870040078801C8442D9D3ED43F4
:109BF00005F0FF052800000901F075FDDFF880146D
:109C000001EB4401487015F00F05280001F06BFDD1
:109C1000DFF86C1401EB440188700320DFF8601456
:109C200001EB4401C8706000001DFFF767FFDFF81B
:109C30007003006850F00200DFF86413086000F061
:109C400047FFDFF828140860DFF81804D0E90001A6
:109C5000DFF81424D2E9002390439943DFF8042469
:109C6000C2E9000131BDF8B5002000E0401CB0F5AC
:109C7000807F09DADFF80C14095C0329F6D10400AF
:109C80000021DFF800241154B0F5807F01DA002CA8
:109C900001D1002074E0651E00E06D1E002D6ED421
:109CA000DFF8E003405D0228F7D10020DFF8D4138D
:109CB0004855641B641C083CE00701D502205FE0A6
:109CC0006408201F792801D3022059E0681C00F0A5
:109CD000FF00411C01F0FF01DFF8A823515CDFF811
:109CE000A423105C00F04DF8DFF86C130870DFF867
:109CF00068030078844201D0022041E00126E81C7C
:109D000000F0FF00411C01F0FF01DFF87823515CF7
:109D1000DFF87023105C00F034F8DFF83C13487073
:109D2000DFF834034078361800271AE0681D10EB7E
:109D3000470000F0FF00411C01F0FF01DFF8442361
:109D4000515CDFF84023105C00F01BF8C249394435
:109D50008870A74204D2C0483844807856FA80F60A
:109D60007F1CBC42E2D2F64306F0FF06BA4820440C
:109D70008078864201D0022002E0012000E000202D
:109D8000F2BD38B50C00C0B201F09AFC05002D01FF
:109D90002000C0B201F094FC45192800C0B232BDC9
:109DA0003320AC49C8703120AA4908713020A94934
:109DB00048713120A7498871704780B5A648C0789E
:109DC0000006A549097910EB0140A349497910EB38
:109DD0000120A1498979401801F0C7F89E48C0794F
:109DE00001F0BBF99C48007A01F0C7F89A48427A22
:109DF00000231B0643EA122312069748807A0021AB
:109E0000090441EA1041000402430B439248C07A1E
:109E10000021090241EA1061000202430B438E480F
:109E2000007B002102430B438B48407B0021010251
:109E3000002002430B438848407B002101000020A2
:109E40001043194301F0ABF88348C07C00068249F7
:109E5000097D10EB01408049497D10EB01207E49CE
:109E6000897D401801F075F97B48C07D00067A496C
:109E7000097E10EB01407849497E10EB01207649BC
:109E8000897E401801F082F97448D0E9000110F091
:109E9000000011F0010100220023994207D19042F5
:109EA00005D16D48017F6C48C07E01F084F86A4896
:109EB000407F01F010F9022000F05CFF04280ED171
:109EC00000F05DFF012804D10421062000F03DFFD1
:109ED00009E06148817F062000F037FF03E00021A0
:109EE000062000F032FF5C4890F8200001F0AEFA46
:109EF0005A48D0E9000110F0000011F020010022C2
:109F00000023994225D1904223D1534890F8231041
:109F1000002001F04BF9504890F82410012001F086
:109F200045F94D4890F82510022001F03FF94A48C4
:109F300090F82610032001F039F9474890F82710CF
:109F4000042001F033F9444890F82810052001F06E
:109F50002DF901BD18B44348D0E90001424AD2E9C5
:109F60000023104319433F4AC2E9000107200021A2
:109F70003C4AD2E9002302430B433A4CC4E9002394
:109F8000364AD2E9002310431943344AC2E900019A
:109F900001200021344AC2E9000111BC70470000D1
:109FA000E0110020F0110020F0B42F48D0E90001AA
:109FB0002C4AD2E9002352F0040253F00003294C4A
:109FC000C4E90023254AD2E9002352F0040253F0E9
:109FD0000003224CC4E90023224AD2E900230240B4
:109FE0000B4000240025AB4209D1A24207D11B4AF5
:109FF000D2E9002382438B43184CC4E9002300229A
:10A0000000E0521C402A1FD200245FF00045A94204
:10A0100008D801D3A04205D200240025A94204D1CA
:10A02000A04202D10120002103E0490041EAD071A1
:10A0300040000C4BD3E9004504400D4000260027AA
:10A04000BD4201D1B442DCD0074AC2E90001F0BCF4
:10A0500070470000200E0020A00D00209811002065
:10A06000EC1100209011002088110020E411002044
:10A07000E8110020007200400440024000D000407F
:10A08000A00B0020A00A002018B58100DFF8702284
:10A09000C0F3072301F47F71D31841EA431343F05F
:10A0A000844301241C600023009302E0009C641C94
:10A0B0000094009B102BF9D3C0F30720121841EA3B
:10A0C000421141F084410020086011BDC0F3072215
:10A0D000DFF8301280008A1800F47F7040EA4210E6
:10A0E00040F08440012101607047C0F30722DFF88F
:10A0F000141280008A1800F47F7040EA421040F089
:10A1000084400021016070470138FDD170477047DD
:10A11000DFF8F8110860704770B5DFF8EC211369BB
:10A12000146A014623F4800301F0010543F400633F
:10A1300003F0010085F0010544F400641361284236
:10A1400014620ED061F0010003404FF48070906003
:10A1500013614FF400201568EE054AD4401EFAD171
:10A1600070BD080960F30A13DFF8B0011361044001
:10A17000DFF8AC0108400443C80000F0400004438D
:10A180001462480B60F34D3360F34D34402090600F
:10A19000002C47BF1462136113611462DFF884015D
:10A1A0000340DFF8840108400343C80D60F3DC542A
:10A1B000480008D5DFF8740124F48004084043F413
:10A1C0008003044301E024F0804408050BD44FF4DD
:10A1D000004057490D68EE0701D4401EFAD123F420
:10A1E000006324F40064136114621020BDE8704021
:10A1F0008AE70028B5D170BDF0B54E490A6D0B6EE7
:10A20000002B4CBF03F0700002F0300040B110286A
:10A2100047D0202847D0302847D0702848D04AE07F
:10A220000FF22C10C2F3841450F82450424C04EA6C
:10A230000306B6F1004F4FF0FF3003D0002B41D49E
:10A2400016053FD4334E376876680968C6F3042C88
:10A2500006F01F060CF1010C761C16FB0CF67600BE
:10A26000B5FBF6F5C7F30906C7F389276F4301F479
:10A270007041BF0AB1F5005F06FB057542F480022C
:10A280000DD0B1F5405F18D0B1F5804F17D0B1F5C2
:10A29000E04F16D0B1F5104F08BF284812E028480B
:10A2A00010E01B4DC2E7274DC0E747F23055BDE730
:10A2B0004FF40045BAE70020F0BD234802E02348F0
:10A2C00000E01548510217D5002B10D559000BD5C9
:10A2D0001C40B4F1004F03D0002B05D4110503D46A
:10A2E0006D00C3F3865104E0C3F3C55101E0C2F32E
:10A2F000C351491CB5FBF1F5A84288BF2846F0BD03
:10A3000000E50F4000E60F4050E00F407CE00F40BA
:10A310000024F40060E10F4040787D018FFFFF7F53
:10A3200030000080FEFF3FF80100C0070000404001
:10A3300068E10F4010E00F4000080080002D31015F
:10A3400000B4C40400093D0080F0FA02005A620221
:10A3500040420F0000201C0080841E000080250069
:10A36000999E36000040380000093D0000803E0004
:10A3700000004B00404B4C0000204E00808D5B00E5
:10A3800000C05D000080700000127A0000007D00B7
:10A3900080969800001BB7000080BB00C0E8CE008C
:10A3A000647ADA000024F4000000FA0080A81201A8
:10A3B000002D310100366E0140787D014C49FFE7E8
:10A3C000012008607047012100F01F0001FA00F031
:10A3D000484908607047012100F01F0001FA00F0B1
:10A3E00045490860704745490860704700F01F0004
:10A3F000012202FA00F0424ACB0748BF10608B07E7
:10A4000048BF90614B0748BF1062090748BF906082
:10A4100070473A4A126800F03F0002EB00123948D8
:10A4200093680340194391607047F0B5334C256839
:10A43000354C00F03F0005EB0016B7682740840656
:10A4400004D5042914BF062941F00101DDF814C028
:10A45000ACF1010E41EA0E14274307F04064B4F159
:10A46000406F04D0A40E0CFA04F4A218521E3260FD
:10A4700007F04042B2F1404F0FD0042918BF06291F
:10A4800006D140F0200005EB001000F10C0304E0C1
:10A49000920F0CFA02F003445B1E7360B760F0BDCC
:10A4A0001649096800F03F0001EB0010806800F0D9
:10A4B00007004108490004291EBF42085200062A2D
:10A4C00004BF40084000704700F0FF0110B5CB0802
:10A4D0000E4A02EB8302890001F01C0113680F246D
:10A4E0008C40000CA34388401843106010BD00004E
:10A4F00004F00F4028F00F402CF00F4008F00F4000
:10A500001CF00F40F73FFC0008C0FFFF10F50F40A4
:10A5100030B5CB4300F58064D50725684CBF0D43AB
:10A520001D40256000F58460920747BF0268114313
:10A5300001681940016030BDF0B5002400F6C47513
:10A540000126A640314211D066002F684FF0030C5F
:10A550000CFA06FC27EA0C072F60C2F34117D5F866
:10A5600000C007FA06F646EA0C062E60641C082CAA
:10A57000E6DBCC4300F5A065D6072E684CBF0E4342
:10A5800026402E6000F2045596072E684CBF0E43FD
:10A5900026402E6000F5A16556072E684CBF0E437D
:10A5A00026402E6000F5A36516072E684CBF0E43AB
:10A5B00026402E6000F23C55D2062A684CBF0A4362
:10A5C00022402A60DD0700F20C5215684CBF0D4393
:10A5D0002540156000F5A2629D0715684CBF0D432C
:10A5E0002540156000F214525D0715684CBF0D43FD
:10A5F0002540156000F21C521D0715684CBF0D4325
:10A600002540156000F244529D0515684CBF0D436E
:10A610002540156000F5A86213F4407F156814BF4B
:10A620000D432540156000F5A560002B07BF0268AB
:10A6300041EA020401680C400460F0BD00EB8100B7
:10A6400002607047012277E738B500F02DF82946FF
:10A65000204601B0BDE830400823F3E738B5044692
:10A660000D460823FFE70122FFF766FF2946204633
:10A67000BDE8384001224BE704460D46022247E779
:10A6800038B5FFF7F9FF2946204601B0BDE8304054
:10A690000823D7E738B5FFF7EFFF2946204601B07A
:10A6A000BDE830400823CDE704460D4600222FE7E1
:10A6B00010B50E4B0FF238021C68C0F30741CC40B6
:10A6C000E40746BF02EBC101496852F8311001F2BC
:10A6D0002C51020A0B680F24944000F00F00A34392
:10A6E00090401843086010BD000000006CE00F406F
:10A6F00000400040008005400050004000900540B0
:10A700000060004000A005400070004000B005401F
:10A710000040024000C005400050024000D005400B
:10A720000060024000E005400070024000F005407B
:10A7300000D0034000000640001006400010064014
:10A740000020064000200640003006400030064051
:10A7500000400640004006400050064000500640C1
:10A760000060064000600640007006400070064031
:10A7700000800640008006400090064000900640A1
:10A78000114340F8341F7047F8B504460E4617468B
:10A790001D4600F035F8B6EB071F04F1300005D276
:10A7A000016841F0200101607F0803E0026822F0A7
:10A7B00020020260F600B6FBF7F0401C400804F1EE
:10A7C00024028109116000F03F0004F128010860B3
:10A7D00004F12C0004F118010560002008602046F7
:10A7E000BDE8F240FFE700F12C010A6842F01002D8
:10A7F0000A6040F2013150F8303F0B43036070476C
:10A8000000F118010A681307FCD400F12C010A6852
:10A8100022F010020A6050F8303F02490B400360FA
:10A8200070470000FEFCFFFF11430160704750F8C5
:10A83000302F22F01002F7E7002914BF40303C30DF
:10A840000068704740F8441F704750F8482FEBE706
:10A8500080B501F0E1F902E080B501F0D9F900B16D
:10A860000120C0B202BD10B50FF2D402830852F825
:10A8700023201368C00000F01800FF248440A34385
:10A8800081401943116010BD04282B4903D1086889
:10A8900040F480300BE0052804D10A6842F400320D
:10A8A0000A607047062804D1086840F480200860D8
:10A8B00070470F2805D12148016841F0020101606D
:10A8C00070470CD90FF21413A0F110011038400991
:10A8D00053F82000012201F01F018A4002607047F6
:10A8E0000428154903D1086820F480300BE00528BE
:10A8F00004D10A6822F400320A607047062804D1A5
:10A90000086820F48020086070470F2805D10B48A4
:10A91000016821F00201016070470CD90FF2D003E9
:10A92000A0F110011038400953F82000012201F075
:10A930001F018A400260704724ED00E010E000E053
:10A940000000000018ED00E01CED00E020ED00E04C
:10A9500000E400E004E400E008E400E00CE400E0CF
:10A9600010E400E014E400E018E400E01CE400E07F
:10A9700020E400E024E400E028E400E02CE400E02F
:10A9800030E400E034E400E038E400E03CE400E0DF
:10A9900040E400E044E400E048E400E04CE400E08F
:10A9A00050E400E054E400E058E400E05CE400E03F
:10A9B00060E400E064E400E068E400E06CE400E0EF
:10A9C00070E400E074E400E078E400E07CE400E09F
:10A9D00080E400E084E400E088E400E000E100E0DE
:10A9E00004E100E008E100E00CE100E010E100E03B
:10A9F00080E100E084E100E088E100E08CE100E03B
:10AA000090E100E080B5102210218B4801F055F94B
:10AA100089480078532833D18748407844282FD17B
:10AA2000854880784B282BD18348C078452827D18A
:10AA300081480079562823D17F4840794F281FD17B
:10AA40007D48807900281BD17B48C079002817D128
:10AA50007948007A002813D17748407A00280FD12E
:10AA60007548807A00280BD17348C07A002807D136
:10AA70007148007B002803D16F48407B002803D039
:10AA8000082000F04AFD02E0082000F03FFD01BD73
:10AA90006949085C704710B504005FF0804001F020
:10AAA000ABF9012803D15FF0804001F09DF96348C4
:10AAB000444321005FF0804001F0A5F95FF0804041
:10AAC00001F08DF910BD5E4800685E49086070476E
:10AAD0005B48006870475C490968C0B208435A493E
:10AAE0000860704780B5FFF7B7FE0F20FFF7F8FE4C
:10AAF0001620FFF7F5FE5548FFF7F7FA5448FFF721
:10AB0000F4FA5448FFF7F1FA534854490860FBE758
:10AB100053480068704780B5FFF79EFE4FF4004031
:10AB20005049086001F07EF94F48FFF7F5FA01201F
:10AB3000FFF7EEFA4D48FFF7C9FA4D48FFF7C6FA9E
:10AB40004C48FFF7C3FA4C48FFF7C0FA4B48FFF7F1
:10AB5000BDFA4B48FFF7BAFA4A48FFF7B7FA01F0D7
:10AB60008FF8002803D001203D49086002E0002052
:10AB70003B490860314801F069F901F05BF90021B7
:10AB80000F20FFF770FE0F20FFF77EFE01F058F94F
:10AB9000FFF75EFE5FF07040FFF798FA5FF08040CD
:10ABA00001F02AF9012803D15FF0804001F01CF97F
:10ABB00035495FF0804001F026F95FF0804001F0F8
:10ABC00008F95FF0804001F026F95FF0804001F065
:10ABD000FFF85FF0804001F002F901BD80B5184830
:10ABE0000068184908601420FFF755FF0020164937
:10ABF000086001BD80B5144800681F2802D00120FC
:10AC000000F08BFC0E4801680E480068091A0B29F9
:10AC100003D3012000F081FC06E0094801680948DF
:10AC20000068091A0B29F8D301BD05480068401CCB
:10AC3000034908607047000074110020803801004B
:10AC4000A4120020A8120020AC120020050400F07D
:10AC5000011800F0000C00F00400FA050CED00E013
:10AC6000B012002008ED00E0800300C1000800F0F1
:10AC7000010800F0020800F0030800F0040800F0EA
:10AC8000050800F0005800F000B4C4040020DFF80C
:10AC9000C8170860DFF8C0070068C043DFF8BC17BA
:10ACA00008600020DFF8B8178870FF20DFF8B017C1
:10ACB000C8700020DFF8AC170860704780B502202C
:10ACC00000F024FCDFF898078078DFF89417C97843
:10ACD00071F0FF01C943884202D0022000F01DFC40
:10ACE000DFF874070068DFF874170968C943884201
:10ACF00002D0022000F011FCDFF864078078002801
:10AD00001CD0DFF85C078078062817D0DFF85007E2
:10AD10008078072812D0DFF84807807808280DD0FF
:10AD2000DFF83C078078042808D0DFF83407807803
:10AD3000092803D0202000F0F0FB02E0202000F0E2
:10AD4000E5FB1020FFF7C7FE01BDC0B202280CD101
:10AD5000042901D0062903D1DFF80407817008E037
:10AD60000020DFF8FC16887003E0DFF8F426C0B29C
:10AD700011547047DFF8E816C0B2085C704780B520
:10AD8000DFF8DC06807804280BD1DFF8D4060078E1
:10AD9000C0B200F095FC032801D2012002E000209F
:10ADA00000E0002002BDDFF8B8068078062801D157
:10ADB000012000E000207047DFF8A4068079072812
:10ADC00006D1DFF89C068078042801D1012000E03C
:10ADD00000207047DFF888068079082806D1DFF860
:10ADE00080068078042801D1012000E0002070470F
:10ADF000DFF86C068079092806D1DFF864068078D0
:10AE0000042801D1012000E000207047DFF850063F
:10AE10008079042806D1DFF848068078042801D11B
:10AE2000012000E000207047DFF834068078042815
:10AE300015D1DFF82C068079042810D0DFF8200621
:10AE4000807909280BD0DFF818068079082806D009
:10AE5000DFF80C068079072801D0012000E00020EF
:10AE600070470E2802D2DFF800261154704738B51B
:10AE700004000D002A00DFF8F015200000F0EEFFBE
:10AE8000DFF8DC058078062806D1DFF8E025290008
:10AE9000200001F05BF967E0DFF8C4058078042842
:10AEA00062D1DFF8BC058079072813D14FF4007018
:10AEB00000F066FB002806D0DFF8B425290020004A
:10AEC00001F044F950E0DFF8AC252900200001F042
:10AED0003DF949E0DFF888058079082805D05FF062
:10AEE000804000F04DFB002813D04FF4007000F0BC
:10AEF00047FB002806D0DFF880252900200001F05C
:10AF000025F931E0DFF874252900200001F01EF951
:10AF10002AE0DFF84C058079042813D14FF4007043
:10AF200000F02EFB002806D0DFF854252900200071
:10AF300001F00CF918E0DFF84C252900200001F0A1
:10AF400005F911E0DFF818058079092806D1DFF846
:10AF500038252900200001F0F9F805E0DFF82C255C
:10AF60002900200001F0F2F831BDDFF82415086057
:10AF70007047DFF8201508607047DFF81C1508607F
:10AF80007047DFF80C15096808407047DFF80415B2
:10AF9000096808407047DFF8000500687047DFF86F
:10AFA000FC24C2E900017047DFF8F024D2E9002355
:10AFB0001040194070470200C943D2B2C9B28A4258
:10AFC0000AD1C0B2DFF890140860DFF88C04006882
:10AFD000C043DFF8881408607047DFF87C14096804
:10AFE000C0B20843DFF870140860DFF86C04006832
:10AFF000C043DFF8681408607047DFF85C14096824
:10B00000C0B231EA0000DFF850140860DFF84804ED
:10B010000068C043DFF8441408607047DFF8381454
:10B020000968C0B208407047DFF82C040078800738
:10B0300001D50A204EE0DFF820040078C00708D5CB
:10B04000DFF814040078400701D5092042E0082009
:10B0500040E0DFF804040078800608D5DFF8F80344
:10B060000078400701D5052034E0042032E0DFF805
:10B07000E8030078400601D50B202BE0DFF8D80369
:10B08000007810F0180F08D1DFF8CC0300784007E3
:10B0900001D502201EE000201CE0DFF8BC03007890
:10B0A000000708D5DFF8B0030078400701D503207A
:10B0B00010E001200EE0DFF8A0030078C00608D5FC
:10B0C000DFF894030078400701D5072002E006204E
:10B0D00000E000207047DFF8C81308707047DFF801
:10B0E000C00300787047DFF8BC1308607047DFF8D2
:10B0F000B81308607047DFF8B00300687047DFF8E6
:10B10000AC1308607047DFF8A40300687047DFF8ED
:10B11000A01308607047DFF8980300687047DFF8F5
:10B12000941308607047DFF88C03006870470104CF
:10B1300003D4DFF88413086006E040F07F4050F449
:10B140007F00DFF8741308607047DFF86C03006855
:10B150007047DFF8681308607047DFF86413086011
:10B160007047DFF8580300687047DFF85403006841
:10B170007047DFF8501308607047DFF84803006835
:10B1800070470020DFF83C1308607047DFF8381381
:10B1900008607047DFF8341308607047DFF8280351
:10B1A00000687047DFF8240300687047DFF8202349
:10B1B000C0B211547047DFF81813C0B2085C704772
:10B1C00080B5202803D3012000F0A7F902E0DFF8C2
:10B1D0000423115401BD80B5202804D3012000F0C0
:10B1E0009CF9002002E0DFF8EC12085C02BD70B4AC
:10B1F0000400039D0120E4B2002C2CD10C00B64EBB
:10B200003678E4B2B44201D0002016E01400B24E09
:10B210007678E4B2B44201D000200EE01C00AE4EBD
:10B22000B678E4B2B44201D0002006E02C00AA4E69
:10B23000F678E4B2B44200D00020C9B2332936D146
:10B24000D2B2312A33D1DBB2302B30D1EDB2312D35
:10B250002DD101202BE00C00A04E3678E4B2B44290
:10B2600001D0002016E014009C4E7678E4B2B4427F
:10B2700001D000200EE01C00984EB678E4B2B44233
:10B2800001D0002006E02C00944EF678E4B2B442DF
:10B2900000D00020C9B2332909D1D2B2312A06D157
:10B2A000DBB2302B03D1EDB2312D00D1012070BCC7
:10B2B000704710B4884C207087484170864882706F
:10B2C0008548C37010BC704710B4844C207083480C
:10B2D0004170824882708148C37010BC7047042856
:10B2E00001D3302001E07C49085C7047042801D379
:10B2F000302001E07949085C704780B5202901D2EF
:10B30000082803D3012000F008F903E0744B400142
:10B310001844425401BD80B5202904D3012000F017
:10B32000FCF800200AE0082804D3012000F0F5F81A
:10B33000002003E06A4A40011044405C02BD694BB2
:10B340001870684841706748827070476549085CAA
:10B3500070476549086070476449086070476449F0
:10B360000860704760480068704780B5562000F05C
:10B3700018F9002802D05E48006800E0002002BDF5
:10B3800080B5562000F00DF9002802D0574800681B
:10B3900000E0002002BD811E0E2905D2554901EBB7
:10B3A000800050F8080C00E000207047821E0E2A32
:10B3B00004D2504A02EB800040F8081C7047811EFE
:10B3C0000E2905D24C4901EBC00050E9040101E00F
:10B3D000002000217047811E0E2904D2464901EB4E
:10B3E000C00040E904237047811E0E2905D243495D
:10B3F00001EB800050F8080C00E000207047821E2E
:10B400000E2A04D23D4A02EB800040F8081C704727
:10B410003B49086070473A480068704739490860FE
:10B420007047384800687047811E0E2904D236499B
:10B43000084410F8020C00E000207047821E0E2A1B
:10B4400003D2314A104400F8021C704705490860D5
:10B4500070470448006870473C12002040120020EA
:10B46000A81100209C1200205411002078F5010042
:10B4700074F0010080F5010080F0010088F5010002
:10B480008CF0010098F0010090F50100A4F001009B
:10B49000441200204C12002048120020B811002055
:10B4A000BB1200205012002054120020581200201D
:10B4B0005C1200206012002064120020681200203C
:10B4C0006C120020801200207012002074120020E4
:10B4D000B0110020BC1000207C1200207812002047
:10B4E000A00C00208412002088120020901200205E
:10B4F0008C120020B80F0020A00E0020F00F0020BA
:10B500009412002098120020641100201B49096841
:10B5100031EA000019490860704718490968084372
:10B520001649086070471549096808407047134874
:10B530000078C00701D565201EE01048007880071C
:10B5400001D5662018E00D480078000701D5682075
:10B5500012E00A480078400701D567200CE0074850
:10B560000078C00601D5692006E00448007880060E
:10B5700001D56A2000E0002070470000DC110020A7
:10B580002749496C084070472549496C08432449BC
:10B59000486470472249496C31EA000020494864F8
:10B5A0007047C0B2442802D11D48406C08E0C0B2C8
:10B5B000402802D11A48006C02E01949C0B2085C68
:10B5C00070471749085C7047602801D2144A11542B
:10B5D000704780B5C0B20200C0B260281BDAC0B2AA
:10B5E000402802D10E48016418E0C0B2442802D1BC
:10B5F0000B48416412E0C0B2382802DBC0B25428C4
:10B6000006D107488154521CC9430548815405E0BE
:10B610000348815402E00120FFF77FFF01BD0000D5
:10B62000100F0020D2B2203A22BF00FA02F100200F
:10B6300070475242D041D2F1200291404140D04067
:10B64000904041407047F0B4024610689568131866
:10B65000506803EB5004C00721D54D441FE0F0BCF7
:10B6600002F10C00704713F8017B05F8017B491EBD
:10B67000F9D1A0B1B60813F8011B06F00306032E9A
:10B6800008BF13F8016B01EB06214942801C2944D5
:10B6900005D011F8016B05F8016B401EF9D1A342EA
:10B6A000DDD013F8016B16F0030104BF13F8011B82
:10B6B000C91C30090F28DAD113F8010B0F30D6E777
:10B6C0000021C0B2B0F130010A2902D23038C0B234
:10B6D00008E0C0B2B0F14101062902D23738C0B249
:10B6E00000E00020704710F00F000149085C70472F
:10B6F000DCED0100002801D120207CE0C10701D54C
:10B70000002078E0810701D5012074E0410701D5D0
:10B71000022070E0010701D503206CE0C10601D5CD
:10B72000042068E0810601D5052064E0410601D5CA
:10B73000062060E0010601D507205CE0C10501D5C7
:10B74000082058E0810501D5092054E0410501D5C4
:10B750000A2050E0010501D50B204CE0C10401D5C1
:10B760000C2048E0810401D50D2044E0410401D5BE
:10B770000E2040E0010401D50F203CE0C10301D5BB
:10B78000102038E0810301D5112034E0410301D5B8
:10B79000122030E0010301D513202CE0C10201D5B5
:10B7A000142028E0810201D5152024E0410201D5B2
:10B7B000162020E0010201D517201CE0C10101D5AF
:10B7C000182018E0810101D5192014E0410101D5AC
:10B7D0001A2010E0010101D51B200CE0C10001D5A9
:10B7E0001C2008E0810001D51D2004E0400001D5A7
:10B7F0001E2000E01F20704730B400220023994231
:10B8000003D1904201D14020FCE10200D20701D5D2
:10B810000020F7E10200920701D50120F2E10200C9
:10B82000520701D50220EDE10200120701D50320E5
:10B83000E8E10200D20601D50420E3E1020092060D
:10B8400001D50520DEE10200520601D50620D9E12E
:10B850000200120601D50720D4E1C20501D5082057
:10B86000D0E1820501D50920CCE1420501D50A20AD
:10B87000C8E1020501D50B20C4E1C20401D50C20AA
:10B88000C0E1820401D50D20BCE1420401D50E20A7
:10B89000B8E1020401D50F20B4E1C20301D51020A4
:10B8A000B0E1820301D51120ACE1420301D51220A1
:10B8B000A8E1020301D51320A4E1C20201D514209E
:10B8C000A0E1820201D515209CE1420201D516209B
:10B8D00098E1020201D5172094E1C20101D5182098
:10B8E00090E1820101D519208CE1420101D51A2095
:10B8F00088E1020101D51B2084E1C20001D51C2092
:10B9000080E1820001D51D207CE1420001D51E208E
:10B9100078E1002801D51F2074E110F0000211F039
:10B92000010300240025AB4201D1A24201D0202016
:10B9300068E110F0000211F0020300240025AB4280
:10B9400001D1A24201D021205CE110F0000211F0EF
:10B95000040300240025AB4201D1A24201D02220E1
:10B9600050E110F0000211F0080300240025AB4262
:10B9700001D1A24201D0232044E110F0000211F0D5
:10B98000100300240025AB4201D1A24201D02420A3
:10B9900038E110F0000211F0200300240025AB4232
:10B9A00001D1A24201D025202CE110F0000211F0BB
:10B9B000400300240025AB4201D1A24201D0262041
:10B9C00020E110F0000211F0800300240025AB42BA
:10B9D00001D1A24201D0272014E110F0000211F49D
:10B9E000807300240025AB4201D1A24201D028205F
:10B9F00008E110F0000211F4007300240025AB42AE
:10BA000001D1A24201D02920FCE010F0000211F483
:10BA1000806300240025AB4201D1A24201D02A203C
:10BA2000F0E010F0000211F4006300240025AB42A6
:10BA300001D1A24201D02B20E4E010F0000211F469
:10BA4000805300240025AB4201D1A24201D02C201A
:10BA5000D8E010F0000211F4005300240025AB429E
:10BA600001D1A24201D02D20CCE010F0000211F44F
:10BA7000804300240025AB4201D1A24201D02E20F8
:10BA8000C0E010F0000211F4004300240025AB4296
:10BA900001D1A24201D02F20B4E010F0000211F435
:10BAA000803300240025AB4201D1A24201D03020D6
:10BAB000A8E010F0000211F4003300240025AB428E
:10BAC00001D1A24201D031209CE010F0000211F41B
:10BAD000802300240025AB4201D1A24201D03220B4
:10BAE00090E010F0000211F4002300240025AB4286
:10BAF00001D1A24201D0332084E010F0000211F401
:10BB0000801300240025AB4201D1A24201D0342091
:10BB100078E010F0000211F4001300240025AB427D
:10BB200001D1A24201D035206CE010F0000211F4E6
:10BB3000800300240025AB4201D1A24201D036206F
:10BB400060E010F0000211F4000300240025AB4275
:10BB500001D1A24201D0372054E010F0000211F0D0
:10BB6000807300240025AB4201D1A24201D03820CD
:10BB700048E010F0000211F0007300240025AB42F1
:10BB800001D1A24201D039203CE010F0000211F0B6
:10BB9000806300240025AB4201D1A24201D03A20AB
:10BBA00030E010F0000211F0006300240025AB42E9
:10BBB00001D1A24201D03B2024E010F0000211F09C
:10BBC000805300240025AB4201D1A24201D03C2089
:10BBD00018E010F0000211F0005300240025AB42E1
:10BBE00001D1A24201D03D200CE010F0000011F084
:10BBF000804100220023994201D1904201D03E2091
:10BC000000E03F2030BC7047012111FA00F070477E
:10BC1000EFF3108072B67047EFF3108062B6704792
:10BC200038B5044600F029F8614D0321296000F081
:10BC300024F80120E40900FA04F45E48E4430460B7
:10BC400000F01BF8002028600A20BDE83240FEF713
:10BC50005BBA10B500F011F8554C0321216000F0DB
:10BC60000CF854490020086000F007F8002020601C
:10BC70000A20BDE81040FEF747BA0A20FEF744BA92
:10BC800010B50220FEF740FA4B4C2168C807FCD4DF
:10BC9000606810F00C0F0CD14848FEF7F5F902204F
:10BCA000FEF732FA2068C107FCD4606810F00C0F70
:10BCB00001D0022010BD002010BD10B5404B8C09F2
:10BCC0001C60C1F38301920859600AD004E05968EE
:10BCD00011B91C68641C1C60521E196940F8041BD1
:10BCE000F5D110BD2DE9F84F81468A46344D68697B
:10BCF000C007FCD4DFF8CC80334F344E4FEA9A10A3
:10BD000028609408CAF38300686005D12AE0686857
:10BD100010B92968491C296030683840404505D170
:10BD20003068010404BF5046FFF77AFFD9F80000DD
:10BD30002861FFF7A2FFD5F814B05FEACB70FAD400
:10BD40005FEACB600AD530680740474504D13068C8
:10BD5000010408BFFFF77DFF58460DE0641E09F19E
:10BD60000409D4D130680740474504D13068010444
:10BD700008BFFFF76EFF6869BDE8F28F38B50D4662
:10BD80001249104B0A6804460F4802409A4205D1F6
:10BD90000968080404BF2846FFF742FF0848A909BC
:10BDA0000160C5F3830141600461406932BD000058
:10BDB000FCD00F40C0E20A4018F00A40005800F0E2
:10BDC00004F00A40000005100000FF7000E00F4082
:10BDD0001BE050F8081F41F002010160704700F5B8
:10BDE000406001210160704700F540600149016039
:10BDF0007047000051E5CC1A00F54060006801284A
:10BE000018BF002070470160704750F8081F41F0CC
:10BE100001010160704700F58360016841F48071A1
:10BE2000016070470248016841F04041016070477D
:10BE300034EF00E00748016841F0050101607047F8
:10BE40000448016841F00201016070470249401E48
:10BE50000860704710E000E014E000E070B50600F4
:10BE60000D001400002E04D14821DFF8500300F02B
:10BE7000ABF9002D04D14921DFF8400300F0A4F90B
:10BE8000002103E0685C7054491C641E002C02D041
:10BE9000685C0028F6D1002C04D000207054491CA6
:10BEA000641EF8E7300070BD2DE9F04706000C0075
:10BEB000170098460020002E04D1A821DFF8FC02CC
:10BEC00000F082F9002C04D1A921DFF8F00200F083
:10BED0007BF9002F04D1AA21DFF8E00200F074F909
:10BEE000002C00D0641E5FF000090AE0D8F80000C2
:10BEF00018F10408002C02D03070761C641E19F171
:10BF000001093878002800F01181002500E06D1C3F
:10BF1000785D252802D0785D0028F8D1AC4207D2A0
:10BF2000220039003000FFF799FF2644002406E084
:10BF30002A0039003000FFF791FF2E44641B15EBF7
:10BF400009092F4438782528DBD17F1C00252022C1
:10BF50000CE017F8010C302802D1002D00D130225E
:10BF60000A20454317F8010C303845193800471CA2
:10BF70000078253800F0BA800B380928E9D928382C
:10BF80005AD00B38B2D0401E0AD0401F08D0C01F74
:10BF900052D0C01E11D0801E46D0C01E4CD0AFE083
:10BFA000D8F8003018F10408002B02D55B420120BC
:10BFB00000E000205FF00A0C45E0D8F8001018F10E
:10BFC00004085FF0000A01E01AF1010A11F80A0002
:10BFD0000028F9D1AA4503D215EB0909B9EB0A09E2
:10BFE000544506D222003000FFF738FF26440024D3
:10BFF00016E052463000FFF731FF5644B4EB0A0416
:10C00000AA450DD2B5EB0A05AC4200D225006C4220
:10C0100002E020203070761C2800451E0028F8D150
:10C020001AEB090AD1466CE7D8F8003018F1040879
:10C030005FF00A0C002006E0D8F8003018F1040880
:10C040005FF0100C0020012102E00CFB01F16D1EDD
:10C050000CFB01FE734505D30CFB01FEBEFBFCFE91
:10C060008E45F2D0002800D06D1E00280BD0002C89
:10C0700009D0D2B2302A06D12D203070761C641E31
:10C0800019F101090020B5F1020E4FF6FE7AD645EE
:10C090000BD26D1E07E0002C02D03270761C641E9D
:10C0A00019F101096D1E002DF5D100281BD0002CBF
:10C0B00019D02D203070761C641E19F1010912E090
:10C0C000002C0CD0B3FBF1F0B0FBFCF20CFB120027
:10C0D000DFF8EC201268105C3070761C641E19F1D9
:10C0E0000109B1FBFCF10029EAD10AE7002C04D0D8
:10C0F00017F8010C3070761C641E19F1010900E775
:10C10000052C08D30522DFF8BC103000FFF7A6FE8F
:10C11000761D641F07E02200DFF8A8103000FFF74B
:10C120009DFE2644002419F10509EAE6002030703E
:10C130004846BDE8F0870CB480B50A0002AB4FF664
:10C14000FF71FFF7B1FE02BC5DF80CFB08B400B54F
:10C1500001ABFFF7A9FE5DF808FB70B406E0DBB2A7
:10C16000E4B2A34224D3401C491C521E002A22D010
:10C170000378002B02D10B78002B0CD00378413BC5
:10C180001A2B0AD2037820330C78413C1A2C06D2A1
:10C190000C78203404E000200EE00378F4E70C78FB
:10C1A00025001E00EDB2F6B2B542D8D2012003E060
:10C1B0005FF0FF3000E0002070BC70470CE9010028
:10C1C000A8F5010098F50100FEE780B5FEF7A3FC95
:10C1D00000F01CF800F0DEF800F0A0FAFEF756FDC3
:10C1E00001F01CFAFCF742F8FEF70CFCFEF7F6FC37
:10C1F00000F03AF8FCF7C7F8FEF760FD01F040FAEE
:10C2000000F09FFAFEF7F6FCF0E7000080B5012190
:10C210005548FEF719FA0A23662201215248FEF713
:10C220008BF902215048FEF70FFA0A2366220221F9
:10C230004D48FEF781F904214B48FEF705FA0A2321
:10C24000662204214848FEF777F908214648FEF7A0
:10C25000FBF90A23662208214348FEF76DF9802185
:10C260004248FEF7F1F901BD10B5414804680020CD
:10C2700040490968002901D150F001003E49096890
:10C28000002901D150F002003C490968002901D180
:10C2900050F004003A490968002901D150F0080023
:10C2A00038490968002901D050F0100000F02DF83D
:10C2B0002F4908602E4800686040334908603248C2
:10C2C00001682B48006881432F48016028480068B6
:10C2D00044402E4804602D4801682548006801400C
:10C2E0002A4801600120FEF7F6FB10BD20490968CD
:10C2F000C0B20840704725490968C0B2084070477D
:10C3000021490968C0B20840704710B401000A0012
:10C31000002304E01E4850F8230002435B1C032B5B
:10C32000F8D31B48C06802400B00002404E0184802
:10C3300050F824000340641C032CF8D31A4314481B
:10C34000C260022008E0124B03EB800353F8043C68
:10C350000F4C44F82030401E0028F4D10C480160F6
:10C36000100010BC704700000070004000500040FA
:10C37000F41100200470004008700040107000406C
:10C380002070004000520040F8110020FC110020F5
:10C390004411002010B584B0DFF85403FDF796FE79
:10C3A000DFF8500302F0B8FD40F60200FEF780F916
:10C3B00041F20200FEF77CF941F20240FEF778F903
:10C3C00034215FF04020FEF75BF902215FF040204E
:10C3D000FEF744F90220DFF820130860FDF70CFF98
:10C3E00008210191DFF814130091002300220100BD
:10C3F000C04802F069FDBF4802F088FD002000F04F
:10C40000F3F8BF48017A002002F0BAFDBC48817AF7
:10C41000012002F0B5FD0422042102A8FFF74DFC23
:10C420000298002806D00298112803D2FEF770FB6C
:10C4300001286AD10120B3490860002000E0401CB7
:10C44000072809D2AE49095CAF4A125C9142F6D086
:10C450000420FFF762F85BE05FF47430029006E0BE
:10C46000029802F093FD029810F580600290029805
:10C47000A6498842F4D3002410E06001203000F087
:10C48000B3F8A34911EB441120229D4802F090FD1E
:10C49000002802D00420FFF740F8641C102CECD3D5
:10C4A000002411E0600110F5087000F09DF8994932
:10C4B00011EB44112022924802F07AFD002802D0AC
:10C4C0000420FFF72AF8641CB4F5A07FEAD300200B
:10C4D00000F08AF820225FF47431894802F068FD88
:10C4E000002802D00420FFF718F80420FFF71BF8FB
:10C4F00000280DD1042204218248FFF7F3FB002815
:10C5000006D00420FFF709F802E002987D49086090
:10C510001FBD7C480068704711B581B04FF47A7038
:10C52000FEF7B9FA0420FEF7F1FF5FF4743404E07B
:10C53000200002F02BFD14F5806474488442F7D388
:10C54000002410E06001203000F04EF8704911EB3B
:10C55000441120226A4802F02BFD002802D004205A
:10C56000FEF7DBFF641C102CECD3002416E00198CE
:10C570004FF42052610102FB00106749081800F0D7
:10C5800033F8644911EB441120225D4802F010FD9C
:10C59000002802D00420FEF7C0FF641CB4F5A07F81
:10C5A000E5D3002000F020F820225FF474315448D5
:10C5B00002F0FEFC002802D00420FEF7AEFF0420AB
:10C5C000FEF7B1FF002806D10422042101A8FFF7DD
:10C5D00089FB002802D00420FEF79FFF01984949FB
:10C5E0000860FEF770FA13BD1CB5040000F049F8AE
:10C5F0000128FBD00020404908600520FDF784FD9C
:10C6000003213C4802F08EFC2100090C394802F05D
:10C6100089FC2100090A374802F084FC21003548D2
:10C6200002F080FC334802F098FC0128FAD0002484
:10C630001BE001A92F4802F083FC0028F9D100215A
:10C640002C4802F06FFC69462A4802F06FFC009803
:10C650002A2801D100200090009829490855254832
:10C6600002F07BFC0128FAD0641C202CE1D30520C9
:10C67000FDF74AFD0220204908600520FDF744FD32
:10C6800013BD00B583B00520FDF73EFD00201A491B
:10C6900008600520FDF738FD0521164802F042FC30
:10C6A00001A9144802F04CFC0028F9D100211148DE
:10C6B00002F038FC0F4802F050FC0128FAD069461D
:10C6C0000C4802F033FC009810F0010000900520A7
:10C6D000FDF71AFD0220084908600520FDF714FD4A
:10C6E0000098002801D0012000E000200EBD0000CD
:10C6F000001C00F0008000400840004080841E00C4
:10C70000DC100020A012002000D00300FFFF030077
:10C7100020D0030020D2030020DAFFFF80B51021D3
:10C72000DFF8180CFDF79AFF10221021DFF80C0C2F
:10C73000FDF784FF02F06EFC0120DFF8041C0860A6
:10C7400001BD80B5DFF8F80B0068002800F09A8082
:10C750004FF480400021FEF727FC0022002399427D
:10C7600005D1904203D101F0DCFE012834D1012033
:10C77000FFF7BCFD00280ED10220FFF7B7FD00280F
:10C7800009D10420FFF7B2FD002804D10820FFF7EB
:10C79000ADFD002804D00020DFF8A81B086006E0EB
:10C7A000DFF8A00B0068401CDFF8981B0860DFF87A
:10C7B000940B006840F2D171884206D30022102108
:10C7C000DFF8780BFDF73AFF10E010221021DFF8B8
:10C7D0006C0BFDF733FF09E010221021DFF85C0B32
:10C7E000FDF72CFF0020DFF85C1B0860DFF8140C5D
:10C7F0000068401CDFF80C1C08606420DFF8041C93
:10C800000968DFF8002C1268B2FBF0F200FB12108E
:10C81000002801D102F094FFDFF8EC0B007800282B
:10C8200002D100F0DCF82AE0DFF8DC0B0078012808
:10C8300002D100F049F922E0DFF8CC0B00780228A1
:10C8400002D100F093FA1AE0DFF8BC0B007803285D
:10C8500002D100F089FB12E0DFF8AC0B007804286D
:10C8600002D100F019FC0AE0DFF89C0B00780528E3
:10C8700002D100F062FC02E00120FEF74EFE04202F
:10C88000FEF729F901BDDFF8801B0870704780B5FD
:10C89000DFF8741B097803290DD1052803D2DFF8CE
:10C8A000DC1C086030E00020DFF8D01C08600120AC
:10C8B000FEF733FE28E0DFF8501B097804290DD17C
:10C8C000092803D2DFF8B41C08601DE00020DFF85F
:10C8D000AC1C08600120FEF720FE15E0DFF8281BE5
:10C8E0000978052903D1DFF8941C08600CE0DFF813
:10C8F000181B0978012903D1DFF8801C086003E0C8
:10C900000020DFF8781C086001BD10B4002309E0A6
:10C91000DFF86C2CC0B2162404FB00F42244CC5C7B
:10C92000D4545B1CCA5C002A01D0152BF0D3DFF86D
:10C93000501CC0B2162202FB00F211440022CA545D
:10C940000022DFF83C3CC0B216214843184442752F
:10C9500010BC704780B5C0B2DFF8281C0860DFF853
:10C96000240C0068002805D1DFF81C0CDFF81C1C23
:10C97000086033E0DFF80C0C0068012805D1DFF80F
:10C98000100CDFF8081C086028E0DFF8F80B0068DE
:10C99000022805D1DFF8FC0BDFF8F01B08601DE072
:10C9A000DFF8E00B0068032805D1DFF8EC0BDFF8B7
:10C9B000DC1B086012E0DFF8CC0B0068042805D10E
:10C9C000DFF8D80BDFF8C41B086007E0DFF8B80B0E
:10C9D000DFF8B81B08600120FEF79FFD01BD70B5B0
:10C9E00086B002F03EFBDFF8B81B0860002007E0CD
:10C9F000DFF8B01B095CDFF8A82B12681154401C4B
:10CA0000B0F5806FF4D3DFF8A04B00216068406878
:10CA10006268126A90476061DFF88C4B7FF07F415B
:10CA2000606840686268126A90472061DFF8784B5E
:10CA3000DFF8785BA06903F052F906005FF0FF327F
:10CA40002900200002F064FF002101917608D6F150
:10CA500005060096022190FBF1F3D3F140035FF04D
:10CA6000FF322900200002F086FF3020009033239F
:10CA7000DFF83C2B0C2102A8FFF768FBDFF8284BFE
:10CA800002ADA06903F02BF906005FF0FF32290028
:10CA9000200002F03DFF002101917608D6F1370613
:10CAA0000096022190FBF1F3D3F140035FF0FF32D7
:10CAB0002900200002F05FFFDFF8EC0A41684868B7
:10CAC000496A884706B070BD70B584B002F0C9FAF3
:10CAD000DFF8CC1A0860002005E00021DFF8C02A4A
:10CAE00012681154401CB0F5806FF6D3DFF8B84AD5
:10CAF0000021606840686268126A90476061DFF8F0
:10CB0000A84A7FF07F41606840686268126A904777
:10CB10002061DFF8A01ADFF8900A03F069F9DFF866
:10CB2000884ADFF8945AA06903F0D9F806005FF04C
:10CB3000FF322900200002F0EBFE0021019176086F
:10CB4000D6F105060096022190FBF1F3D3F14003E4
:10CB50005FF0FF322900200002F00DFFDFF85C1AC1
:10CB6000DFF8440A03F044F9DFF83C4ADFF8505A92
:10CB7000A06903F0B4F806005FF0FF32290020003E
:10CB800002F0C6FE002101917608D6F11206009649
:10CB9000022190FBF1F3D3F140035FF0FF32290053
:10CBA000200002F0E8FEDFF8004ADFF8185AA0691A
:10CBB00003F095F806005FF0FF322900200002F034
:10CBC000A7FE002101917608D6F11D0600960221EC
:10CBD00090FBF1F3D3F140035FF0FF322900200016
:10CBE00002F0C9FEDFF8C049DFF8DC59A06903F0A4
:10CBF00076F806005FF0FF322900200002F088FE80
:10CC0000002101917608D6F135060096022190FBAD
:10CC1000F1F3D3F140035FF0FF322900200002F06E
:10CC2000AAFE0220FEF7FAF900280FD0DFF87009FB
:10CC300000680290DFF8940901900020009015230D
:10CC400015222B21002002F00FFA10E00120FEF740
:10CC5000E5F9DFF84C1909680291DFF870190191C4
:10CC60000090152315222B21002002F0FDF902204F
:10CC7000FEF7D4F9DFF8281909680291DFF8501996
:10CC800001910090152315222B21162002F0ECF9BA
:10CC9000DFF80C0900680290DFF8380901900020E5
:10CCA0000090152315222B21552002F0DDF9DFF825
:10CCB000F00800680290DFF8200901900020009041
:10CCC000152315222B216B2002F0CEF9DFF8AC08DA
:10CCD0000078C0070ED5DFF8C80800680290DFF8BA
:10CCE000FC08019000200090082307220221022066
:10CCF00002F0BAF9DFF88408007880070AD500202E
:10CD000001900D2000900323012295A1DFF89808DF
:10CD100002F031FEDFF86408007840070FD5DFF835
:10CD2000800800680290DFF8B808019000200090A9
:10CD3000092307220221772002F096F90FE0DFF89D
:10CD40003C08007800070AD50020019002200090DE
:10CD50007723012283A1DFF8500802F00CFEDFF8F0
:10CD6000480841684868496A88477FBD2DE9FE4305
:10CD700002F077F9DFF82818086000200EE00021A3
:10CD8000DFF81C281268115407E0B0F5807FF6D256
:10CD90000121DFF80C2812681154401CB0F5806F97
:10CDA00007D28028F1D2FF21DFF8F427126811544E
:10CDB000F3E72020FEF732F9002802D0DFF82448FC
:10CDC0000DE04020FEF72AF9002806D0FDF7EBFF22
:10CDD000002802D1DFF8104801E0DFF810481020E9
:10CDE000FEF71CF9002802D0DFF8045809E00820FB
:10CDF000FEF714F9002802D0DFF8F85701E0DFF859
:10CE0000F8570420FEF70AF9002802D0DFF8EC6793
:10CE100001E0DFF8EC67DFF890777FF07F4178681A
:10CE200040687A68126A90477861DFF87C77002161
:10CE3000786840687A68126A90473861DFF86877E6
:10CE4000DFF83C87B86902F04AFF81465FF0FF32A5
:10CE50004146380002F05CFD002101915FEA59096A
:10CE6000D9F10309CDF80090022190FBF1F3D3F141
:10CE700040035FF0FF324146380002F07CFDDFF8EE
:10CE800020070068029001940020009015231522CD
:10CE90001421052002F0E8F8DFF80407006802908A
:10CEA000019500200090152315221421242002F062
:10CEB000DBF8DFF8EC060068029001960020009095
:10CEC000152315221421452002F0CEF8DFF8D006F4
:10CED00000680290DFF82C070190002000901523D5
:10CEE00015221421652002F0BFF8DFF8BC460021AE
:10CEF000606840686268126A90476061DFF8A8461F
:10CF00007FF07F41606840686268126A90472061E4
:10CF1000DFF89446DFF8AC56A06902F0E0FE0600A8
:10CF20005FF0FF322900200002F0F2FC00210191A5
:10CF30007608D6F134060096022190FBF1F3D3F186
:10CF400040035FF0FF322900200002F014FDDFF8FB
:10CF5000580641684868496A8847BDE8F783000079
:10CF6000540000002A0000007CB500F0EDF9DFF865
:10CF700038467FF07F41606840686268126A904777
:10CF80006061DFF824460021606840686268126AC8
:10CF900090472061DFF81046DFF8E455A06902F001
:10CFA0009EFE06005FF0FF322900200002F0B0FC78
:10CFB000002101917608D6F103060096022190FB2C
:10CFC000F1F3D3F140035FF0FF322900200002F0BB
:10CFD000D2FCDFF8D4450021606840686268126ABC
:10CFE00090476061DFF8C0457FF07F41606840682E
:10CFF0006268126A90472061002001900D20009025
:10D0000008235FF0FF32DFF80016DFF89C0502F01E
:10D01000B2FC002001901720009008235FF0FF323F
:10D02000DFF8E815DFF8800502F0A5FC002001908C
:10D030002120009008235FF0FF32DFF8D415DFF8DD
:10D04000680502F098FC002001902B200090082336
:10D050005FF0FF32DFF8BC15DFF84C0502F08BFC07
:10D06000DFF81805006800280FD000200190DFF8D5
:10D070000C0501680A204143C91C009101230122CB
:10D08000ADA1DFF8240502F076FCDFF81C0541684D
:10D090004868496A884773BD7CB500F055F9DFF8E8
:10D0A00008457FF07F41606840686268126A904777
:10D0B0006061DFF8F4440021606840686268126AC9
:10D0C00090472061DFF8E044DFF8B454A06902F033
:10D0D00006FE06005FF0FF322900200002F018FC77
:10D0E000002101917608D6F103060096022190FBFB
:10D0F000F1F3D3F140035FF0FF322900200002F08A
:10D100003AFCDFF8A4440021606840686268126A53
:10D1100090476061DFF890447FF07F41606840682D
:10D120006268126A9047206100F070F9DFF87804B5
:10D1300041684868496A884773BD2DE9F04385B066
:10D1400002A8052102F056FE00F0FEF8DFF8584470
:10D150007FF07F41606840686268126A9047606152
:10D16000DFF844440021606840686268126A9047B2
:10D170002061DFF83444DFF80854A06902F0AFFD05
:10D1800006005FF0FF322900200002F0C1FB002101
:10D1900001917608D6F103060096022190FBF1F387
:10D1A000D3F140035FF0FF322900200002F0E3FBDF
:10D1B00000244AE0DFF8F073DFF85C04052101FB8E
:10D1C00004F100EB0108B86902F089FD81465FF0C7
:10D1D000FF324146380002F09BFB01210191B6EB82
:10D1E00059060096022190FBF1F02D1A2B005FF0FA
:10D1F000FF324146380002F0BEFB25E0062C05D088
:10D20000072C03D0082C01D0092CD3D1DFF8987358
:10D210000DF10808B86902F062FD81465FF0FF3247
:10D220004146380002F074FB01210191B6EB59062A
:10D230000096022190FBF1F02D1A2B005FF0FF32D7
:10D240004146380002F097FB641C102C6CD214F09D
:10D25000030F01D110250CE014F00300012801D1C7
:10D26000302506E014F00300022801D1502500E02B
:10D270007025042C01D20F2608E0082C01D21926B3
:10D2800004E00C2C01D2232600E02D26BB480068C8
:10D29000E040C00711D5C44F7FF07F4178684068F7
:10D2A0007A68126A90477861BF4F002178684068B9
:10D2B0007A68126A9047386110E0BB4F00217868A5
:10D2C00040687A68126A90477861B74F7FF07F4173
:10D2D000786840687A68126A90473861FDF763FDA4
:10D2E00001288BD1B04FCC48052101FB04F100EBA4
:10D2F0000108B86902F0F3FC81465FF0FF32414655
:10D30000380002F005FB01210191B6EB59060096A9
:10D31000022190FBF1F02D1A2B005FF0FF32414605
:10D32000380002F028FB8FE79F4841684868496A47
:10D33000884705B0BDE8F0833E0000000050004083
:10D3400084110020D011002038B501F08AFE9449E4
:10D35000086000200CE08D4B1B680B4493F8803074
:10D360008F4C246855186355491C8029F3D3401C01
:10D37000082846D200280AD1002200218029F6D2AE
:10D38000FF23874C246855186355491CF6E701288C
:10D390000CD1802202FB00F200218029E7D2012378
:10D3A0007F4C246855186355491CF6E7022805D0C0
:10D3B000032803D0042801D005280CD1802202FBC9
:10D3C00000F200218029D2D20023754C2468551820
:10D3D0006355491CF6E706280ED1802202FB00F2B5
:10D3E00000218029C3D2694B1B685B5C6C4C2468AC
:10D3F00055186355491CF4E7802202FB00F2002116
:10D40000B3E731BDD4110020BA120020F0B58BB0C3
:10D4100001220EE0491C5A48162303FB02F318446C
:10D42000405C0028F6D102A800EB820040F8041C02
:10D43000521C092A01D20021EDE7029D03984519EB
:10D440000498451905984519069C079804190898E9
:10D4500004190998041906204543D5F180056D0883
:10D4600001263EE0504F0021786840687A68126AD1
:10D47000904778614C4F7FF07F41786840687A68C8
:10D48000126A9047386114E03C480068B042E9D124
:10D49000454F7FF07F41786840687A68126A90470C
:10D4A0007861414F0021786840687A68126A904735
:10D4B000386101200190142000902B005FF0FF32B2
:10D4C0002F48162101FB06F10144374802F053FAB8
:10D4D00002A800EB860050F8041C062000FB015552
:10D4E000761C052ED0D306204443D4F18004640872
:10D4F00005253EE02C4E0021706840687268126A73
:10D5000090477061284E7FF07F4170684068726874
:10D51000126A9047306114E018480068A842E9D1C7
:10D52000214E7FF07F41706840687268126A9047B0
:10D5300070611D4E0021706840687268126A9047E1
:10D540003061012001902020009023005FF0FF3225
:10D550000B48162101FB05F10144134802F00BFAB8
:10D5600002A800EB850050F8041C062000FB0144D3
:10D570006D1C092DD0D30BB0F0BD0000C8110020E8
:10D5800080090020CC11002090E10100C41100208E
:10D5900090DF010090E0010090DE010090DD0100CD
:10D5A000C011002088D6010028100020B0F0010032
:10D5B0000CED0100C0D50100880A002090E20100B6
:10D5C0005C0A0020460A0020720A00208CE5010057
:10D5D000CCE501004CE601000CE60100B8F00100CA
:10D5E0001CED01008CE601008CE80100CCE6010096
:10D5F0004CE701008CE701000CE701000CE801009A
:10D60000CCE701004CE8010096090020AC0900209D
:10D61000C2090020D8090020F8E4010080B50020EC
:10D62000144988610321002001F003F8042220211D
:10D630001148FEF742FB10480068002806D00E484B
:10D640000068012802D0002001F07EFB042228217E
:10D650000A48FEF732FB09480068002806D0074850
:10D660000068012802D0002001F07FFB0120014961
:10D67000086001BD700F00201C1200202012002045
:10D6800080B5DFF8DC060068002800F0498701F06B
:10D6900079FB1020FEF72AFE002804D00020DFF8D6
:10D6A000C416086003E00120DFF8B8160860DFF850
:10D6B000B8060068002812D10020DFF8A4168860A0
:10D6C000DFF8A0060068012804D10020DFF89016DA
:10D6D000486016E00120DFF88816486011E000205D
:10D6E000DFF87C164860DFF87C060068012804D16A
:10D6F0000120DFF86C16886003E00020DFF8601678
:10D700008860DFF85C064068012803D1032101200E
:10D7100000F08FFF5FF0FF30FDF705FF00280CD011
:10D72000DFF8CC06DFF838168969405C082810D08D
:10D730000321082000F07DFF0BE0DFF8B406DFF8DE
:10D7400020168969405C082803D10321012000F0DC
:10D7500070FFDFF89C06DFF808168969405C002836
:10D7600005D1DFF8FC0502F049FB00F085BEDFF8CB
:10D770008006DFF8EC158969405C012805D1DFF8E7
:10D78000E00502F05FFB00F077BEDFF86406DFF82B
:10D79000D0158969405C062805D1DFF8C40502F080
:10D7A00052FD00F069BEDFF84806DFF8B41589695C
:10D7B000405C092805D1DFF8A80502F074FE00F0EE
:10D7C0005BBEDFF82C06DFF898158969405C0728F6
:10D7D00005D1DFF88C0502F0B5FF00F04DBEDFF893
:10D7E0001006DFF87C158969405C082805D1DFF850
:10D7F000700502F0F5FF00F03FBEDFF8F405DFF83A
:10D8000060158969405C022805D1DFF8540503F0F2
:10D8100063FD00F031BEDFF8D805DFF844158969F3
:10D82000405C852805D1DFF8380503F0E3F800F007
:10D8300023BEDFF8BC05DFF828158969405C0328A2
:10D8400003D103F06DFE00F017BEDFF8A405DFF88A
:10D8500010158969405C102805D1DFF8040503F034
:10D860003AF900F009BEDFF88805DFF8F414896999
:10D87000405C112805D1DFF8E80403F0EDF900F071
:10D88000FBBDDFF86C05DFF8D8148969405C12280D
:10D8900005D1DFF8CC0403F09BFA00F0EDBDDFF812
:10D8A0005005DFF8BC148969405C132805D1DFF806
:10D8B000B00403F077FB00F0DFBDDFF83405DFF8DC
:10D8C000A0148969405C142805D1DFF8940403F0A2
:10D8D0004FFC00F0D1BDDFF81805DFF8841489692A
:10D8E000405C152803D103F0AEFC00F0C5BDDFF8A5
:10D8F0000005DFF86C148969405C1B2805D1DFF84E
:10D90000600403F073FE00F0B7BDDFF8E404DFF855
:10D9100050148969405C1C2805D1DFF8440403F0E9
:10D92000F9FE00F0A9BDDFF8C804DFF834148969F6
:10D93000405C1D2805D1DFF8280403F09DFF00F0AE
:10D940009BBDDFF8AC04DFF818148969405C1E2821
:10D9500005D1DFF80C0404F085F900F08DBDDFF887
:10D960009004DFF8FC138969405C0A2803D104F0B5
:10D97000A2FA00F081BDDFF87804DFF8E4138969CA
:10D98000405C0D2803D104F068FC00F075BDDFF8A1
:10D990006004DFF8CC138969405C0B2803D104F0E4
:10D9A00015FA00F069BDDFF84804DFF8B41389699F
:10D9B000405C0C2803D104F029FB00F05DBDDFF8CA
:10D9C0003004DFF89C138969405C0E2803D104F011
:10D9D000B9FB00F051BDDFF81804DFF88413896942
:10D9E000405C162805D1DFF8780304F019FD00F03B
:10D9F00043BDDFF8FC03DFF868138969405C172832
:10DA000003D104F0B0FD00F037BDDFF8E403DFF828
:10DA100050138969405C182805D1DFF8440304F0ED
:10DA200017FE00F029BDDFF8C803DFF83413896959
:10DA3000405C192805D1DFF8280304F099FF00F0B5
:10DA40001BBDDFF8AC03DFF818138969405C1A28A6
:10DA500003D105F005F800F00FBDDFF89403DFF8FF
:10DA600000138969405C392803D105F081F800F082
:10DA700003BDDFF87C03DFF8E8128969405C3A28CF
:10DA800003D105F0FDF800F0F7BCDFF86403DFF820
:10DA9000D0128969405C1F2805D1DFF8C40205F067
:10DAA00025FA00F0E9BCDFF84803DFF8B412896911
:10DAB000405C3B2805D1DFF8A80206F065FE00F0C7
:10DAC000DBBCDFF82C03A6498969405C3C2804D103
:10DAD000A34806F059FF00F0CFBCDFF81403A049BB
:10DAE0008969405C3D2804D19D4807F00BF800F09F
:10DAF000C3BCDFF8FC029A498969405C3E2804D126
:10DB0000974807F061F900F0B7BCDFF8E4029449E8
:10DB10008969405C402804D1914807F07AF800F008
:10DB2000ABBCDFF8CC028E498969405C3F2804D148
:10DB30008B4807F0D7F800F09FBCDFF8B4028849A3
:10DB40008969405C412804D1854807F007FA00F054
:10DB500093BCA74882498969405C432804D1804826
:10DB600007F058FE00F088BCA1487D498969405CF7
:10DB7000422804D17A4807F049FD00F07DBC9C485A
:10DB800077498969405C442804D1754808F0B2F9A6
:10DB900000F072BC964872498969405C452804D1FE
:10DBA0006F4808F014FA00F067BC91486C49896925
:10DBB000405C462804D16A4808F064FB00F05CBC75
:10DBC0008B4867498969405C472804D1644808F05C
:10DBD000C3FA00F051BC864861498969405C482815
:10DBE00004D15F4808F0FCFB00F046BC80485C496B
:10DBF0008969405C492804D1594808F07DFC00F04F
:10DC00003BBC7B4856498969405C4A2804D154484A
:10DC100008F04EFD00F030BC754851498969405C00
:10DC20004B2804D14E4808F0AEFD00F025BC7048EA
:10DC30004B498969405C4C2804D1494808F012FEE0
:10DC400000F01ABC6A4846498969405C4D2804D1F5
:10DC5000434808F075FE00F00FBC654840498969EB
:10DC6000405C4E2804D13E4808F0E8FE00F004BCB9
:10DC70005F483B498969405C4F2803D1384808F028
:10DC800067FFF9E35A4836498969405C502803D157
:10DC9000334808F0C9FFEFE3554831498969405CD2
:10DCA000512803D12E4809F065F8E5E350482C4986
:10DCB0008969405C522803D1294809F034F9DBE333
:10DCC0004B4827498969405C532803D1244809F00F
:10DCD00097F9D1E3464822498969405C542803D129
:10DCE0001F4809F0FFF9C7E341481D498969405CB5
:10DCF000552803D11A4809F063FABDE33C48184996
:10DD00008969405C562803D1154809F0C7FAB3E386
:10DD1000374813498969405C572803D1104809F0F6
:10DD200036FBA9E332480E498969405C582803D183
:10DD30000B4809F099FB9FE32D4809498969405C2C
:10DD4000592803D1064809F0F9FB95E3284804490E
:10DD50008969405C5A2809D1014809F05FFC8BE3CE
:10DD6000700F00202C1200201C1200202048DFF829
:10DD7000841B8969405C5B2802D109F0EFFC7BE3DE
:10DD80001B48DFF8701B8969405C5C2802D109F0F0
:10DD900084FD71E31648DFF85C1B8969405C5D28EF
:10DDA00002D109F0E8FD67E31148DFF8481B8969F3
:10DDB000405C5E2802D109F04CFE5DE30C48DFF8C0
:10DDC000341B8969405C242804D1DFF8280B05F056
:10DDD0003FFD51E30648DFF81C1B8969405C782849
:10DDE00004D1DFF8100B09F0B9FE45E3004801E06B
:10DDF000A0110020DFF8FC1A8969405C792804D161
:10DE0000DFF8F00A0AF00EF836E3DFF8EC0ADFF884
:10DE1000E41A8969405C7A2804D1DFF8D80A0AF04C
:10DE200044F929E3DFF8D00ADFF8C81A8969405CB1
:10DE30007B2804D1DFF8BC0A09F051FF1CE3DFF8AE
:10DE4000B80ADFF8B01A8969405C7D2804D1DFF890
:10DE5000A40A0AF078F80FE3DFF89C0ADFF8941AB6
:10DE60008969405C7C2804D1DFF8880A0AF09EF9B1
:10DE700002E3DFF8840ADFF87C1A8969405C7E28B7
:10DE800004D1DFF8700A0AF08BFAF5E2DFF8680ACD
:10DE9000DFF8601A8969405C7F2804D1DFF8540AF2
:10DEA0000AF054FBE8E2DFF8500ADFF8481A896903
:10DEB000405C802804D1DFF83C0A0AF0DFFBDBE29B
:10DEC000DFF8340ADFF82C1A8969405C812804D114
:10DED000DFF8200A0AF076FCCEE2DFF81C0ADFF851
:10DEE000141A8969405C822804D1DFF8080A0AF014
:10DEF0000BFDC1E2DFF8000ADFF8F8198969405C20
:10DF0000832804D1DFF8EC090AF058FDB4E2DFF809
:10DF1000E809DFF8E0198969405C842804D1DFF85A
:10DF2000D4090AF06FF8A7E2DFF8CC09DFF8C419CA
:10DF30008969405C252804D1DFF8B80905F018FD8F
:10DF40009AE2DFF8B409DFF8AC198969405C262849
:10DF500004D1DFF8A00905F00FFE8DE2DFF8980983
:10DF6000DFF890198969405C272804D1DFF884091B
:10DF700005F01FFF80E2DFF88009DFF87819896972
:10DF8000405C282804D1DFF86C0905F095FE73E2A7
:10DF9000DFF86409DFF85C198969405C292804D13D
:10DFA000DFF8500905F09AFF66E2DFF84C09DFF868
:10DFB00044198969405C2A2804D1DFF8380906F041
:10DFC00015F859E2DFF83009DFF828198969405C53
:10DFD0002B2804D1DFF81C0906F0FAF84CE2DFF830
:10DFE0001809DFF810198969405C2C2804D1DFF882
:10DFF000040906F087F93FE2DFF8FC08DFF8F418BF
:10E000008969405C2D2804D1DFF8E80806F046FA5B
:10E0100032E2DFF8E408DFF8DC188969405C2E287A
:10E0200004D1DFF8D00806F0CFFA25E2DFF8C808FF
:10E03000DFF8C0188969405C5F2804D1DFF8B408B4
:10E040000AF0A8FD18E2DFF8B008DFF8A81889691F
:10E05000405C202804D1DFF89C0805F041F90BE270
:10E06000DFF89408DFF88C188969405C212804D116
:10E07000DFF8800805F007FAFEE1DFF87C08DFF83A
:10E0800074188969405C222804D1DFF8680805F01B
:10E09000B3FAF1E1DFF86008DFF858188969405CED
:10E0A000232804D1DFF84C0805F034FBE4E1DFF865
:10E0B0004808DFF840188969405C602804D1DFF81F
:10E0C00034080AF0C5FED7E1DFF82C08DFF8241881
:10E0D0008969405C612804D1DFF818080AF0B3FFB1
:10E0E000CAE1DFF81408DFF80C188969405C62287F
:10E0F00004D1DFF800080AF024FFBDE1DFF8F807DB
:10E10000DFF8F0178969405C632802D10BF016F83C
:10E11000B2E1DFF8E407DFF8DC178969405C6428C6
:10E1200002D10BF065F8A7E1DFF8CC07DFF8C417E0
:10E130008969405C652802D10BF0D2F89CE1DFF8D8
:10E14000B807DFF8B0178969405C662802D10BF088
:10E1500011F991E1DFF8A007DFF898178969405CB1
:10E16000672804D1DFF88C070BF06AFA84E1DFF846
:10E170008807DFF880178969405C682804D1DFF8D8
:10E1800074070BF008FD77E1DFF86C07DFF8641720
:10E190008969405C762804D1DFF858070CF0B2F8A2
:10E1A0006AE1DFF85407DFF84C178969405C692899
:10E1B00004D1DFF840070BF067FD5DE1DFF83807B9
:10E1C000DFF830178969405C6A2804D1DFF824073A
:10E1D0000BF0FDFD50E1DFF82007DFF81817896923
:10E1E000405C6B2804D1DFF80C070BF05DFE43E1C7
:10E1F000DFF80407DFF8FC168969405C6C2804D15D
:10E20000DFF8F0060BF0BCFE36E1DFF8EC06DFF8D5
:10E21000E4168969405C6D2804D1DFF8D8060BF05C
:10E2200029FF29E1DFF8D006DFF8C8168969405CCC
:10E230006E2804D1DFF8BC060BF0A2FF1CE1DFF86A
:10E24000B806DFF8B0168969405C6F2804D1DFF8A2
:10E25000A4060CF0D1F80FE1DFF89C06DFF8941665
:10E260008969405C702804D1DFF888060CF032F927
:10E2700002E1DFF88406DFF87C168969405C7128CA
:10E2800004D1DFF870060CF0FBF9F5E0DFF8680662
:10E29000DFF860168969405C722804D1DFF8540603
:10E2A0000CF08AFAE8E0DFF85006DFF848168969D2
:10E2B000405C732804D1DFF83C060CF019FBDBE06E
:10E2C000DFF83406DFF82C168969405C742804D125
:10E2D000DFF820060CF086FBCEE0DFF81C06DFF846
:10E2E00014168969405C772804D1DFF808060CF021
:10E2F0005DF9C1E0DFF80006DFF8F8158969405CD8
:10E30000752804D1DFF8EC050CF0E8FBB4E0DFF889
:10E31000E805DFF8E0158969405C862804D1DFF85C
:10E32000D4050CF093FCA7E0DFF8CC05DFF8C415AA
:10E330008969405C872804D1DFF8B8050CF0FCFC43
:10E340009AE0DFF8B405DFF8AC158969405C8828ED
:10E3500004D1DFF8A0050CF060FD8DE0DFF8980532
:10E36000DFF890158969405C2F2804D1DFF8840517
:10E370000CF02CFE80E0DFF88005DFF87815896965
:10E38000405C302804D1DFF86C050CF064FF73E0CA
:10E39000DFF86405DFF85C158969405C312804D139
:10E3A000DFF850050CF0D6FF66E0DFF84C05DFF82B
:10E3B00044158969405C322804D1DFF838050DF036
:10E3C000F1F859E0DFF83005DFF828158969405C7D
:10E3D000332804D1DFF81C050DF012FC4CE0DFF807
:10E3E0001805DFF810158969405C342804D1DFF87E
:10E3F00004050DF053FD3FE0DFF8FC04DFF8F414F2
:10E400008969405C352804D1DFF8E8040DF008FE86
:10E4100032E0DFF8E404DFF8DC148969405C362878
:10E4200004D1DFF8D0040DF0A9FE25E0DFF8C80420
:10E43000DFF8C0148969405C372804D1DFF8B404E0
:10E440000DF032FF18E0DFF8B004DFF8A814896996
:10E45000405C382804D1DFF89C040EF0D7F90BE0BB
:10E46000DFF89404DFF88C148969405C0F2803D12D
:10E47000DFF8800402F022FA0220FDF73CFF0028BA
:10E4800022D10420FDF737FF00281DD10120FDF720
:10E4900032FF002818D10820FDF72DFF002813D1E6
:10E4A0000220FDF723FF002804D00420FDF71EFF03
:10E4B000002809D00220FDF719FF00280AD1042006
:10E4C000FDF714FF002805D0FCF702FBDFF8FC186D
:10E4D000086022E0DFF82004DFF818148969405C46
:10E4E000012815D0FCF7F4FADFF8E0180968401AA3
:10E4F000DFF8DC18884210D30120DFF8FC13DFF8C6
:10E50000F42392698854DFF8EC0301F09BFC04E0EB
:10E51000FCF7DEFADFF8B41808600220FCF7DBFA3B
:10E5200001BDDFF8B00800687047011FDFF8A828B8
:10E53000DFF8C0339B6952F82320914207D2011FB4
:10E54000DFF89428DFF8AC339B6942F82310DFF83A
:10E550008C18DFF8A023926951F82210042907D300
:10E560000321DFF87828DFF88C339B6942F8231009
:10E57000DFF86C18DFF87C23926951F82210814291
:10E5800007D3411EDFF85828DFF868339B6942F84B
:10E59000231005280DD2DFF84808DFF858138969E1
:10E5A00050F82100DFF83418DFF84823926941F869
:10E5B0002200704780B5022807D1DFF81C08DFF879
:10E5C0003413896950F8210017E0012807D1DFF8DA
:10E5D0001008DFF82013896950F821000DE00028A9
:10E5E00007D1DFF8F807DFF80C13896950F821002C
:10E5F00003E00120FCF791FF002002BD002806D1B6
:10E60000DFF8D807BB4A926940F8221010E00128D1
:10E6100006D1DFF8CC07B74A926940F8221007E02C
:10E62000022805D1DFF8B007B24A926940F82210FB
:10E63000704710B50400C9B201290DD1AD488069F9
:10E64000052805D2AB488069401CAA49886110E0C2
:10E650000120FCF762FF0CE0C9B2032903D10020BE
:10E66000A449886105E0C9B2022902D00120FCF763
:10E6700054FFA1489F4989694454FCF729FA9D49F0
:10E68000C861FCF725FA9B4908620020DFF84817AB
:10E69000984A926941F822000020DFF84017954A15
:10E6A000926941F822000020DFF83417914A9269FC
:10E6B00041F8220000208F490863E4B2122C17D0E1
:10E6C000E4B2132C14D0E4B2142C11D0E4B2152C03
:10E6D0000ED000200AE03021864A024482F824103D
:10E6E0003021844A024482F82910401C0528F2D3C4
:10E6F000E4B2012C05D100207E49486100207D490B
:10E70000086110BDDFF8DC068069002806D0DFF85C
:10E71000D4068069401EDFF8CC16886170477648C1
:10E72000DFF8C0168969405C70477348DFF8B4169B
:10E730008969084410F8010C704738B504000325B6
:10E74000641EAC4200D225000420FDF7D4FD002851
:10E7500030D00020FFF72EFFA84215D30120FFF78D
:10E7600029FFA0425BD20120FFF724FF0100491CD2
:10E770000120FFF743FF0220FFF71CFF0100491CA7
:10E780000220FFF73BFF4AE00120FFF713FFA04202
:10E7900045D20120FFF70EFF0100491C0120FFF7C1
:10E7A0002DFF0020FFF706FF0100491C0020FFF7A6
:10E7B00025FF34E00220FDF79EFD00282FD0002029
:10E7C000FFF7F8FE002815D00120FFF7F3FE002820
:10E7D00025D00120FFF7EEFE0100491E0120FFF7C2
:10E7E0000DFF0020FFF7E6FE0100491E0020FFF7A5
:10E7F00005FF14E00120FFF7DDFE00280FD0012007
:10E80000FFF7D8FE0100491E0120FFF7F7FE0220A6
:10E81000FFF7D0FE0100491E0220FFF7EFFE31BDD9
:10E820002DE9F04104000D0016001F000798C0B24A
:10E83000002807D10F20DFF8B01508600F20DFF89F
:10E84000AC150860DDF818800220FDF754FD0028A3
:10E8500009D10220FDF74AFD00280FD0DFF88C0512
:10E86000006800280AD1DFF884050068002803D179
:10E870000F20DFF8781508603C1923E00420FDF72D
:10E880003AFD002809D10420FDF730FD002819D0F9
:10E89000DFF854050068002814D1DFF84C05006843
:10E8A000002803D10F20DFF840150860A64201D2EE
:10E8B000E41B07E05FFA88F8B8F1010F01D12C00E2
:10E8C00000E03400A54207D25FFA88F8B8F1010FE2
:10E8D00001D1340000E02C00B44207D25FFA88F87E
:10E8E000B8F1010F01D12C0000E034002000BDE898
:10E8F000F0810000700F0020A011002070B404000F
:10E900000026002500E0761CA05D0028FBD1D01A6F
:10E91000864215D2D21A921B02E0605D48556D1CEA
:10E92000B542FAD3002003E020234B556D1C401C58
:10E930009042F9D3002048550CE0605D48556D1CAD
:10E94000D01A8542F9D300204855202001EB05025A
:10E9500002F8010C0020887570BC704780B5C9B200
:10E96000002905D11622DFF88814FDF777FA80E038
:10E97000C9B2012905D11622DFF87814FDF76EFA25
:10E9800077E0C9B2022905D11622DFF86C14FDF731
:10E9900065FA6EE0C9B2032905D11622DFF85C14CE
:10E9A000FDF75CFA65E0C9B2042905D11622DFF84B
:10E9B0005014FDF753FA5CE0C9B2052905D11622BF
:10E9C000DFF84014FDF74AFA53E0C9B2062905D131
:10E9D0001622DFF83414FDF741FA4AE0C9B20729DC
:10E9E00005D11622DFF82414FDF738FA41E0C9B248
:10E9F000082905D11622DFF81814FDF72FFA38E0A0
:10EA0000C9B2092905D11622DFF80814FDF726FA44
:10EA10002FE0C9B20A2905D11622DFF8FC13FDF751
:10EA20001DFA26E0C9B20B2905D11622DFF8EC1336
:10EA3000FDF714FA1DE0C9B20C2905D11622DFF842
:10EA4000E013FDF70BFA14E0C9B20D2905D1162227
:10EA5000DFF8D013FDF702FA0BE0C9B2802905DB1D
:10EA60001622DFF8C413FDF7F9F902E00120FCF7E4
:10EA700054FD01BD80B5012905D11622DFF8AC1384
:10EA8000FDF7ECF9DCE0022905D11622DFF8A0132E
:10EA9000FDF7E4F9D4E0032905D11622DFF8941339
:10EAA000FDF7DCF9CCE0042905D11622DFF8881344
:10EAB000FDF7D4F9C4E0052905D11622DFF87C134F
:10EAC000FDF7CCF9BCE0062905D11622DFF870135A
:10EAD000FDF7C4F9B4E0072905D11622DFF8641365
:10EAE000FDF7BCF9ACE0082905D11622DFF8581370
:10EAF000FDF7B4F9A4E0092907D1DFF85033DFF8B6
:10EB000050231621FDF722FB9AE00A2905D1DFF8F0
:10EB100044231621FDF71AFB92E00B2907D1DFF8F9
:10EB20003833DFF82C231621FDF710FB88E00C2981
:10EB300005D11622DFF82413FDF790F980E00D29A6
:10EB400005D11622DFF81813FDF788F978E00E29B1
:10EB500005D11622DFF80C13FDF780F970E00F29BC
:10EB600005D11622DFF80013FDF778F968E01029C7
:10EB700005D11622DFF8F412FDF770F960E01129D3
:10EB800005D11622DFF8E812FDF768F958E01229DE
:10EB900005D11622DFF8DC12FDF760F950E01329E9
:10EBA00004D11622B449FDF759F949E0142905D1D9
:10EBB000B24BB34A1621FDF7C9FA41E0152905D138
:10EBC000B04BAF4A1621FDF7C1FA39E0162905D13D
:10EBD000AD4BAB4A1621FDF7B9FA31E0172905D143
:10EBE0008B4BA74A1621FDF7B1FA29E0182905D168
:10EBF000864BA34A1621FDF7A9FA21E0192905D170
:10EC0000954B9F4A1621FDF7A1FA19E01A2905D163
:10EC10009E4B9B4A1621FDF799FA11E01B2904D15E
:10EC200016229B49FDF71AF90AE01C2904D1162285
:10EC30009849FDF713F903E016229749FDF70EF9FD
:10EC400001BD10B50400C9B2002905D116229249B0
:10EC50002000FDF703F973E0C9B2012905D116229E
:10EC60008E492000FDF7FAF86AE0C9B2022905D101
:10EC700016226C492000FDF7F1F861E0C9B20329C2
:10EC800005D1162286492000FDF7E8F858E0C9B200
:10EC9000042905D1162283492000FDF7DFF84FE053
:10ECA000C9B2052905D116227F492000FDF7D6F803
:10ECB00046E0C9B2062905D116227C492000FDF79D
:10ECC000CDF83DE0C9B2072905D1162278492000C8
:10ECD000FDF7C4F834E0C9B2082905D116227549F8
:10ECE0002000FDF7BBF82BE0C9B2092905D1162297
:10ECF00071492000FDF7B2F822E0C9B20A2905D116
:10ED000016226E492000FDF7A9F819E0C9B20B29B7
:10ED100005D1162251492000FDF7A0F810E0C9B234
:10ED20000C2905D1162266492000FDF797F807E067
:10ED30000120FCF7F2FB16223A492000FDF78EF87D
:10ED400010BD60480068704780B5002801D00128D8
:10ED500007D15C49086020215A480068FDF70EF889
:10ED600002E00120FCF7D9FB01BD80B5002801D0ED
:10ED7000012806D117490860282116480068FCF7C9
:10ED8000FDFF01BD80B50220FDF7B5FA002802D0D5
:10ED90006420164908600420FDF7ADFA002802D06F
:10EDA00064201149086011480068002804D00F4809
:10EDB0000068401E0D4908600B480068002804D018
:10EDC00009480068401E0849086001BD3012002053
:10EDD000C1D4010020120020FC10002014110020DA
:10EDE0002C110020700F0020281200202412002077
:10EDF000A0E30300C0E3030080DD0300E0E30300C1
:10EE000000E4030020E4030040E4030060E40300A6
:10EE100080E40300A0E40300C0E40300E0E4030096
:10EE200020DF030020E5030040E5030080E7030046
:10EE300000EA030020EA030060E70300C0E90300E2
:10EE4000E0E90300C0E60300E0E6030000E703009A
:10EE5000E0F20100A8EF010020F3030040E7030007
:10EE6000E0E70300C0E70300A0E7030080E8030039
:10EE700060E8030040E8030020E8030000F203001C
:10EE8000B4EF0100A0E6030000E8030080F40300F3
:10EE9000E0D20300C0F0010080E60300A0E8030018
:10EEA000C0E80300E0E8030000E9030020E90300F4
:10EEB00040E9030060E9030080E90300A0E90300E2
:10EEC000C0D403001C12002030B5002B0CBF00245E
:10EED0000424039B051DB1FBF3F12C6000239B1C54
:10EEE000B1FBF3F4641EB4F5807FF8D2049900F10D
:10EEF0001005491E2B60930103F0C00343EA04236D
:10EF000002F030021A430A43026030BD50F8041F79
:10EF100041F002010160704750F8041F21F0020126
:10EF20000160704710B500F021F81CE010B500F149
:10EF30000C0213685C07FCD508300068086010BD3F
:10EF400010B500F10C0213685C0704D508300068A6
:10EF50000860012010BD002010BD0C3000680009C1
:10EF600000F00100704740F8081F10BD00F10C02CE
:10EF700013689C07FCD57047C0B20349085C704712
:10EF8000C0B2014A11547047B81200201D4940F622
:10EF900001224A6108601C48886088688307FCD4A5
:10EFA000C868104202D04FF0FF3070470020704711
:10EFB000F0B5144C154F42F201650B46656118E03F
:10EFC000D909C901216013F07C0F01D1216B59B916
:10EFD00052B103F07C0150F8046B79181B1D0E60D0
:10EFE000121FF0E70020F0BD09492162216ACE0717
:10EFF000FCD4002AE4D1E0682842F3D04FF0FF307F
:10F00000F0BD000000D00F40020042A400D10F402C
:10F01000010042A480B5002004E00021DFF80827A9
:10F020001154401C40F205418842F6D300F0ACFB7D
:10F0300040238022DFF8F016DFF8F00600F070F8C9
:10F04000DFF8E40600F062FBDFF8E016DFF8E00628
:10F050000DF03EFEDFF8DC16DFF8D40600F0C8FE47
:10F0600001BDDFF8D40670472DE9F0470A9C0D007A
:10F07000ED0811F00701802606FB050004EB0005F2
:10F080001C00E40813F0070F00D0641C099B0898CB
:10F09000D2F18006002701E035447F1CA7423DD213
:10F0A0005FF0000C9445F7D2002814D195F800E0E9
:10F0B00093F8008018FA01F858EA0E0E85F800E07F
:10F0C00015F1800E93F80080D1F1080958FA09F87B
:10F0D0008EF800801DE095F800E093F800807FEA4C
:10F0E000080818FA01F858EA0E0E85F800E015F144
:10F0F000800E9EF8008093F800907FEA0909D1F114
:10F10000080A59FA0AF959EA080818F007088EF8A7
:10F1100000806D1C5B1C1CF1010CC3E7BDE8F0878F
:10F12000F8B504000D0016001F00002C05D140F2B8
:10F130002B11DFF80806FDF747F8002D05D14FF435
:10F140009671DFF8F805FDF73FF82820206065602C
:10F15000268167810FF23500E0600FF275002061B3
:10F160000FF2592060610FF2A520A0610FF29530D7
:10F17000E0610FF25D5020620FF291506062012059
:10F180002870A5F80160A5F80370F1BDF8B504007A
:10F190000F0015001E00002C05D14FF4C271DFF8DE
:10F1A0009C05FDF711F8B4F80100082195FBF1F179
:10F1B00000FB017704EB0700401D15F007050178FF
:10F1C0000122AA40914316FA05F50D430570F1BDE1
:10F1D0002DE9F84306000F0091469846002E05D110
:10F1E00040F2CF11DFF85405FCF7EEFF0A9D002D29
:10F1F00005D14FF4E871DFF84405FCF7E5FF0B9CFF
:10F20000002C05D140F2D111DFF83005FCF7DCFF0E
:10F21000099B0898B6F80110C91D082291FBF2F26B
:10F22000082197FBF1F109FB021906EB09014A1DC0
:10F2300017F00707D7F10707012B00F08A80042B8E
:10F2400003D0082B00F0B380B5E018F001085FFA96
:10F2500088F8B8F1000F03D0B8F1010F2ED07EE08E
:10F2600000287CD02B78DBB21B09DBB203214B4397
:10F27000E35823F07F4316780121B9408E43C3F34E
:10F28000074C44F6CD4EC3F3072849F20A7101FB3F
:10F2900008F80EFB0C8C03F0FF0341F6294101FB3B
:10F2A00003C3DB0DBB403343137039004F1E0029ED
:10F2B00001D10727521C401E0028D1D02B7813F013
:10F2C0000F0303214B436D1CE35823F07F43167853
:10F2D0000121B9408E43C3F3074C44F6CD4EC3F32E
:10F2E000072849F20A7101FB08F80EFB0C8C03F0A9
:10F2F000FF0341F6294101FB03C3DB0DBB40334350
:10F30000137039004F1E002901D10727521C401EDF
:10F31000A6E711780126BE40B143D8F107069C4606
:10F320003CFA06FC1CF0010C54F82C60BE40314342
:10F33000117039004F1E002901D10727521C18F106
:10F340000108401EB8F1080F01DA0028E1D15FF092
:10F350000008002802D02B786D1CF3E72BE02AE090
:10F360002B7803214B436D1CE35823F07F43167821
:10F370000121B9408E43C3F3074C44F6CD4EC3F38D
:10F38000072849F20A7101FB08F80EFB0C8C03F008
:10F39000FF0341F6294101FB03C3DB0DBB403343AF
:10F3A000137039004F1E002901D10727521C01009C
:10F3B000481E0029D4D1BDE8F1830000F8B504004F
:10F3C0000E0017001D00002C05D140F2B921DFF816
:10F3D0006C03FCF7F9FE0699B4F80100082295FBCE
:10F3E000F2F200FB02602044421D15F0070509E01F
:10F3F00013780120A840834311FA05F003431370EA
:10F40000521C761CB742F3DAF1BD0000F8B50400D7
:10F410000F0015001E00002C04D140F2FD21C7484A
:10F42000FCF7D2FE0698B4F80120082195FBF1F113
:10F4300002FB017704EB07014B1D002800D0FF20E1
:10F4400015F0070F19D015F00704D4F10804711B4B
:10F45000491CA14201DA741B641C012111FA04F455
:10F46000641E15F007018C401978A14304400C4339
:10F470001C701344ED1D35F007051900C90705D5AB
:10F48000711B072902DB187013440835190089071E
:10F4900015D5711B0F2912DB187003EB02010870E0
:10F4A00001EB020310350AE0187003EB020108704B
:10F4B000114408701144087001EB0203203515F166
:10F4C0001F018E42F0DA15F10F018E4206DB187033
:10F4D00003EB0201087001EB02031035E91D8E42B7
:10F4E00002DB187013440835AE420ADBFF21751B9E
:10F4F0006D1C11FA05F519782940ED4305400D43BF
:10F500001D70F1BDF8B506000C001500002E04D1E9
:10F510004FF46F718948FCF757FE002C04D140F27C
:10F52000BD318648FCF750FEB6F80110B4F9020070
:10F53000082290FBF2F2B4F9000001FB020206EB94
:10F540000200431D002D00D0FF25B4F9022012F067
:10F55000070F2DD012F00707D7F10807B4F90600FE
:10F56000801A401CB84203DAB4F90670BF1A7F1C37
:10F57000012010FA07F77F1E12F007008740B4F948
:10F5800000C01E000CE096F800E03EEA070E17EA05
:10F59000050050EA0E0E86F800E01CF1010C761C06
:10F5A000B4F904006045EEDA0B44D21D32F00702D4
:10F5B0001800C00711D5B4F90600801A07280CDB23
:10F5C000B4F90060180002E00570761C401CB4F924
:10F5D0000470B742F8DA0B440832180080071FD5D0
:10F5E000B4F90600801A0F281ADBB4F9006018007D
:10F5F00006E0058008441D804F423844761C401CBC
:10F60000B4F90470B742F4DA0B44103208E0056034
:10F61000761C401CB4F90470B742F8DA0B44083287
:10F62000B4F9060012F11F06B04203DBB4F9006022
:10F630001800EFE7B4F9060012F10F06B0421BDB29
:10F64000B4F90060180002E00580761C401CB4F993
:10F650000470B742F8DA03EB01000832B4F9006035
:10F66000030002E01D80761C5B1CB4F90470B742F5
:10F67000F8DA00EB01030832B4F90600D61DB042F7
:10F680000CDBB4F90060180002E00570761C401C29
:10F69000B4F90470B742F8DA0B440832B4F9060042
:10F6A000904214DBFF20E1888A1A521C10FA02F201
:10F6B000B4F9000007E019781140D6432E403143D9
:10F6C0001970401C5B1CB4F904108142F3DAF1BDDF
:10F6D00010B50C00002804D140F292411748FCF705
:10F6E00073FDC4F3074144F6CD42C4F3072349F246
:10F6F0000A70434302FB013104F0FF0441F6294044
:10F7000000FB0414E40D200010BD000010B504003F
:10F71000002C04D140F2B5410848FCF755FD20000B
:10F7200000F082F810BD0000A0010020541000205D
:10F730002810002090E20100A501002048E501000A
:10F7400080B5002201216548FAF778FF01220121E6
:10F750006248FAF773FFA02000F09AF8C82000F082
:10F7600097F8812000F094F81F2000F091F82F20E6
:10F7700000F08EF8402000F08BF8A62000F088F80A
:10F78000AF2000F085F801BD00B583B0FAF734FD75
:10F79000534908605348FAF799FC5348FAF796FC26
:10F7A0005248FAF793FC524852490860FF205249E8
:10F7B00008605248FFF7B0FB5148FAF779FF51480B
:10F7C000FAF776FF06214548FAF75AFF0121434828
:10F7D000FAF744FF04214C48FAF740FF08214A4851
:10F7E000FAF73CFF082001904848009000230322CC
:10F7F0003B4801684148FFF767FB4048FFF786FB3D
:10F80000042204214048FAF719FF082208213E4843
:10F81000FAF714FF324800686421B0FBF1F0FAF700
:10F8200073FCFFF78DFF07BD70B5441D002515E083
:10F830003248FFF792FB0028FAD121782F48FFF7D2
:10F8400071FB641C761C802EF2D30920FAF75CFC55
:10F85000042204212C48FAF7F1FE6D1C082D16D263
:10F8600055F0B000C0B200F013F8102000F010F80E
:10F87000002000F00DF8002204212348FAF7DEFEF4
:10F88000082208212048FAF7D9FE0026DBE770BDE0
:10F8900010B50400002208211B48FAF7CFFE002211
:10F8A00004211948FAF7CAFE1448FFF756FB00284E
:10F8B000FAD1E4B221001148FFF734FB0F48FFF7FB
:10F8C0004CFB0028FAD1042204210F48FAF7B6FEB7
:10F8D000082208210C48FAF7B1FE10BD0050024082
:10F8E000D8110020011C00F0010800F0050800F00C
:10F8F0004B434F4C2055024024550240009000409D
:10F90000020405000208050000500040002D3101EE
:10F91000FEB504460D461746002657B302AB3A46DD
:10F920002946204600F08EF818B30146A06901AAC6
:10F9300000F0EDF9B0B9A06901AA2E2100F0E7F9B5
:10F9400080B9A06901AA202100F0E1F950B90DF1B8
:10F95000060000900DF10703A06901AA0DF1050151
:10F9600000F0A8F99DF804003618029805443F1AE3
:10F97000D3E73046FEBD30B583B0069C079D05B188
:10F980000125EDB200940195C469A04737BD2DE96A
:10F99000F041054686B003A800900F4614469846ED
:10F9A0000C9EA8690DF109030DF10A020DF10B017E
:10F9B00000F080F9B5F90E10B142A1BF9DF8090021
:10F9C0003018B5F90A10884239DB0D988DF83400EB
:10F9D0002CE09DF80A0025E0B5F90C1088452EDAD8
:10F9E0000146A86902AA00F092F950B9A86902AAD2
:10F9F0002E2100F08CF920B9A86902AA202100F07C
:10FA000086F90028E5D00D999DF80B20019102F0B0
:10FA100001020092014633464246284600F027F88C
:10FA20009DF80800804404980744241A3CB104ABB4
:10FA300022463946284600F005F80028CCD106B009
:10FA4000BDE8F08138B50446084611001A4601D1D8
:10FA5000002032BD54F8203F2BB1E47903EBC403FE
:10FA60005D68A84732BD01211160007832BD2DE9E3
:10FA7000FC4F064683B0B6F90C00904216DB1046E8
:10FA80004A788018B6F9082090420FDB4FF0000941
:10FA9000CB460227D84600E001990878874280F2D9
:10FAA000E480049AB6F90E0042449042C0F2DD8030
:10FAB0000E98C0B900250A78974213DAC85D0BF199
:10FAC00018029040B0FA80FABAF1080FC8BFCBF123
:10FAD000080AD344BBF1080F554404BF4FF0000B94
:10FAE0007F1CE8D0C4E0CC5D2CB1250904F00F04E4
:10FAF0007F1C01912BE0C819BF1C4078C50000068F
:10FB0000F7D505F47E7401917AE0B6F908108C45BA
:10FB1000A1BFB6F90C106145B6F90A1088420CDB9A
:10FB20000F9951B17168736901F1040E0246614683
:10FB3000DEF80000DEF808C0E0476D1ED1460198EF
:10FB40004178894504BF08F101084FF00009002DF4
:10FB500056D000F0A9F853DBDDF80CC0012DCC44E1
:10FB600009F1010AD1DD019949788A45CDDA05EB21
:10FB700009029142B4BFA1EB090AAA46B6F90A10DC
:10FB8000884219DB0F99B9B1B6F90820614694454E
:10FB9000B8BF1146B6F90C20D444ACF101039A4227
:10FBA000C8BF1A46D6F804C0736900930346DCF850
:10FBB0000400DCF814C0E047A5EB0A05D144BEE719
:10FBC000B6F908108C45A1BFB6F90C106145B6F91D
:10FBD0000A1088420ADB7168336901F1040E02469B
:10FBE0006146DEF80000DEF808C0E047641EA94662
:10FBF00001984178894504BF08F101084FF00009D8
:10FC0000002C3FF449AF00F04FF8FFF645AFDDF8A8
:10FC10000CC0012CCC4409F10105D1DD01994A78D1
:10FC20009542CDDA04EB09018A42B6F90A10B4BF55
:10FC3000A2EB090AA246884213DBB6F90810B6F90E
:10FC40000C2075688C45A8BF6146D444ACF1010313
:10FC50009A42C8BF1A4633690093034668686D69C3
:10FC6000A847A4EB0A04D144C2E705B0BDE8F08F71
:10FC700000240191019801788F4214DAC05D0BF1E4
:10FC800018018840C043B0FA80FABAF1080FC8BF23
:10FC9000CBF1080AD344BBF1080F544404BF4FF022
:10FCA000000B7F1CE6D052E70498B6F90E104044D2
:10FCB0008142704770B582B0044625780698AE063A
:10FCC00005D500906068A4682568A84773BD0D70CD
:10FCD00061781170A1781970E178017073BD30B549
:10FCE000044683B02078202801D0E0783EBD01A8EA
:10FCF00000900DF10503FFE76068A46825680DF129
:10FD000006020DF10701A8479DF804003EBDF8B5B5
:10FD100003461878202804D158689B685C68A0477F
:10FD2000F2BD400618D50020DD880C244443A842CB
:10FD30001C442BD2A668B14203D3E768BE19B14276
:10FD400024D3401CF0E720690344A068091A53F843
:10FD50002100D0B1184414E01878040604D5D868FE
:10FD60009C681D795B7904E0D3F8C4001C1D202534
:10FD70007E23A94228BF8B4206D3491B34F81110B9
:10FD8000084441781170F2BD0020F2BDA842DAD1DA
:10FD9000FAE701460878420601D588887047800650
:10FDA00003D5486889688A68104700207047F8B50D
:10FDB0000446A069C8B1FFF7ECFF04F12602014632
:10FDC0001378256A002000E0401C98420BD235F8D9
:10FDD0003060A78CBE4202BF05EBC00677888F4219
:10FDE000F2D15070F2BD002050704FF0FF30F2BDE4
:10FDF0008161DCE700220CF0A7BF000010B5040011
:10FE00000020FCF740FDFAF763FEE169401A40F676
:10FE1000B931884215D30220FAF7ACFF002810D080
:10FE20000020A0615FF0FF30FBF77DFB002804D0CD
:10FE300003210820FEF7FDFB03E003210120FEF76C
:10FE4000F8FB10BD30B597B0050040F25A200021F4
:10FE5000F8F78FFC162110A8FBF709F8FBF79BF8C1
:10FE60000400002C0AD14FF480400021FBF79CF8DD
:10FE700000220023994201D1904243D0FAF728FE94
:10FE8000DFF8CC1A0968401A40F2F511884212D303
:10FE9000FAF71EFEDFF8B81A0860DFF8B80A006843
:10FEA000012804D10020DFF8AC1A086003E001202B
:10FEB000DFF8A01A0860DFF89C0A0068002805D166
:10FEC0004CA2162104A8FCF741F938E04FF4804019
:10FED0000021FBF769F800220023994201D19042EA
:10FEE00006D01622DFF8701A04A8FBF7B7FF26E049
:10FEF0000094DFF8683ADFF8682A162104A8FCF7B6
:10FF000025F91CE0FBF731FA002810D0FBF72DFA99
:10FF1000FBF7F0FB0190DFF84C0A0090DFF83C3A69
:10FF2000DFF8442A162104A8FCF710F907E004A81A
:10FF30000CF0B3FFFAF7CCFDDFF8141A0860FBF7FA
:10FF4000CEF8802806DBDFF8242A16210AA8FCF761
:10FF5000FDF805E0FBF768F80AA9C0B20CF024FF31
:10FF60000020FBF728F904000120FBF724F9030027
:10FF70000094DFF8FC29062102A8FCF7E7F800242A
:10FF8000FAF711FF00280DD1DFF8E8090021FBF78F
:10FF90000BF800220023994201D1904202D054F084
:10FFA000010410E0FAF7FFFE01280CD1DFF8C409C4
:10FFB0000021FAF7F9FF00220023994201D1904273
:10FFC00001D054F001045FF080500021FAF7ECFFFB
:10FFD00000220023994201D1904201D054F0020442
:10FFE0006868012802D0E868012805D154F00404AB
:10FFF00007E000BF00000000A868012801D154F00C
:020000040001F9
:1000000008040120FCF73FFC10A90C20FCF77DFC44
:1000100004A90A20FCF779FC0AA90920FCF775FC61
:1000200002A90B20FCF771FC2000FCF730FC68688B
:10003000002840F006810120FCF758F900282AD05A
:100040000820FCF753F9002825D00420FCF74EF9CE
:10005000002820D10220FCF749F900281BD1FAF72B
:1000600037FD2862FAF734FDE969401A41F2893117
:100070008842C0F0E680FAF72BFDE8610120DFF846
:10008000F8180860E868012802D10020E860D8E08C
:100090000120E860D5E00420FCF728F9002825D0ED
:1000A0000220FCF723F9002820D00120FCF71EF9DC
:1000B00000281BD10820FCF719F9002816D1FAF7FF
:1000C00007FDE861FAF704FD296A401A40F6B931E4
:1000D0008842C0F0B680FAF7FBFC28620120FBF7EB
:1000E00048F800208021F8F744FBAAE0FAF7F0FC7A
:1000F000E861FAF7EDFC2862E868002840F0938098
:100100000420FCF7FDF8002819D0FAF738FE012882
:1001100004D101210F20FEF78CFA84E0A8680128A1
:1001200004D103210920FEF784FA7CE00321092091
:10013000FEF77FFA01210220FEF77BFA73E0082028
:10014000FCF7DEF8002809D0DFF82C08006800284A
:1001500004D101210620FEF76CFA64E00120FCF7CF
:10016000CFF8002832D0DFF81008006800282DD121
:100170000220FAF753FF002855D1A868012808D0BB
:10018000FAF711FE002804D00120FAF747FF0028F3
:1001900013D00120FAF742FF002803D00120FAF71C
:1001A0002CFF05E00120FAF718FF4020FAF725FFA1
:1001B00000200121F8F7DDFA35E003210420FEF7E5
:1001C00038FA01210220FEF734FA2CE00220FCF775
:1001D00097F8002827D0A868012808D0FAF7E3FD8F
:1001E000002804D00220FAF719FF002813D00220BB
:1001F000FAF714FF002803D00220FAF7FEFE05E00C
:100200000220FAF7EAFE4020FAF7F7FE002001216B
:10021000F8F7AFFA07E003210520FEF70AFA0121FB
:100220000220FEF706FA0820FCF760F8002808D143
:100230000120FCF75BF8002803D10020DFF8381715
:10024000086017B030BD00B587B042200021F8F734
:1002500090FA1622DFF824176846FBF7FFFD69467F
:100260000020FCF752FBFAF7DFFE6946C0B20CF043
:100270009BFD0220FCF707FB69460920FCF745FBC4
:100280005620FBF78EF902280ED04020FAF7C6FE62
:10029000002809D02020FAF7B0FE4020FAF7ADFE82
:1002A00000200121F8F765FA0120FCF729F8002861
:1002B00045D0FAF778FD012810D12020FAF7AEFEDC
:1002C000002803D02020FAF798FE02E02020FAF759
:1002D00084FE00200121F8F74CFA26E04020FAF7CE
:1002E0009DFE002815D1DFF89806006801281CD073
:1002F0002020FAF793FE002803D02020FAF77DFE95
:1003000002E02020FAF769FE00200121F8F731FA17
:100310000BE0DFF86C060068012806D04020FAF7F1
:100320006CFE00200121F8F724FAFAF7D1FBDFF880
:10033000541608600020DFF848160860B1E001207C
:10034000FBF7D4FF002845D05620FBF72AF90228F6
:1003500036D15720FBF725F9012831D1DFF82006E7
:100360000068002840F09D80FAF7B2FBDFF8141611
:100370000968401A40F6B9318842C0F092800120E5
:10038000DFF8FC1508604020FAF748FE002803D18A
:100390004020FAF722FE02E04020FAF72EFE20204D
:1003A000FAF72BFE0820FAF728FE1020FAF725FEB0
:1003B0000420FAF722FE00200121F8F7DAF970E0B4
:1003C0000020DFF8BC150860FAF782FBDFF8B415EF
:1003D000086066E00220FBF793FF002838D0FAF7A8
:1003E000E2FC01280FD10820FAF718FE002803D1FB
:1003F0000820FAF7F2FD02E00820FAF7FEFD1020CF
:10040000FAF7FBFD1FE00820FAF708FE002808D1E4
:100410001020FAF703FE002803D10820FAF7DDFDCB
:1004200011E00820FAF7FAFD002806D01020FAF7AC
:10043000D4FD0820FAF7E1FD05E01020FAF7DDFD14
:100440000820FAF7DAFD00200121F8F792F928E0F8
:100450000420FBF755FF002810D00420FAF7DEFD3A
:10046000002803D00420FAF7C8FD02E00420FAF7C0
:10047000B4FD00200121F8F77CF912E00820FBF719
:100480003FFF002808D003210120FEF7D2F800200A
:10049000DFF8EC14086004E0FAF71AFBDFF8E41464
:1004A000086007B000BD70B5BEB00500582000213F
:1004B000F8F75FF95620FBF774F8002809D05720A9
:1004C000FBF76FF8012804D101240A20FEF72DF86C
:1004D00003E000240920FEF728F81622DFF8A8140C
:1004E0006846FBF7BBFC69460020FCF70EFA0320C8
:1004F000FCF7C9F90420FCF72DFADFF89034DFF897
:100500009024162106A8FBF721FEDFF88834DFF8D7
:10051000882416210DF12E00FBF718FEDFF87C343D
:10052000DFF87C24162111A8FBF710FEDFF87434E5
:10053000DFF8742416210DF15A00FBF707FEDFF8EF
:100540006C34DFF86C2416211CA8FBF7FFFDDFF8E4
:100550006434DFF8642416210DF18600FBF7F6FD04
:10056000DFF85834DFF85824162127A8FBF7EEFDF2
:10057000DFF85034DFF8502416210DF1B200FBF7FC
:10058000E5FD002C0ED1DFF84434DFF844241621B9
:1005900032A8FBF7DBFD91A216210DF1DE00FBF77F
:1005A000D5FD10E0DFF82C34DFF82424162132A822
:1005B000FBF7CCFDDFF81434DFF81C2416210DF115
:1005C000DE00FBF7C3FD0020FDF7F4FF401CFCF745
:1005D0005EF90220FDF7EEFF060006A8162101FBDA
:1005E00006F101440120FCF790F906A8162101FB51
:1005F00006F1084410F116010220FCF786F906A85E
:10060000162101FB06F1084410F12C010320FCF730
:100610007CF906A91620464301EB060010F14201C1
:100620000420FCF772F90820FBF76AFE002874D05A
:100630000120FDF7BFFF002804D101213920FDF77B
:10064000F8FF7DE0012813D1A868012802D068696D
:10065000002808D101211F20FDF7EBFF0121022016
:10066000FDF7E7FF6CE001211F20FDF7E2FF67E0E7
:10067000022818D1FAF797FB012804D101210B2099
:10068000FDF7D7FF5CE04FF40070FAF779FF002820
:1006900004D001210B20FDF7CCFF51E001210A20FD
:1006A000FDF7C7FF4CE0032804D101210E20FDF720
:1006B000C0FF45E0042804D101211620FDF7B9FF51
:1006C0003EE0052804D101211B20FDF7B2FF37E0F1
:1006D000062808D1FAF7A8FB002831D101212F20E4
:1006E000FDF7A7FF2CE0072804D101218520FDF7A5
:1006F000A0FF25E008280BD1012C04D101217C208A
:10070000FDF797FF1CE001218620FDF792FF17E01F
:1007100001218620FDF78DFF12E00120FBF7F0FD9F
:10072000002804D003210120FDF783FF08E0002CFE
:1007300003D10920FEF701F802E00A20FDF7FDFFD2
:100740003EB070BD00B587B078200021F8F711F8F1
:10075000162290496846FBF781FB69460020FCF7AA
:10076000D4F80420FCF78FF80120FCF7F3F81622E8
:100770009A496846FBF772FB69460120FCF7C5F809
:10078000162297496846FBF769FB69460520FCF786
:10079000BCF812A10220FCF7B8F810A10320FCF766
:1007A000B4F80EA10420FCF7B0F80CA10620FCF769
:1007B000ACF80AA10720FCF7A8F808A10820FCF76C
:1007C000A4F80020FCF763F80820FBF799FD002847
:1007D00001D0FDF797FF07B000BD0000000000004A
:1007E00010B588B0040002200021F7F7C2FF1622DE
:1007F0007C4901A8FBF732FB01A90020FCF785F832
:10080000FAF795FE0090554B774A162101A8FBF7A1
:100810009DFC0420FCF737F80020FCF79BF801A9A9
:100820000120FCF772F80020FCF731F847A1022004
:10083000FCF76BF845A10320FCF767F843A10420FF
:10084000FCF763F841A10520FCF75FF83FA1062003
:10085000FCF75BF83DA10720FCF757F83BA1082007
:10086000FCF753F80420FBF741FD002810D00220CC
:10087000FBF73CFD00280BD00120FBF737FD0028DB
:1008800006D10820FBF732FD002801D1FAF72AF93A
:10089000FAF71EF9E169401A41F2893188420BD317
:1008A0001020FAF740FE002806D12020FAF73BFE80
:1008B000002801D1FAF716F908B010BD00B593B0C1
:1008C000162231490CA8FBF7C9FA1622474906A897
:1008D000FBF7C4FA464A16216846FBF737FC0420AA
:1008E000FBF7D1FF0120FCF735F80CA90020FCF73D
:1008F0000CF806A90120FCF708F869460520FCF76A
:1009000004F812A10220FCF700F810A10320FBF765
:10091000FCFF0EA10420FBF7F8FF0CA10620FBF75B
:10092000F4FF0AA10720FBF7F0FF08A10820FBF75E
:10093000ECFF0020FBF7ABFF0820FBF7E1FC0028F1
:1009400001D0FDF7DFFE13B000BD00000000000085
:10095000081200200412002020E3030020E5030019
:10096000ACEE01002CEA0100B8EE0100E0F101005C
:10097000C4EE0100299E3F6C0C12002020EC030005
:100980001012002014120020C0D9030020D203004E
:10099000E8F1010040D20300F0F1010060D2030051
:1009A000F8F1010080D2030000F20100A0D20300A0
:1009B00008F20100C0D2030010F20100E0D20300EF
:1009C00018F2010000D3030020F2010020D303003D
:1009D00028F2010020F6030030F20100E0EB0300F2
:1009E00000EC030000D0030038F2010040F70300E0
:1009F00040F2010010B592B0040002200021F7F788
:100A0000B8FE0220FDF791FD1622DFF8B01B684604
:100A1000FBF724FA69460020FBF777FF0320FBF77A
:100A200032FF0420FBF796FFDFF8943BDFF8942BAE
:100A3000162106A8FBF78AFBDFF88C3BDFF88C2B2E
:100A400016210DF12E00FBF781FB06A90120FBF713
:100A50005CFF0DF12E010220FBF757FF7DA1032063
:100A6000FBF753FF7BA10420FBF74FFF0020FDF7AE
:100A7000A1FD401CFBF70BFF0820FBF741FC002801
:100A80001CD00120FDF796FD00280CD160690128DB
:100A900004D101211020FDF7CCFD1AE0012107202F
:100AA000FDF7C7FD15E0012804D101211120FDF754
:100AB000C0FD0EE00120FAF730FD0AE00120FBF74F
:100AC0001FFC002802D0FDF71DFE02E00220FDF70A
:100AD00034FE12B010BD30B587B0050002200021F1
:100AE000F7F747FE1622DFF8E81A01A8FBF7B6F978
:100AF00001A90020FBF709FF0420FBF7C4FE042036
:100B0000FBF728FFB1A10120FBF7FFFEAFA10220F8
:100B1000FBF7FBFEADA10320FBF7F7FEABA1042022
:100B2000FBF7F3FE4BA10520FBF7EFFE49A10620E2
:100B3000FBF7EBFE47A10720FBF7E7FE45A10820E6
:100B4000FBF7E3FE0020FBF7A2FE286B284490F899
:100B500024008DF8000000208DF80100286B01288A
:100B600004D169460120FBF7D0FE16E0286B02286D
:100B700004D169460220FBF7C8FE0EE0286B03286B
:100B800004D169460320FBF7C0FE06E0286B042869
:100B900003D169460420FBF7B8FE2C6B0220FBF75B
:100BA000AAFB00281BD0002C03D1286B401C286313
:100BB0004DE005EB040090F82400392809DA05EB34
:100BC000040090F82400401C05EB040181F8240087
:100BD0003DE0302005EB040181F8240037E00420DB
:100BE000FBF789FB00281BD0002C03D1286B401C8D
:100BF00028632CE005EB040090F82400312809DB81
:100C000005EB040090F82400401E05EB040181F878
:100C100024001CE0392005EB040181F8240016E0D3
:100C20000820FBF76DFB00280AD0042C04D1022118
:100C30001220FDF7FEFC0AE0286B401C286306E04A
:100C40000120FBF75DFB002801D0FDF75BFD07B03D
:100C500030BD00000000000030B587B00500022064
:100C60000021F7F786FD1622DFF8681901A8FBF7C7
:100C7000F5F801A90020FBF748FE0420FBF703FE6E
:100C80000420FBF767FE51A10120FBF73EFE4FA1B8
:100C90000220FBF73AFE4DA10320FBF736FE4BA1E5
:100CA0000420FBF732FEBDA10520FBF72EFEBBA101
:100CB0000620FBF72AFEB9A10720FBF726FEB7A105
:100CC0000820FBF722FE0020FBF7E1FD2C6B05EB73
:100CD000040090F824008DF8000000208DF8010039
:100CE000012C04D169460120FBF70FFE13E0022C12
:100CF00004D169460220FBF708FE0CE0032C04D166
:100D000069460320FBF701FE05E0042C03D1694688
:100D10000420FBF7FAFD0220FBF7EDFA00281BD0B8
:100D2000002C03D1286B401C28634DE005EB040028
:100D300090F82400392809DA05EB040090F8240023
:100D4000401C05EB040181F824003DE0302005EB58
:100D5000040181F8240037E00420FBF7CCFA0028D6
:100D60001BD0002C03D1286B401C28632CE005EB22
:100D7000040090F82400312809DB05EB040090F80A
:100D80002400401E05EB040181F824001CE03920FA
:100D900005EB040181F8240016E00820FBF7B0FA07
:100DA00000280AD0042C04D102211320FDF741FCB5
:100DB0000AE0286B401C286306E00120FBF7A0FA3C
:100DC000002801D0FDF79EFC07B030BD2A000000CE
:100DD00030B587B0050002200021F7F7CAFC1622C3
:100DE000DFF8F41701A8FBF739F801A90020FBF799
:100DF0008CFD0420FBF747FD0420FBF7ABFD68A149
:100E00000120FBF782FD66A10220FBF77EFD64A1B5
:100E10000320FBF77AFD62A10420FBF776FD5FA1BA
:100E20000520FBF772FD5DA10620FBF76EFD5BA1BF
:100E30000720FBF76AFD59A10820FBF766FD00209B
:100E4000FBF725FD2C6B05EB040090F829008DF8CD
:100E5000000000208DF80100012C04D1694601201A
:100E6000FBF753FD13E0022C04D169460220FBF787
:100E70004CFD0CE0032C04D169460320FBF745FD33
:100E800005E0042C03D169460420FBF73EFD022057
:100E9000FBF731FA00281BD0002C03D1286B401C33
:100EA000286379E005EB040090F82900392809DA75
:100EB00005EB040090F82900401C05EB040181F8C3
:100EC000290069E0302005EB040181F8290063E086
:100ED0000420FBF710FA00281BD0002C03D1286B4C
:100EE000401C286358E005EB040090F829003128E5
:100EF00009DB05EB040090F82900401E05EB040116
:100F000081F8290048E0392005EB040181F8290027
:100F100042E00820FBF7F4F9002836D0042C30D149
:100F200095F82A0095F82510884225D195F82B00D0
:100F300095F8261088421FD195F82C0095F82710B7
:100F4000884219D195F82D0095F82810884213D1C0
:100F500002211420FDF76DFB95F82D3095F82C201B
:100F600095F82B1095F82A00FAF7A3F900204FF412
:100F70008071F7F7FEFB0FE002211220FDF759FB0D
:100F80000AE0286B401C286306E00120FBF7B8F953
:100F9000002801D0FDF7B6FB07B030BD000000000F
:100FA0002A00000030B587B0050002200021F7F7C5
:100FB000E0FB1622DFF8241601A8FAF74FFF01A97B
:100FC0000020FBF7A2FC0420FBF75DFC0420FBF7EC
:100FD000C1FCBFA10120FBF798FCBDA10220FBF7DB
:100FE00094FCBBA10320FBF790FCB9A10420FBF704
:100FF0008CFCB8A10520FBF788FCB6A10620FBF706
:1010000084FCB4A10720FBF780FCB2A10820FBF709
:101010007CFC0020FBF73BFC2C6B05EB040090F8FC
:1010200029008DF8000000208DF80100012C04D16A
:1010300069460120FBF769FC13E0022C04D16946E4
:101040000220FBF762FC0CE0032C04D1694603206C
:10105000FBF75BFC05E0042C03D169460420FBF799
:1010600054FC0220FBF747F900281BD0002C03D1C9
:10107000286B401C286379E005EB040090F82900F8
:10108000392809DA05EB040090F82900401C05EB2B
:10109000040181F8290069E0302005EB040181F8A2
:1010A000290063E00420FBF726F900281BD0002C60
:1010B00003D1286B401C286358E005EB040090F82E
:1010C0002900312809DB05EB040090F82900401EB7
:1010D00005EB040181F8290048E0392005EB040103
:1010E00081F8290042E00820FBF70AF9002836D0F1
:1010F000042C30D195F82A0095F82510884225D186
:1011000095F82B0095F8261088421FD195F82C00F1
:1011100095F82710884219D195F82D0095F82810D8
:10112000884213D102211520FDF783FA95F82D305E
:1011300095F82C2095F82B1095F82A00FAF7C4F8AA
:1011400000204FF40071F7F714FB0FE00221132089
:10115000FDF76FFA0AE0286B401C286306E00120C7
:10116000FBF7CEF8002801D0FDF7CCFA07B030BD70
:1011700010B586B0040002200021F7F7FAFA162213
:10118000DFF84C146846FAF769FE69460020FBF761
:10119000BCFB0420FBF777FB0120FBF7DBFB002007
:1011A000FAF79DF894F82A10C0B2814222D10120AA
:1011B000FAF795F894F82B10C0B281421AD10220A8
:1011C000FAF78DF894F82C10C0B2814212D10320A6
:1011D000FAF785F894F82D10C0B281420AD1162290
:1011E000DFF8FC136846FAF739FE69460120FBF781
:1011F0008CFB03E037A10120FBF787FB35A1022020
:10120000FBF783FB33A10320FBF77FFB31A1042015
:10121000FBF77BFB2FA10520FBF777FB2DA1062019
:10122000FBF773FB2BA10720FBF76FFB29A108201D
:10123000FBF76BFB0820FBF763F8002801D0FDF7F4
:1012400061FA06B010BD00B587B002200021F7F7A3
:1012500090FA1622DFF87C136846FAF7FFFD69461C
:101260000020FBF752FB0420FBF70DFB0120FBF7EE
:1012700071FB1622DFF868136846FAF7EFFD69463E
:101280000120FBF742FB13A10220FBF73EFB11A15B
:101290000320FBF73AFB0FA10420FBF736FB0DA15F
:1012A0000520FBF732FB0BA10620FBF72EFB09A163
:1012B0000720FBF72AFB07A10820FBF726FB0820E5
:1012C000FBF71EF8002801D0FDF71CFA07B000BD9F
:1012D0002A0000000000000030B587B005000220A1
:1012E0000021F7F746FA1622BE4901A8FAF7B6FD23
:1012F00001A90020FBF709FB0420FBF7C4FA042036
:10130000FBF728FBABA10120FBF7FFFAA9A1022004
:10131000FBF7FBFAA7A10320FBF7F7FAA5A104202E
:10132000FBF7F3FAA4A10520FBF7EFFAA2A1062030
:10133000FBF7EBFAA0A10720FBF7E7FA9EA1082034
:10134000FBF7E3FA0020FBF7A2FA2C6B05EB040095
:1013500090F824008DF8040000208DF80500012C81
:1013600004D101A90120FBF7D0FA13E0022C04D12B
:1013700001A90220FBF7C9FA0CE0032C04D101A952
:101380000320FBF7C2FA05E0042C03D101A90420D5
:10139000FBF7BBFA0220FAF7AEFF00281ED0002CA4
:1013A00007D1286B401C2863296B0020FDF726F924
:1013B00014E005EB040090F82400392809DA05EB65
:1013C000040090F82400401C05EB040181F824007F
:1013D00004E0302005EB040181F824000420FAF732
:1013E0008AFF00281ED0002C07D1286B401C2863E0
:1013F000296B0020FDF702F914E005EB040090F8DA
:101400002400312809DB05EB040090F82400401E7D
:1014100005EB040181F8240004E0392005EB040108
:1014200081F824000820FAF76BFF00286DD0042C07
:1014300063D195F82800009095F8273095F826207C
:1014400095F825100120F9F7D2FE286195F82800BB
:10145000009095F8273095F8262095F82510002063
:10146000F9F7C5FE68612869012802D0686901287A
:101470003ED1FDF747F9FDF752F904001F2C09D1C1
:101480002869012806D16869002803D102210720B4
:10149000FDF7CFF8042C14D103210120FDF7C9F882
:1014A0000120F9F7BBFD002803D00120F9F7A5FDC5
:1014B00002E00120F9F791FD00200121F7F759F929
:1014C0002CE0052C2AD103210120FDF7B2F80220DF
:1014D000F9F7A4FD002803D00220F9F78EFD02E001
:1014E0000220F9F77AFD00200121F7F742F915E013
:1014F00002210320FDF79DF810E0286B401C2863B3
:10150000296B0020FDF77AF808E00120FAF7F8FED1
:10151000002803D003210120FDF78BF807B030BD70
:1015200000B587B002200021F7F723F916222349DE
:101530006846FAF793FC69460020FBF7E6F90420B9
:10154000FBF7A1F90120FBF705FA162226496846A8
:10155000FAF784FC69460120FBF7D7F916A10220AF
:10156000FBF7D3F914A10320FBF7CFF912A1042054
:10157000FBF7CBF910A10520FBF7C7F90EA1062058
:10158000FBF7C3F90CA10720FBF7BFF90AA108205C
:10159000FBF7BBF90120FAF7B3FE002804D10820BD
:1015A000FAF7AEFE002803D003210120FDF741F831
:1015B00007B000BD2A0000000000000000D30300B7
:1015C00040EE030088F3010060EE030090F3010099
:1015D00080EE0300C0EE0300A0EE0300E0EE030087
:1015E00000EF030060EC030040EC030010B598B07E
:1015F000040040200021F7F7BCF8DFF870379BA209
:1016000016216846FAF7A2FD69460020FBF77DF92E
:101610000320FBF738F90420FBF79CF90020FCF7C6
:10162000C9FF401CFBF733F9DFF84437DFF84427E4
:10163000162106A8FAF78AFDDFF83C37DFF83C27C9
:1016400016210DF12E00FAF781FDDFF83437DFF8AF
:101650003427162111A8FAF779FD06A90120FBF716
:1016600054F90DF12E010220FBF74FF911A90320C7
:10167000FBF74BF97EA10420FBF747F90120FAF7AD
:101680003FFE002802D0FDF73DF841E00820FAF7C0
:1016900037FE002839D00120FCF78CFF002810D13C
:1016A00001211D20FCF7C5FF0220F9F784FD6063CE
:1016B0000420F9F780FDA0630520F9F77CFDE063C5
:1016C0001EE001280CD101211C20FCF7B2FF0120F3
:1016D000F9F771FD60630020F9F76DFDA0630FE07D
:1016E00002280DD101211E20FCF7A3FF0120F9F7EC
:1016F00047FF002802D00120606301E00020606302
:101700000020DFF88416086002E00320FDF715F8DA
:1017100018B010BD10B588B004001622DFF85816B6
:1017200002A8FAF79BFB02A90020FBF7EEF80420C1
:10173000FBF7A9F80420FBF70DF9636BDFF84C26E3
:10174000032102A8FAF702FD02A90120FBF7DDF848
:1017500048A10220FBF7D9F8A36BDFF8302603215C
:1017600002A8FAF7F3FC02A90320FBF7CEF840A188
:101770000420FBF7CAF83EA10520FBF7C6F83CA100
:101780000620FBF7C2F83AA10720FBF7BEF838A104
:101790000720FBF7BAF8DFF8F0050068FBF777F8E9
:1017A0000120FAF7ADFD002802D0FCF7ABFF5BE0AB
:1017B0000820FAF7A5FD00281BD0DFF8CC0500684B
:1017C00003280ED1616B0120F9F7F0FCA16B00201A
:1017D000F9F7ECFC00202021F6F7CBFFFCF792FF95
:1017E00042E0DFF8A4050068401CDFF89C150860A3
:1017F0003AE0DFF894050068002807D1DFF8880593
:101800000068401CDFF8801508602DE0DFF87805DF
:10181000006801280BD101200190012000900123D4
:1018200000221721606BFCF7FBFF60631CE0DFF810
:1018300058050068022807D1DFF84C050068401CF5
:10184000DFF8441508600FE0DFF83C050068032866
:101850000AD10120019001200090012300223B21A8
:10186000A06BFCF7DDFFA06308B010BD257300007E
:10187000000000003A000000F0B597B0040008A88E
:10188000DFF80C1538220BF08BFB1622DFF8E01482
:1018900002A8FAF7E3FA02A90020FBF736F80420C1
:1018A000FAF7F1FF0420FBF755F8DFF8DC040068D5
:1018B00000281AD1E06B0190A06B0090636BDFF8F9
:1018C000D424092102A8FAF741FC02A90120FBF760
:1018D0001CF877A10220FBF718F875A10320FBF78D
:1018E00014F873A10420FBF710F8DFF89C040068DB
:1018F000012820D1636BDFF89424032102A8FAF7B2
:1019000025FC02A90120FBF700F8E06B0090A36B17
:10191000DFF88424072102A8FAF718FC02A90220A4
:10192000FAF7F3FF62A10320FAF7EFFF60A10420AA
:10193000FAF7EBFF4AE0DFF850040068022825D1EF
:10194000636BDFF85824042102A8FAF7FFFB02A911
:101950000120FAF7DAFFA36BDFF83024032102A895
:10196000FAF7F4FB02A90220FAF7CFFFE36BDFF8E6
:101970003024042102A8FAF7E9FB02A90320FAF7B0
:10198000C4FF4BA10420FAF7C0FF1FE0A06B00903A
:10199000636BDFF81024062102A8FAF7D7FB02A92F
:1019A0000120FAF7B2FFAEA10220FAF7AEFFE36B17
:1019B000DFF8D823032102A8FAF7C8FB02A9032005
:1019C000FAF7A3FF3AA10420FAF79FFF616B072201
:1019D000B1FBF2F002FB101094F83C1011F0030F71
:1019E0000BD1A16B012902D0A16B022905D108A955
:1019F000626B01EB8201C96A05E008A9A26B01EBE9
:101A0000820151F8041CE36B1C25E66B1C27B3FB19
:101A1000F5F205FB1232B6FBF7F307FB136612EB88
:101A2000960208181018801D0721B0FBF1F201FB87
:101A30001200002806D10422DFF86C1302A8FAF77E
:101A40000DFA3AE0012806D10422DFF8601302A85B
:101A5000FAF704FA31E0022806D10422DFF8501325
:101A600002A8FAF7FBF928E0032806D10422DFF8E0
:101A7000441302A8FAF7F2F91FE0042806D1042261
:101A8000DFF8341302A8FAF7E9F916E0052806D1C1
:101A90000422DFF8281302A8FAF7E0F90DE006287F
:101AA00008D10422C64902A8FAF7D8F905E000BF18
:101AB000000000000120F9F730FD00208DF80B0038
:101AC000606B00280AD0A06B002807D0E06B0028CC
:101AD00004D002A90520FAF718FF03E0A1A1052010
:101AE000FAF713FF9FA10620FAF70FFF9DA1072029
:101AF000FAF70BFF9BA10820FAF707FFA24800683E
:101B0000FAF7C5FE0120FAF7FBFB002802D0FCF72C
:101B1000F9FDA3E00820FAF7F3FB002865D09A4806
:101B20000068032830D1606B1D2808D1A06B022803
:101B300005D194F83C0010F0030F40F08F80022094
:101B4000F9F739FB616B81420BD10420F9F733FBC4
:101B5000A16B814205D10520F9F72DFBE16B814294
:101B60000FD0616B0220F9F721FBA16B0420F9F77C
:101B70001DFBE16B0520F9F719FB00202021F6F78A
:101B8000F8FDFCF7BFFD69E07F480068022826D118
:101B9000A06B022808D1606B1E285FD27A480068CB
:101BA000401C7949086059E0A06B042808D0A06B5C
:101BB000062805D0A06B092802D0A06B0B2808D1FD
:101BC000606B1F284AD270480068401C6E4908604C
:101BD00044E06D480068401C6B4908603EE06A487C
:101BE0000068401C6849086038E0674800680028C1
:101BF00005D165480068401C634908602EE06248D2
:101C0000006801280BD101200190012000900123E0
:101C100001221F21606BFCF703FE60631EE05A483F
:101C2000006802280BD101200190012000900123BF
:101C300001220C21A06BFCF7F3FDA0630EE05248DB
:101C4000006803280AD1012001900120009001239F
:101C500000226321E06BFCF7E3FDE06317B0F0BD09
:101C60002F00000010B588B0040040200021F6F7D6
:101C700080FD434B3CA2162102A8FAF767FA02A99D
:101C80000020FAF742FE0420FAF7FDFD0420FAF7DF
:101C900061FE606B002805D116224A4902A8FAF7B6
:101CA000DDF804E01622484902A8FAF7D7F802A99D
:101CB0000120FAF72AFE2BA10220FAF726FE29A11D
:101CC0000320FAF722FE27A10420FAF71EFE25A121
:101CD0000520FAF71AFE23A10620FAF716FE21A125
:101CE0000720FAF712FE1FA10820FAF70EFE0820BF
:101CF000FAF706FB002820D0606B002804D00120F2
:101D0000F9F73EFC002807D0606B002812D10120B3
:101D1000F9F736FC00280DD0606B002803D10120B4
:101D2000F9F738FC02E00120F9F72EFC0020082129
:101D3000F6F71FFDFCF7E6FC12E00120FAF7E0FAE7
:101D4000002802D0FCF7DEFC0AE000200190002011
:101D50000090012300220121606BFCF761FD6063AC
:101D600008B010BD0000000025730000C0D20300C1
:101D700080ED030088F10100A0ED030090F1010067
:101D800060ED030098F1010000120020A0F10100B5
:101D900048E901003CED010058EE0100A8F1010006
:101DA000B0F1010064EE0100C0EB030000EB0300A2
:101DB00020EB030040EB030060EB030080EB03002B
:101DC000A0EB030080E60300E0D9030010B592B059
:101DD0004FF400600021F6F7CCFC1622DFF8F01576
:101DE0006846FAF73BF8DFF8E835DFF8E825162112
:101DF00006A8FAF7ABF9F8F7D6FF012809D1DFF802
:101E0000D035DFF8D42516210DF12E00FAF79EF912
:101E100008E0DFF8BC35DFF8C42516210DF12E00EF
:101E2000FAF794F90220FCF780FB0320FAF72BFD68
:101E30000420FAF78FFD69460020FAF766FD0020BE
:101E4000FCF7B8FB401CFAF722FD0220FCF7B2FBBE
:101E5000040006A90120FAF758FD0DF12E01022019
:101E6000FAF753FDB6A10320FAF74FFDB4A1042001
:101E7000FAF74BFD0120FAF743FA002802D0FCF7ED
:101E800041FC16E00820FAF73BFA00280ED00120AA
:101E9000FCF790FB012804D101210C20FCF7C9FBC1
:101EA00007E001210A20FCF7C4FB02E02000FCF758
:101EB00044FC12B010BD70B5B2B01622DFF8101598
:101EC0006846F9F7CBFF69460020FAF71EFD0320AC
:101ED000FAF7D9FC0420FAF73DFD00200AE00022C1
:101EE00006AB162404FB00F423445A54491C16295B
:101EF000F5D3401C082801D20021F8E70124002670
:101F00005FF0FF30F9F73DF805000EE025420BD0F9
:101F1000F8F749FF0200210006A8162303FB06F389
:101F2000184400F0E1F9761C6400082E01D2002C60
:101F3000ECD13000FCF7F9FA002D03D10020FAF7BC
:101F4000A6FC05E00020FCF735FB401CFAF79FFCDF
:101F50000220FCF72FFB040006A8162101FB04F168
:101F600001440120FAF7D1FC06A8162101FB04F177
:101F7000084410F116010220FAF7C7FC06A8162142
:101F800001FB04F1084410F12C010320FAF7BDFC19
:101F900006A91620444301EB040010F1420104207D
:101FA000FAF7B3FC0120FAF7ABF9002802D0FCF7EE
:101FB000A9FB29E00820FAF7A3F9002821D0012085
:101FC000FCF7F8FA0400F8F7EEFE0200102168466C
:101FD00000F08AF91222694606AB1620444303EB4F
:101FE0000400FAF7BAF8002808D1F9F732FA002805
:101FF00004D002210D20FCF71CFB05E0FCF782FB5E
:1020000002E03000FCF799FB32B070BD70B5B2B0A1
:102010004FF400600021F6F7ACFBF8F7C4FE01288E
:1020200008D1DFF8AC33DFF8B82316216846FAF799
:102030008DF807E0DFF89833DFF8A823162168460B
:10204000FAF784F869460020FAF75FFC0320FAF7F4
:102050001AFC0420FAF77EFC00200AE0002206ABFE
:10206000162404FB00F423445A54491C1629F5D3C2
:10207000401C082801D20021F8E7012400265FF067
:10208000FF30F8F783FF05000BE0254208D0210060
:1020900006A8162202FB06F2104400F06BF9761C2B
:1020A0006400082E01D2002CEFD13000FCF73DFA7D
:1020B000002D03D10020FAF7EAFB05E00020FCF731
:1020C00079FA401CFAF7E3FB0220FCF773FA0400EC
:1020D00006A8162101FB04F101440120FAF715FCC2
:1020E00006A8162101FB04F1084410F11601022094
:1020F000FAF70BFC06A8162101FB04F1084410F1C5
:102100002C010320FAF701FC06A91620444301EB39
:10211000040010F142010420FAF7F7FB0820FAF757
:10212000EFF8002804D10120FAF7EAF8002802D0DD
:10213000FCF7E8FA02E03000FCF7FFFA32B070BDBD
:102140000000000070B5B2B048200021F6F711FB86
:102150001622A5496846F9F781FE00200AE0002210
:1021600006AB162404FB00F423445A54491C1629D8
:10217000F5D3401C082801D20021F8E701240025EE
:102180005FF0FF300021F8F70FFF06000CE0264259
:1021900009D02200002306A8162101FB05F10844FE
:1021A00000F0FBF86D1C6400082D01D2002CEED16C
:1021B0002800FCF7BAF90320FAF765FB0420FAF7C8
:1021C000C9FB69460020FAF7A0FB002E03D10020CE
:1021D000FAF75DFB05E00020FCF7ECF9401CFAF78C
:1021E00056FB0220FCF7E6F9040006A8162101FBC5
:1021F00004F101440120FAF788FB06A8162101FB2F
:1022000004F1084410F116010220FAF77EFB06A83B
:10221000162101FB04F1084410F12C010320FAF708
:1022200074FB06A91620444301EB040010F142019F
:102230000420FAF76AFB0820FAF762F8002804D1B4
:102240000120FAF75DF8002802D0FCF75BFA02E003
:102250002800FCF772FA32B070BD10B58CB0F9F7F7
:10226000F8F80400614B57A2162106A8F9F76EFF93
:10227000230055A216216846F9F768FF0420FAF7F3
:1022800002FB0120FAF766FB06A90020FAF73DFBE6
:1022900069460120FAF739FB4CA10220FAF735FB19
:1022A0004AA10320FAF731FB48A10420FAF72DFBDD
:1022B00046A10520FAF729FB44A10620FAF725FBE1
:1022C00042A10720FAF721FB40A10820FAF71DFBE5
:1022D0000020FAF7DCFA0820FAF712F8002801D0FB
:1022E000FCF710FA0CB010BD38B504000800F9F77F
:1022F00001FA05003E4850F8250000903D4850F88E
:1023000025303D4A16212000F9F720FF0A2D08D17B
:102310003A4800900B233A4A16212000F9F716FF9D
:1023200027E00B2D08D1354800900C23354A1621A3
:102330002000F9F70BFF1CE00C2D0CD1F8F733FD52
:10234000012808D12D4800900D232F4A1621200086
:10235000F9F7FCFE0DE00D2D0BD1F8F724FD012857
:1023600007D1264800900E23284A16212000F9F7AD
:10237000EDFE31BD10B582B004000800F9F7BAF9DE
:10238000234951F820100091224951F820301A4A6F
:1023900016212000F9F7DAFE13BD10B582B0040053
:1023A00010001900F9F728FA1B4951F82010009184
:1023B0001A4951F82030104A16212000F9F7C6FEBC
:1023C00013BD00002573000025640000000000001C
:1023D00060D20300B8F1010070EE0100C0F101000D
:1023E000C8F10100D0F1010080D20300E0DD03005C
:1023F00000000020F8E30100D8F10100E0DF030055
:102400007CEE010088EE010094EE0100A0EE0100D8
:102410002001002078E401008000002058E3010042
:1024200010B598B0040041200021F6F7A2F903206E
:10243000FCF77BF81622DFF8DC166846F9F70EFD8C
:1024400069460020FAF761FA0320FAF71CFA042023
:10245000FAF780FADFF8C036DFF8C026162106A8A2
:10246000F9F774FEDFF8B836DFF8B82616210DF15B
:102470002E00F9F76BFEDFF8B036DFF8B026162134
:1024800011A8F9F763FE0020FCF794F8401CFAF756
:10249000FEF906A90120FAF738FA0DF12E01022003
:1024A000FAF733FA11A90320FAF72FFA67A10420EB
:1024B000FAF72BFA0820F9F723FF002846D001206D
:1024C000FCF778F8002804D101211720FCF7B1F8B7
:1024D00047E001282BD101211820FCF7AAF8502051
:1024E000F9F75FF860635120F9F75BF8A0635220B9
:1024F000F9F757F8E0636069012804D10121002051
:10250000FCF77CF803E000210020FCF777F8606B13
:10251000002805D0A06B002802D0E06B002820D155
:10252000002060630020A0630020606319E002289F
:1025300017D16069012804D101211A20FCF779F82C
:102540000FE001210720FCF774F80AE00120F9F7F9
:10255000D7FE002802D0FCF7D5F802E00320FCF7F4
:10256000ECF818B010BD00B58DB041200021F6F791
:1025700000F91622DFF8A01501A8F9F76FFC01A9F0
:102580000020FAF7C2F90420FAF77DF90120FAF7E2
:10259000E1F90A23152207A9DFF89405FCF7AEF943
:1025A000F8F700FEDFF88C15884201D3DFF88805C4
:1025B000F8F7F8FD009007ABDFF88025162101A899
:1025C000F9F7C4FD01A90120FAF79FF90A231522A2
:1025D00007A9DFF86C05FCF791F9F8F7DFFDDFF8E4
:1025E0005415884201D3DFF85005009007ABDFF89F
:1025F0004C25162101A8F9F7A9FD01A90520FAF734
:1026000084F912A10220FAF780F910A10320FAF749
:102610007CF90EA10420FAF778F90CA10620FAF74C
:1026200074F90AA10720FAF770F908A10820FAF74F
:102630006CF90020FAF72BF90820F9F761FE002861
:1026400001D0FCF75FF80DB000BD000000000000F5
:1026500070B588B0050040200021F6F78AF8686B55
:10266000002805D0A86B002802D0E86B002801D113
:10267000012600E000261622DFF8C81402A8F9F7A8
:10268000EDFB02A90020FAF740F90420FAF7FBF865
:102690006869012803D10420FAF75CF902E00320FD
:1026A000FAF758F90020FBF785FF04002000FAF73D
:1026B000EEF8002C1BD1E86B0190A86B00906B6BBF
:1026C000DFF88424092102A8F9F740FD02A90120BE
:1026D000FAF71BF9A5A10220FAF717F9A3A1032025
:1026E000FAF713F9A1A10420FAF70FF96AE0012C17
:1026F00020D16B6BDFF85424032102A8F9F726FDE3
:1027000002A90120FAF701F9E86B0090AB6BDFF842
:102710004024072102A8F9F719FD02A90220FAF7BF
:10272000F4F892A10320FAF7F0F890A10420FAF748
:10273000ECF847E0022C25D16B6BDFF8182404215C
:1027400002A8F9F703FD02A90120FAF7DEF8AB6B46
:10275000DFF8F823032102A8F9F7F8FC02A9022008
:10276000FAF7D3F8EB6BDFF8F023042102A8F9F7AE
:10277000EDFC02A90320FAF7C8F87CA10420FAF7BF
:10278000C4F81FE0A86B00906B6BDFF8D023062124
:1027900002A8F9F7DBFC02A90120FAF7B6F8AFA10D
:1027A0000220FAF7B2F8EB6BDFF8A023032102A8AE
:1027B000F9F7CCFC02A90320FAF7A7F86BA10420D3
:1027C000FAF7A3F8012E0AD11622DFF8941302A813
:1027D000F9F744FB02A90520FAF797F803E063A193
:1027E0000520FAF792F861A10620FAF78EF85FA1AA
:1027F0000720FAF78AF85DA10820FAF786F8012089
:10280000F9F77EFD002802D0FBF77CFFABE0082043
:10281000F9F776FD00287DD0032C36D1686B1D2892
:1028200008D1A86B022805D195F83C0010F0030FE1
:1028300040F099805020F8F7B4FE696B81420BD1CB
:102840005120F8F7AEFEA96B814205D15220F8F76E
:10285000A8FEE96B81420FD000200821F5F789FF1F
:10286000696B5020F8F7B5FEA96B5120F8F7B1FE5F
:10287000E96B5220F8F7ADFE02211920FBF7D9FED3
:102880004020F8F78EFE68636DE0022C26D1A86B1D
:10289000022808D1686B1E2865D2641C2100002024
:1028A000FBF7ACFE5FE0A86B042808D0A86B0628F5
:1028B00005D0A86B092802D0A86B0B2808D1686B3B
:1028C0001F2850D2641C21000020FBF797FE4AE02D
:1028D000641C21000020FBF791FE44E0012C10D184
:1028E000686B002808D102211920FBF7A2FE4020C6
:1028F000F8F757FE686336E002210020FBF77EFE02
:1029000031E002211920FBF794FE4020F8F749FE40
:10291000686328E0012C0BD1012001900120009078
:10292000012300221F21686BFBF77AFF68631AE01E
:10293000022C0BD1012001900120009001230022E4
:102940000C21A86BFBF76CFFA8630CE0032C0AD1E9
:102950000120019001200090012300226321E86BF7
:10296000FBF75EFFE86308B070BD000000000000E8
:1029700010B588B0040040200021F5F7FAFE1622B9
:10298000784902A8F9F76AFA02A90020F9F7BDFF11
:102990000420F9F778FF6069012803D10420F9F7D2
:1029A000D9FF02E00320F9F7D5FF636B56A2082197
:1029B00002A8F9F7CBFB02A90120F9F7A6FF53A162
:1029C0000220F9F7A2FF51A10320F9F79EFF4FA1C2
:1029D0000420F9F79AFF4DA10520F9F796FF4BA1C6
:1029E0000620F9F792FF49A10720F9F78EFF47A1CA
:1029F0000820F9F78AFF0020F9F749FF0120F9F7CD
:102A00007FFC002802D0FBF77DFE25E00820F9F7C7
:102A100077FC002810D04020F8F7C3FD616B81429D
:102A200007D0616B4020F8F7D4FD00200821F5F7AE
:102A3000A0FEFBF767FE0FE0606901280CD10120C2
:102A40000190012000904FF47A734FF47A72464956
:102A5000606BFBF7E5FE606308B010BD2F0000005F
:102A600000B587B0162230496846F9F7F7F969468C
:102A70000020F9F74AFF0420F9F705FF0320F9F7D2
:102A800069FF3A4B22A216216846F9F75FFB6946B7
:102A90000120F9F73AFF0020F9F7F9FE1BA1022007
:102AA000F9F733FF19A10320F9F72FFF17A104202D
:102AB000F9F72BFF15A10520F9F727FF13A1062031
:102AC000F9F723FF11A10720F9F71FFF0FA1072036
:102AD000F9F71BFF0120F9F713FC002802D0FBF7E0
:102AE00011FE0EE00820F9F70BFC002809D05FF07A
:102AF0000070F8F73EFB00208021F5F73AFEFBF767
:102B000001FE07B000BD00002564000000000000C9
:102B100025733F00A0D2030000ED030050F1010037
:102B200020ED030058F1010040ED030060F10100C9
:102B3000C0EC030000CA9A3BFFC99A3B68F1010050
:102B4000E0EC030080EC03002CED010070F10100CB
:102B500040EE010078F1010080F101004CEE01002F
:102B600080E60300A0DD030040420F00E0DA03002E
:102B700010B5A8B00620FBF7D8FC1622C34968465A
:102B8000F9F76CF9C24BC34A162106A8F9F7DEFA29
:102B9000C14BC24A16210DF12E00F9F7D7FAC04BEE
:102BA000C04A162111A8F9F7D1FABF4BBF4A162126
:102BB0000DF15A00F9F7CAFABD4BBE4A16211CA8FE
:102BC000F9F7C4FABC4BBD4A16210DF18600F9F79E
:102BD000BDFA0320F9F757FE0420F9F7BBFE69465A
:102BE0000020F9F792FE0220FBF7E4FC040006A89F
:102BF000162101FB04F101440120F9F786FE06A825
:102C0000162101FB04F1084410F116010220F9F726
:102C10007CFE06A8162101FB04F1084410F12C01EA
:102C20000320F9F772FE06A91620444301EB0400C5
:102C300010F142010420F9F768FE0020FBF7BAFC0E
:102C4000401CF9F724FE0820F9F75AFB00280AD0A7
:102C50000120FBF7AFFC401C9949086001213A2094
:102C6000FBF7E7FC0AE00120F9F74AFB002802D055
:102C7000FBF748FD02E00620FBF75FFD28B010BD22
:102C800000B58DB01622814906A8F9F7E7F88C48FF
:102C90000068012806D17E4B7AA216216846F9F712
:102CA00055FAA7E086480068022806D17A4B75A23B
:102CB00016216846F9F74AFA9CE081480068032823
:102CC00006D1774B6FA216216846F9F73FFA91E0DB
:102CD0007B480068042806D1734B6AA21621684617
:102CE000F9F734FA86E076480068052806D1704B7B
:102CF00064A216216846F9F729FA7BE0704800685B
:102D0000062806D16C4B5FA216216846F9F71EFA19
:102D100070E06B480068072806D16A4B59A216215B
:102D20006846F9F713FA65E065480068082806D197
:102D3000654B54A216216846F9F708FA5AE0604834
:102D40000068092806D1614B4EA216216846F9F7A2
:102D5000FDF94FE05A4800680A2806D15C4B49A2A9
:102D600016216846F9F7F2F944E0554800680B2847
:102D700006D1584B43A216216846F9F7E7F939E026
:102D80004F4800680C2806D1534B3EA216216846D6
:102D9000F9F7DCF92EE04A4800680D2806D14F4BC0
:102DA00038A216216846F9F7D1F923E044480068B3
:102DB0000E2806D14A4B33A216216846F9F7C6F908
:102DC00018E03F4800680F2806D1464B2DA2162177
:102DD0006846F9F7BBF90DE039480068102806D1BC
:102DE000414B28A216216846F9F7B0F902E001200C
:102DF000F8F793FB0420F9F746FD0320F9F7AAFD45
:102E000006A90020F9F781FD69460120F9F77DFD4B
:102E10001DA10220F9F779FD1BA10320F9F775FD2B
:102E200019A10420F9F771FD17A10520F9F76DFD2F
:102E300015A10620F9F769FD13A10720F9F765FD33
:102E400011A10820F9F761FD0020F9F720FD01200C
:102E5000F9F756FA002802D0FBF754FC10E00820DE
:102E6000F9F74EFA00280BD0F9F753FB144909681B
:102E7000814203D012480068F9F74EFBFBF742FC91
:102E80000DB000BD25733F000000000020D20300FC
:102E900020D00300B0F2010040D00300B8F20100DE
:102EA00060D00300C0F2010080D00300C8F201002E
:102EB000A0D00300D0F20100C0D00300D8F201007E
:102EC00018120020E0D0030000D1030020D103003D
:102ED00040D1030060D1030080D10300A0D10300E2
:102EE000C0D10300E0D1030000D2030030B5BDB073
:102EF000050070200021F5F73CFCF7F754FF01288E
:102F000003D10920FBF711FB02E00A20FBF70DFBC0
:102F10001622DFF8301A6846F8F7A0FFF7F743FFEC
:102F2000012855D1DFF8203ADFF8202A162106A81B
:102F3000F9F70CF9DFF8183ADFF8182A16210DF125
:102F40002E00F9F703F9DFF8103ADFF8102A1621FE
:102F500011A8F9F7FBF8DFF8083ADFF8082A16217C
:102F60000DF15A00F9F7F2F8DFF8FC39DFF8FC2927
:102F700016211CA8F9F7EAF8DFF8D83BDFF8D82BC0
:102F800016210DF18600F9F7E1F8DFF8D03BDFF804
:102F9000D02B162127A8F9F7D9F8DFF8C83BDFF8BE
:102FA000C82B16210DF1B200F9F7D0F8DFF8BC3BC1
:102FB000DFF8BC2B162132A8F9F7C8F803A21621B6
:102FC0000DF1DE00F9F7C2F857E000BF0000000085
:102FD000DFF8A03BDFF87429162106A8F9F7B6F848
:102FE000DFF86439DFF86C2916210DF12E00F9F7AE
:102FF000ADF8DFF85C39DFF86429162111A8F9F77C
:10300000A5F8DFF85439DFF85C2916210DF15A00D4
:10301000F9F79CF8DFF84839DFF8502916211CA889
:10302000F9F794F8DFF84039DFF82C2B16210DF171
:103030008600F9F78BF8DFF81C3BDFF8242B16210C
:1030400027A8F9F783F8DFF8143BDFF81C2B1621CB
:103050000DF1B200F9F77AF8DFF8083BDFF8102B32
:10306000162132A8F9F772F8DFF8003BDFF8442C9C
:1030700016210DF1DE00F9F769F80320F9F703FCDA
:103080000420F9F767FC69460020F9F73EFC0020B0
:10309000FBF790FA401CF9F7FAFB0220FBF78AFADB
:1030A000040006A8162101FB04F101440120F9F7F0
:1030B0002CFC06A8162101FB04F1084410F11601AE
:1030C0000220F9F722FC06A8162101FB04F10844AE
:1030D00010F12C010320F9F718FC06A9162044432F
:1030E00001EB040010F142010420F9F70EFC01206D
:1030F000F9F706F9002802D0FBF704FBEEE0082000
:10310000F9F7FEF8002800F0E6800120FBF752FAFC
:103110000400F7F748FE012849D1002C04D1012111
:103120003B20FBF786FAD3E0012C04D10121482093
:10313000FBF77FFACCE0022C04D101215B20FBF7E6
:1031400078FAC5E0032C0ED101212420FBF771FA97
:103150001020F8F715FA002802D001206863B7E0C4
:1031600000206863B4E0042C04D101212520FBF782
:1031700060FAADE0052C04D101212A20FBF759FAB1
:10318000A6E0062C04D101215F20FBF752FA9FE054
:10319000072C04D101217820FBF74BFA98E0082C8A
:1031A00040F0968001216720FBF743FA90E0002C65
:1031B00022D101212020FBF73CFAF7F7FDFD012881
:1031C00002D10420686383E0F7F704FE012802D1EE
:1031D000032068637CE0F7F70BFE012802D1012091
:1031E000686375E0F7F712FE012802D102206863D8
:1031F0006EE0002068636BE0012C08D1F7F714FE45
:10320000002804D101213B20FBF713FA60E0022CD7
:1032100008D1F7F709FE002804D101214820FBF767
:1032200008FA55E0032C08D1F7F7FEFD002804D179
:1032300001215B20FBF7FDF94AE0042C12D1F7F7DE
:10324000F3FD00280ED101212420FBF7F2F9102014
:10325000F8F796F9002802D00120686338E00020D2
:10326000686335E0052C08D1F7F7DEFD002804D1AE
:1032700001212520FBF7DDF92AE0062C08D1F7F71C
:10328000D3FD002804D101212A20FBF7D2F91FE049
:10329000072C08D1F7F7C8FD002804D101215F20D1
:1032A000FBF7C7F914E0082C08D1F7F7BDFD00289B
:1032B00004D101217820FBF7BCF909E0092C07D1E2
:1032C000F7F7B2FD002803D101216720FBF7B1F920
:1032D000686B286402E00A20FBF72FFA3DB030BD8E
:1032E00010B594B0040050200021F5F742FA1622E0
:1032F000DFF880180EA8F8F7B1FD606B01280BD13C
:10330000DFF8C82B162108A8F8F720FFB4A2162171
:1033100002A8F8F71BFF36E0606B02280BD1DFF83C
:10332000B02B162108A8F8F711FFAEA2162102A8AB
:10333000F8F70CFF27E0606B03280BD1DFF8942B24
:10334000162108A8F8F702FFA7A2162102A8F8F78D
:10335000FDFE18E0606B04280BD1DFF87C2B1621F2
:1033600008A8F8F7F3FEA1A2162102A8F8F7EEFECE
:1033700009E09FA2162108A8F8F7E8FE9DA21621F1
:1033800002A8F8F7E3FE0420F9F77DFA0420F9F724
:10339000E1FA0EA90020F9F7B8FA08A90120F9F717
:1033A000B4FA02A90520F9F7B0FA92A10220F9F7C0
:1033B000ACFA90A10320F9F7A8FA8EA10420F9F73E
:1033C000A4FA8CA10620F9F7A0FA8AA10720F9F740
:1033D0009CFA88A10820F9F798FA0020F9F757FA23
:1033E0000820F8F78DFF002829D0F7F7C8FC01283E
:1033F00002D1FBF787F944E0606B002841D0606B95
:10340000216C884204D001212120FBF712F938E019
:10341000606B042810D101212220FBF70AF9022059
:10342000F8F7AEF8002802D10020606301E0012027
:103430006063606B206424E0FBF764F921E0012005
:10344000F8F75EFF002802D0FBF75CF919E0606B2B
:1034500000280BD0002001900120009001230122C0
:103460000421606BFBF7DCF960630AE00020019047
:1034700001200090012300220421606BFBF7D0F9AA
:10348000606314B010BD10B592B004007820002124
:10349000F5F76FF91622DFF8DC160CA8F8F7DEFC5A
:1034A000DFF8343B9AA2162106A8F8F74FFE606BAE
:1034B000042806D1DFF8242B16216846F8F746FECB
:1034C00019E0606B022806D1DFF8142B162168463C
:1034D000F8F73CFE0FE0606B032806D1DFF8042B01
:1034E00016216846F8F732FE05E0DFF8FC2A1621BF
:1034F0006846F8F72BFE0420F9F7C5F90320F9F721
:1035000029FA0020F9F7C3F90CA90020F9F7FDF911
:1035100006A90120F9F7F9F936A10220F9F7F5F922
:1035200034A10320F9F7F1F932A10420F9F7EDF9FC
:1035300030A10520F9F7E9F92EA10620F9F7E5F900
:103540002CA10720F9F7E1F92AA10820F9F7DDF904
:103550000820F8F7D5FE002838D0606B042804D185
:1035600007211E20F8F735F813E0606B022804D11C
:1035700004211E20F8F72DF80BE0606B032804D11E
:1035800008211E20F8F725F803E009211E20F8F78E
:1035900020F800200221F5F7ECF8606B042810D128
:1035A00002212220FBF745F80220F7F7E9FF002867
:1035B00002D10020606301E001206063606B206441
:1035C0000CE0FBF79FF8FBF79DF807E00120F8F708
:1035D00097FE002802D0200001F0B0F812B010BD14
:1035E00028312900283229002833290028342900CD
:1035F0004E4F00000000000010B58EB0040078208F
:103600000021F5F7B6F81622DFF8B81B08A8F8F77E
:1036100025FC606B002806D11622DFF8AC1B02A83F
:10362000F8F71CFC05E01622DFF8A01B02A8F8F74B
:1036300015FC0420F9F727F90420F9F78BF900208D
:10364000F9F725F908A90020F9F75FF902A9012087
:10365000F9F75BF9BAA10220F9F757F9B8A10320ED
:10366000F9F753F9B6A10420F9F74FF9B4A10520F1
:10367000F9F74BF9B2A10620F9F747F9B0A10720F5
:10368000F9F743F9AEA10820F9F73FF90820F8F758
:1036900037FE002826D0206C616B88420DD0606B0D
:1036A000002803D00220F7F76FFF02E00220F7F7AF
:1036B00071FF00200821F5F75CF81E20F7F771FF75
:1036C00007280AD15E20F7F76CFF6063606B206407
:1036D00002212320FAF7ADFF18E0FBF713F8FBF700
:1036E00011F813E00120F8F70BFE002803D02000AA
:1036F00001F024F80AE0002001900120009001234D
:1037000000220121606BFBF78BF860630EB010BDE7
:1037100025733F0010B58EB0040048200021F5F756
:1037200028F81622DFF8C01B08A8F8F797FB02203C
:10373000F7F726FF616B00290FD1002806D1DFF8CB
:10374000AC2B162102A8F8F701FD28E0DFF8A02B2A
:10375000162102A8F8F7FAFC21E0616B01290FD1CC
:10376000002806D1DFF88C2B162102A8F8F7EEFC12
:1037700015E0DFF8842B162102A8F8F7E7FC0EE02D
:10378000002806D1DFF8742B162102A8F8F7DEFC1A
:1037900005E0DFF86C2B162102A8F8F7D7FC04200F
:1037A000F9F771F80420F9F7D5F80020F9F76FF868
:1037B00008A90020F9F7A9F802A90120F9F7A5F84E
:1037C0005FA10220F9F7A1F85DA10320F9F79DF8A8
:1037D0005BA10420F9F799F859A10520F9F795F8AC
:1037E00057A10620F9F791F855A10720F9F78DF8B0
:1037F00053A10820F9F789F80820F8F781FD00287F
:1038000010D0206C616B884207D0616B5E20F7F7A7
:10381000E0FE00200821F4F7ACFFFAF773FFFAF797
:1038200071FF13E00120F8F76BFD002803D02000A2
:1038300000F084FF0AE000200190012000900123A5
:1038400000220221606BFAF7EBFF60630EB010BD3F
:1038500010B58EB0040070200021F4F78AFF162204
:103860003F4908A8F8F7FAFA606B002806D116223B
:10387000DFF8201C02A8F8F7F1FA05E01622DFF8BD
:10388000181C02A8F8F7EAFA0420F8F7FCFF042055
:10389000F9F760F80020F8F7FAFF08A90020F9F717
:1038A00034F802A90120F9F730F825A10220F9F730
:1038B0002CF823A10320F9F728F821A10420F9F717
:1038C00024F81FA10520F9F720F81DA10620F9F71B
:1038D0001CF81BA10720F9F718F819A10820F9F71F
:1038E00014F80820F8F70CFD002814D0606B216C48
:1038F00088420DD0606B002803D11020F7F74AFEF4
:1039000002E01020F7F740FE00200821F4F731FF15
:10391000FAF7F8FE12E00120F8F7F2FC002802D0D6
:10392000FAF7F0FE0AE00020019001200090012348
:1039300000220121606BFAF773FF60630EB010BDC7
:103940000000000040D2030040D3030098F30100C0
:1039500060D30300A0F3010080F10300A8F301008D
:1039600080D30300B0F30100A0D30300B8F301003B
:1039700030B59DB0040070200021F4F7FAFE042059
:10398000FAF7D3FD1622DFF81C1C01A8F8F766FA37
:10399000DFF8143CDFF8142C162107A8F8F7D6FB43
:1039A000DFF80C3CDFF80C2C16210DF13200F8F793
:1039B000CDFBDFF8040C0090DFF8EC3BDFF8FC2BCC
:1039C000162112A8F8F7C2FBDFF8F43BDFF8F42B5E
:1039D00016210DF15E00F8F7B9FB0320F8F753FF4D
:1039E0000420F8F7B7FF0020FAF7E4FD401CF8F7D1
:1039F0004EFF01A90020F8F788FF0220FAF7DAFD50
:103A0000050007A8162101FB05F101440120F8F784
:103A10007CFF07A8162101FB05F1084410F11601EF
:103A20000220F8F772FF07A8162101FB05F10844F0
:103A300010F12C010320F8F768FF07A91620454371
:103A400001EB050010F142010420F8F75EFF0820A9
:103A5000F8F756FC00286FD00120FAF7ABFD0028DC
:103A600016D101212620FAF7E4FD4E20F7F799FD43
:103A7000C00702D4002060635BE04E20F7F791FDA1
:103A8000800702D50120606353E00220606350E0AC
:103A9000012817D14E20F7F784FD10F00100606374
:103AA000606B002845D001212720FAF7C2FD4E2087
:103AB000F7F777FD000602D40020606339E00120AB
:103AC000606336E0022817D14E20F7F76AFD10F048
:103AD00001006063606B00282BD001212820FAF7D9
:103AE000A8FD4E20F7F75DFD400702D50120606379
:103AF0001FE0002060631CE0032817D14E20F7F779
:103B000050FD10F001006063606B002811D00121AE
:103B10002920FAF78EFD4E20F7F743FD400602D428
:103B20000020606305E00120606302E00120F7F7F8
:103B3000F4FC606B20640AE00120F8F7E1FB002848
:103B400002D0FAF7DFFD02E00420FAF7F6FD1DB01F
:103B500030BD0000C0D30300C0F30100E0D3030078
:103B6000C8F301004CEA0100D0F3010020D40300A7
:103B7000D8F3010060F4030010B58EB0040070208B
:103B80000021F4F7F6FD1622DFF8541B08A8F8F719
:103B900065F9606B012806D11622DFF8481B02A8E0
:103BA000F8F75CF911E0606B022806D11622DFF805
:103BB000381B02A8F8F752F907E01622DFF8D418EC
:103BC00002A8F8F74BF9002060630420F8F75BFEC9
:103BD000F7F7E9F8012803D10120F8F7BBFE02E06E
:103BE0000420F8F7B7FE0020F8F751FE08A90020DE
:103BF000F8F78BFE02A90120F8F787FEB2A1022098
:103C0000F8F783FEB0A10320F8F77FFEAEA10420F1
:103C1000F8F77BFEACA10520F8F777FEAAA10620F5
:103C2000F8F773FEA8A10720F8F76FFEA6A10820F9
:103C3000F8F76BFE0820F8F763FB00281ED0606BD6
:103C4000216C884217D04E20F7F7ABFC01008908A1
:103C50008900606B012802D151F0030104E0606B20
:103C6000022801D151F001014E20F7F7B2FC0020EB
:103C70000821F4F77EFDFAF745FD18E00120F8F77A
:103C80003FFB002802D0FAF73DFD10E00020019034
:103C900001200090012300220221606BFAF7C0FD91
:103CA0006063F7F780F8012801D1012060630EB04E
:103CB00010BD0000E0F3010010B58EB004007020CC
:103CC0000021F4F756FD1622DFF8201A08A8F8F7AD
:103CD000C5F8606B002806D11622DFF80C1A02A87E
:103CE000F8F7BCF805E01622DFF8F81902A8F8F793
:103CF000B5F80420F8F7C7FD0420F8F72BFE0020E4
:103D0000F8F7C5FD08A90020F8F7FFFD02A901207A
:103D1000F8F7FBFD6CA10220F8F7F7FD6AA103207C
:103D2000F8F7F3FD68A10420F8F7EFFD66A1052080
:103D3000F8F7EBFD64A10620F8F7E7FD62A1072084
:103D4000F8F7E3FD60A10820F8F7DFFD0820F8F799
:103D5000D7FA002818D0606B216C884211D04E2011
:103D6000F7F71FFC010031F00401606B012801D15D
:103D700051F004014E20F7F72CFC00200821F4F745
:103D8000F8FCFAF7BFFC12E00120F8F7B9FA0028B6
:103D900002D0FAF7B7FC0AE0002001900120009061
:103DA000012300220121606BFAF73AFD60630EB037
:103DB00010BD10B58EB0040070200021F4F7D9FCBE
:103DC0001622DFF8EC1708A8F8F748F8606B00280F
:103DD00006D11622DFF8181902A8F8F73FF805E017
:103DE0001622DFF8101902A8F8F738F80420F8F7BF
:103DF0004AFDF6F7D8FF012803D10120F8F7AAFD04
:103E000002E00420F8F7A6FD0020F8F740FD08A91D
:103E10000020F8F77AFD02A90120F8F776FD2AA123
:103E20000220F8F772FD28A10320F8F76EFD26A105
:103E30000420F8F76AFD24A10520F8F766FD22A109
:103E40000620F8F762FD20A10720F8F75EFD1EA10D
:103E50000820F8F75AFD0820F8F752FA002818D081
:103E6000606B216C884211D04E20F7F79AFB01005D
:103E700031F08001606B002801D051F080014E20AC
:103E8000F7F7A7FB00200821F4F773FCFAF73AFCD8
:103E900018E00120F8F734FA002802D0FAF732FCD3
:103EA00010E0002001900120009001230022012158
:103EB000606BFAF7B5FC6063F6F775FF012801D176
:103EC000002060630EB010BD00000000E8F30100A8
:103ED000FCEF0100F0F30100F8F3010010B58EB023
:103EE000040070200021F4F744FC1622DFF8D016FD
:103EF00008A8F7F7B3FF606B002806D11622DFF899
:103F0000F01702A8F7F7AAFF05E01622DFF8E4177A
:103F100002A8F7F7A3FF0420F8F7B5FC0420F8F790
:103F200019FD0020F8F7B3FC08A90020F8F7EDFC14
:103F300002A90120F8F7E9FCA1A10220F8F7E5FCAD
:103F40009FA10320F8F7E1FC9DA10420F8F7DDFC18
:103F50009BA10520F8F7D9FC99A10620F8F7D5FC1C
:103F600097A10720F8F7D1FC95A10820F8F7CDFC20
:103F70000820F8F7C5F9002818D0606B216C88423A
:103F800011D04E20F7F70DFB010031F04001606BBE
:103F9000002801D051F040014E20F7F71AFB002015
:103FA0000821F4F7E6FBFAF7ADFB12E00120F8F781
:103FB000A7F9002802D0FAF7A5FB0AE0002001903B
:103FC00001200090012300220121606BFAF728FCF8
:103FD00060630EB010BD0000E0DA030094EC010055
:103FE000A8EC0100BCEC0100BCED010010B59CB0D8
:103FF000040070200021F4F7BCFB0420FAF795FAC6
:104000001622DFF8F4166846F7F728FFDFF8EC36DB
:10401000DFF89825162106A8F8F798F8DFF8883514
:10402000DFF8902516210DF12E00F8F78FF8DFF854
:10403000D036DFF8D026162111A8F8F787F8DFF878
:10404000C836DFF8802516210DF15A00F8F77EF802
:104050000320F8F718FC0420F8F77CFC0020FAF79E
:10406000A9FA401CF8F713FC69460020F8F74DFC4C
:1040700006A90120F8F749FC0DF12E010220F8F7FE
:1040800044FC11A90320F8F740FC0DF15A0104206B
:10409000F8F73BFC0820F8F733F9002800F083809C
:1040A0000120FAF787FA002818D101212B20FAF70E
:1040B000C0FA4D20F7F775FA10F0C0006063606B2E
:1040C000802802D1012060636AE0606BC02802D1C1
:1040D0000220606364E00020606361E0012824D175
:1040E00001212C20FAF7A5FA4D20F7F75AFA10F023
:1040F0000F006063606B012802D1012060634FE014
:10410000606B032802D10220606349E0606B0528E0
:1041100002D10320606343E0606B0F2802D10420CA
:1041200060633DE0002060633AE0022817D14D2033
:10413000F7F737FA10F00F006063606B00282FD09C
:1041400001212D20FAF775FA2020F7F719FA002837
:1041500002D10020606323E00120606320E04D2055
:10416000F7F71FFA10F00F006063606B002817D09C
:1041700001212E20FAF75DFA4D20F7F712FA10F020
:1041800030006063606B002802D10020606307E0AC
:10419000606B102802D10120606301E0022060639F
:1041A000606B20640AE00120F8F7AAF8002802D02A
:1041B000FAF7A8FA02E00420FAF7BFFA1CB010BD23
:1041C0000000000000DA0300C0DA0300A0DA0300F8
:1041D00030B58FB0040070200021F4F7CAFA16221F
:1041E000DFF8181508A8F7F739FE606B002806D12C
:1041F000DFF81825162102A8F7F7A8FF05E0DFF879
:104200001025162102A8F7F7A1FF0420F8F73BFBC1
:104210000420F8F79FFB0020F8F739FB08A90020DD
:10422000F8F773FB02A90120F8F76FFB98A10220B1
:10423000F8F76BFB96A10320F8F767FB94A1042025
:10424000F8F763FB92A10520F8F75FFB90A1062029
:10425000F8F75BFB8EA10720F8F757FB8CA108202D
:10426000F8F753FB0820F8F74BF8002820D0606BD4
:10427000216C884219D04D20F7F793F9050035F0ED
:10428000C005606B002803D12020F7F783F904E014
:1042900055F0C0052020F7F777F929004D20F7F7F2
:1042A00098F900200821F4F764FAFAF72BFA19E0DC
:1042B0000120F8F725F8002802D0FAF723FA11E0D8
:1042C000F6F796FD012802D1002060630AE0002085
:1042D000019001200090012300220121606BFAF778
:1042E0009FFA60630FB030BD00F6030008F00100D4
:1042F00014F00100D0EC0100CCED010020F0010031
:104300002CF0010010B58EB0040070200021F4F7ED
:1043100030FA1622DFF8FC1308A8F7F79FFD606B50
:10432000002805D116225B4902A8F7F797FD2DE07A
:10433000606B012805D116229F4902A8F7F78EFD70
:1043400024E0606B022806D11622DFF8CC1302A805
:10435000F7F784FD1AE0606B032811D1F6F723FD0F
:10436000012806D11622DFF8B41302A8F7F776FD6C
:104370000CE01622DFF8A81302A8F7F76FFD05E09E
:104380001622DFF8A01302A8F7F768FD0420F8F75B
:104390007AFA0420F8F7DEFA0020F8F778FA08A98C
:1043A0000020F8F7B2FA02A90120F8F7AEFA38A116
:1043B0000220F8F7AAFA36A10320F8F7A6FA34A1EA
:1043C0000420F8F7A2FA32A10520F8F79EFA30A1EE
:1043D0000620F8F79AFA2EA10720F8F796FA2CA1F2
:1043E0000820F8F792FA0820F7F78AFF00282AD069
:1043F000606B216C884223D04D20F7F7D2F8010082
:1044000009090901606B012802D151F0010110E096
:10441000606B022802D151F003010AE0606B0328AF
:1044200002D151F0050104E0606B042801D151F084
:104430000F014D20F7F7CDF800200821F4F799F986
:10444000FAF760F921E00120F7F75AFF002802D0BF
:10445000FAF758F919E0F6F7A6FC01280AD14D2021
:10446000F7F79FF810F0C000C02801D1032102E047
:10447000022100E00421002001900120009001238E
:104480000022606BFAF7CCF960630EB010BD00003B
:104490000000000080E60300E0D9030010B58EB0F4
:1044A000040070200021F4F764F91622944908A84A
:1044B000F7F7D4FC606B002805D116229A4902A8B0
:1044C000F7F7CCFC0AE0606B012805D1162297496A
:1044D00002A8F7F7C3FC01E0002060630420F8F7AE
:1044E000D2F90420F8F736FA0020F8F7D0F908A935
:1044F0000020F8F70AFA02A90120F8F706FA77A1D6
:104500000220F8F702FA75A10320F8F7FEF973A16B
:104510000420F8F7FAF971A10520F8F7F6F96FA170
:104520000620F8F7F2F96DA10720F8F7EEF96BA174
:104530000820F8F7EAF90820F7F7E2FE002814D07F
:10454000606B216C88420DD0606B002803D1202065
:10455000F7F720F802E02020F7F716F800200821EE
:10456000F4F707F9FAF7CEF81AE00120F7F7C8FEDA
:10457000002802D0FAF7C6F812E0002001900120CE
:104580000090012300220121606BFAF749F9606372
:104590004D20F7F706F810F00F0F01D100206063EF
:1045A0000EB010BDA0D3030040D8030098F3010063
:1045B00060D80300A0F3010080E4030000F40100D0
:1045C00060F30300B0F3010010B58EB0040070205A
:1045D0000021F4F7CEF816224B4908A8F7F73EFC65
:1045E000606B002805D11622514902A8F7F736FC66
:1045F0000DE0606B012805D116224E4902A8F7F79D
:104600002DFC04E016224C4902A8F7F727FC0420F1
:10461000F8F739F90420F8F79DF90020F8F737F991
:1046200008A90020F8F771F902A90120F8F76DF93F
:104630002AA10220F8F769F928A10320F8F765F903
:1046400026A10420F8F761F924A10520F8F75DF907
:1046500022A10620F8F759F920A10720F8F755F90B
:104660001EA10820F8F751F90820F7F749FE0028A5
:104670001ED0606B216C884217D04D20F6F791FF59
:10468000010031F03001606B002807D0606B012819
:1046900002D151F0100101E051F020014D20F6F758
:1046A00098FF00200821F4F764F8FAF72BF812E0DD
:1046B0000120F7F725FE002802D0FAF723F80AE0D8
:1046C0000020019001200090012300220221606B54
:1046D000FAF7A6F860630EB010BD000000000000FD
:1046E000A0D80300E0D80300C0D8030080F3030083
:1046F00080D50300A0D50300C0D3030040F303001E
:1047000080D80300A8F3010000F4030008F40100BE
:1047100010F4010000D9030080EA0300C0EA03009E
:1047200080F50300E0EA030080E60300E0D903001F
:1047300080E4030000F2030020F4030010B504003D
:10474000F6F73AFB012802D10420606316E0F6F781
:1047500041FB012802D1032060630FE0F6F748FB1C
:10476000012802D10120606308E0F6F74FFB012821
:1047700002D10220606301E000206063606B20646E
:10478000F9F7C0FF10BD000030B5A7B004007020DD
:104790000021F3F7EEFF0620F9F7C7FEF6F703FB5B
:1047A000012801D1062500E005251622C4496846E6
:1047B000F7F754FBF6F7F7FA012827D1C14BC24AA5
:1047C000162106A8F7F7C2FCC04BC14A16210DF10D
:1047D0002E00F7F7BBFCBB4BBE4A162111A8F7F71A
:1047E000B5FCB84BBC4A16210DF15A00F7F7AEFCE8
:1047F000B44BBA4A16211CA8F7F7A8FCB84BB94A23
:1048000016210DF18600F7F7A1FC25E0AD4BAE4A6D
:10481000162106A8F7F79AFCAC4BAD4A16210DF10C
:104820002E00F7F793FCA74BAF4A162111A8F7F714
:104830008DFCA44BAD4A16210DF15A00F7F786FC0A
:10484000A74BAB4A16211CA8F7F780FC9BA21621A8
:104850000DF18600F7F77AFC0320F8F714F804202E
:10486000F8F778F80020F9F7A5FE401CF8F70FF8E4
:1048700069460020F8F749F80220F9F79BFE06AADE
:104880001621484302EB00010120F8F73EF8022010
:10489000F9F790FE06AA16214843104410F11601BC
:1048A0000220F8F732F80220F9F784FE06AA162152
:1048B0004843104410F12C010320F8F726F8022099
:1048C000F9F778FE06AA16214843104410F1420178
:1048D0000420F8F71AF80120F7F712FD002802D09B
:1048E000F9F710FF4EE00820F7F70AFD002846D040
:1048F0000120F9F75FFE002804D101213D20F9F7DE
:1049000098FE3FE0012804D101214420F9F791FEEF
:1049100038E0022804D101213E20F9F78AFE31E077
:1049200003280DD1F6F73FFA012804D101213F20D9
:10493000F9F77FFE26E001214020F9F77AFE21E019
:10494000042811D1F6F72FFA012804D101214020C3
:10495000F9F76FFE16E001213C20F9F76AFE3B20D3
:10496000F6F71FFE60630DE005280BD101213C2006
:10497000F9F75FFE3B20F6F714FE606302E02800C3
:10498000F9F7DBFE27B030BD10B58CB00400702005
:104990000021F3F7EEFE524B564A162106A8F7F710
:1049A000D5FB606B012805D1162253496846F7F7FD
:1049B00055FA0FE0606B032805D116224F4968466F
:1049C000F7F74CFA06E016224D496846F7F746FA23
:1049D000002060630420F7F756FF0420F7F7BAFFC2
:1049E00006A90020F7F791FF69460120F7F78DFF30
:1049F00032A10220F7F789FF30A10320F7F785FFE6
:104A00002EA10420F7F781FF2CA10520F7F77DFFE9
:104A10002AA10620F7F779FF28A10720F7F775FFED
:104A200026A10820F7F771FF0020F7F730FF0120DB
:104A3000F7F766FC002802D0F9F764FE3CE0082096
:104A4000F7F75EFC002810D03B20F6F7AAFD616B5B
:104A5000814207D0616B3B20F6F7BBFD00200421AB
:104A6000F3F787FEF9F74EFE26E00220F7F743FC46
:104A700000280ED0606B012802D1032060631BE088
:104A8000606B032802D10020606315E001206063A1
:104A900012E00420F7F72FFC00280DD0606B0328EC
:104AA00002D10120606307E0606B012802D1002081
:104AB000606301E0032060630CB010BD00000000E3
:104AC00040D3030080D4030000EF0100A0D4030012
:104AD0000CEF010018EF010024EF010030EF01009E
:104AE00020D503003CEF010048EF010054EF010026
:104AF00060EF010050F2010080D90300A0D903004B
:104B000080E6030010B59CB0040070200021F3F78C
:104B100030FE0420F9F709FDDFF8E43ADFF8E42A73
:104B200016216846F7F712FB1622A3A106A8F7F78D
:104B300095F91622A1A10DF12E00F7F78FF9162293
:104B40009FA111A8F7F78AF916229EA10DF15A002C
:104B5000F7F784F90320F7F796FE0420F7F7FAFE3B
:104B60000020F9F727FD401CF7F791FE6946002069
:104B7000F7F7CBFE06A90120F7F7C7FE0DF12E01CE
:104B80000220F7F7C2FE11A90320F7F7BEFE0DF1D0
:104B90005A010420F7F7B9FE0120F7F7B1FB00280E
:104BA00002D0F9F7AFFD32E00820F7F7A9FB0028A3
:104BB0002AD00120F9F7FEFC002806D1012001F0DF
:104BC00005F860630120606417E0012806D1022027
:104BD00000F0FCFF6063022060640EE0022806D152
:104BE00003206064032000F0F1FF606305E004200F
:104BF0006064042000F0EAFF606301214120F9F7BE
:104C000018FD606B206402E00420F9F796FD1CB0EB
:104C100010BD10B592B0040070200021F3F7A9FD7B
:104C20000220F9F782FCDFF8D839DFF8DC291621F9
:104C30006846F7F78BFA69460020F7F766FE03200F
:104C4000F7F721FE0420F7F785FE1622BAA106A881
:104C5000F7F704F91622B9A10DF12E00F7F7FEF8C7
:104C60000020F9F7A7FC401CF7F711FE06A9012068
:104C7000F7F74BFE0DF12E010220F7F746FEB0A12B
:104C80000320F7F742FEAEA10420F7F73EFE08200E
:104C9000F7F736FB002818D00120F9F78BFC002825
:104CA00006D109206064092000F090FF606305E0F0
:104CB0000A2060640A2000F089FF6063012141201E
:104CC000F9F7B7FC606B20640AE00120F7F718FBE6
:104CD000002802D0F9F716FD02E00220F9F72DFDB9
:104CE00012B010BD10B592B0040070200021F3F78F
:104CF00040FD0220F9F719FCDFF80439DFF8102B2A
:104D000016216846F7F722FA69460020F7F7FDFDFD
:104D10000320F7F7B8FD0420F7F71CFE0020F9F791
:104D200049FC401CF7F7B3FD86A2162106A8F7F749
:104D30000DFA85A216210DF12E00F7F707FA06A944
:104D40000120F7F7E2FD0DF12E010220F7F7DDFD5E
:104D50007BA10320F7F7D9FD79A10420F7F7D5FD52
:104D60000820F7F7CDFA002818D00120F9F722FC27
:104D7000002806D10B2060640B2000F027FF606341
:104D800005E00C2060640C2000F020FF606301212E
:104D90004120F9F74EFC606B20640AE00120F7F730
:104DA000AFFA002802D0F9F7ADFC02E00220F9F7D3
:104DB000C4FC12B010BD00004931000049320000AF
:104DC000493300004934000030B59DB00500F5F7C7
:104DD000EAFF012801D1042400E002247020002110
:104DE000F3F7C7FC0420F9F7A0FBDFF81438DFF86D
:104DF000742B162116A8F7F7A9F954A216216846B4
:104E0000F7F7A4F952A216210DF11600F7F79EF953
:104E1000F5F7C9FF01280BD14EA216210BA8F7F711
:104E200095F94DA216210DF14200F7F78FF90AE02E
:104E300043A216210BA8F7F789F941A216210DF11B
:104E40004200F7F783F90320F7F71DFD0420F7F779
:104E500081FD0020F9F7AEFB401CF7F718FD16A9FD
:104E60000020F7F752FD69460120F7F74EFD0DF1DE
:104E700016010220F7F749FD0BA90320F7F745FDBE
:104E80000DF142010420F7F740FD0120F7F738FA51
:104E9000002802D0F9F736FC4CE00820F7F730FA8A
:104EA000002844D00120F9F785FB0400002C06D12E
:104EB000052000F08BFE68630520686430E0012C5B
:104EC00011D1F5F770FF012806D1062000F07EFE13
:104ED00068630620686423E0082000F077FE6863BA
:104EE000082068641CE0022C0AD1F5F75CFF012859
:104EF00006D1072000F06AFE6863072068640FE0AF
:104F0000032C0AD1F5F74FFF012806D1082000F045
:104F10005DFE68630820686402E00120F6F7FDFA90
:104F200001214120F9F785FB686B286402E020002D
:104F3000F9F703FC1DB030BD4531000045320000DB
:104F4000000000002049000020450000533100000F
:104F500053320000533300005334000030B58FB09B
:104F6000040070200021F3F704FC02A9606C00F03B
:104F7000FBFCDFF8D80A009002ABDFF8D42A162138
:104F800008A8F7F7E3F8616B02A8F9F773FD0420AE
:104F9000F7F779FC0420F7F7DDFC08A90020F7F704
:104FA000B4FC02A90120F7F7B0FC41A10220F7F7F9
:104FB000ACFC3FA10320F7F7A8FC3DA10420F7F7C4
:104FC000A4FC606B002805D139A2162102A8F7F7CE
:104FD000BDF80BE0606BC0B200F0FEFE05002B00D8
:104FE000DFF8702A162102A8F7F7B0F802A9052009
:104FF000F7F78BFC2EA10620F7F787FC2CA10720E2
:10500000F7F783FC2AA10820F7F77FFC0020F7F7C9
:105010003EFC0820F7F774F9002800F02581606B4A
:10502000216C884227D0606C00F03CFD050015F033
:10503000C005606BC0B200F041FE0543606B0C28F8
:1050400004D0606B0D2801D035F04005606B00285E
:105050000BD0606B022808D0606B032805D0606B12
:10506000052802D0606B062801D135F080052900A3
:10507000606C00F062FDF5F796FE012840F0CA80F2
:105080000020A063606B172808D0606B182805D03B
:10509000606B0E2802D0606B0F283ED1606C012837
:1050A00008D12900022000F048FD0120A063B1E0F2
:1050B00000000000606C032806D12900042000F0E5
:1050C0003CFD0120A063A5E0606C052806D1290005
:1050D000062000F032FD0120A0639BE0606C0728F1
:1050E00006D12900082000F028FD0120A06391E0EE
:1050F000606C092806D129000A2000F01EFD01205D
:10510000A06387E0606C0B2840F0848029000C20AD
:1051100000F013FD0120A0637CE0606C012811D138
:10512000022000F0BFFC30F0C000102805D011288C
:1051300003D00B2801D00A286CD100212A20F6F7D1
:1051400048FA67E0606C032811D1042000F0AAFC43
:1051500030F0C000102805D0112803D00B2801D052
:105160000A2857D100212E20F6F733FA52E0606C5E
:10517000092811D10A2000F095FC30F0C000102859
:1051800005D0112803D00B2801D00A2842D10021D4
:105190003220F6F71EFA3DE0606C052811D106209A
:1051A00000F080FC30F0C000102805D0112803D09A
:1051B0000B2801D00A282DD100212220F6F709FA68
:1051C00028E0606C072811D1082000F06BFC30F05B
:1051D000C000102805D0112803D00B2801D00A28C0
:1051E00018D100212620F6F7F4F913E0606C0B28A3
:1051F00010D10C2000F056FC30F0C000102805D073
:10520000112803D00B2801D00A2803D10021362011
:10521000F6F7DFF900200421F3F7ABFA606B002802
:105220001FD0606B02281CD0606B032819D0606B04
:10523000052816D0606B062813D0606C00F032FC95
:1052400010F08000002802D00120606301E00020FF
:10525000606302214220F9F7ECF9606B20640FB023
:1052600030BDF9F74FFAFAE70120F7F749F80028BF
:1052700002D0F9F747FAF2E7F5F795FD01285BD17F
:10528000606C02280ED0606C04280BD0606C06287D
:1052900008D0606C082805D0606C0A2802D0606CC9
:1052A0000C2849D1606C022804D1012000F08EFC4A
:1052B000050026E0606C042804D1032000F086FC81
:1052C00005001EE0606C0A2804D1092000F07EFC75
:1052D000050016E0606C062804D1052000F076FC7D
:1052E00005000EE0606C082804D1072000F06EFC79
:1052F000050006E0606C0C2803D10B2000F066FC72
:105300000500172D05D0182D03D00E2D01D00F2D1F
:1053100004D165630120F7F71DFBA0E7606B172838
:1053200008D0606B182805D0606B0E2802D0606B27
:105330000F2801D10020606300200190012000901F
:10534000012300221C21606BF9F76AFA6063F5F70C
:105350002AFD012840F0FA80606C0B282DD1606B8B
:10536000162812D0606B10280FD0606B11280CD05B
:10537000606B122809D0606B132806D0606B1A2866
:1053800003D0606B16287FF46AAF002001900120E3
:105390000090012300221C21606BF9F741FA606341
:1053A0000220F6F7A8FF0028D9D10420F6F79EFFC7
:1053B0000028D4D100206063D1E7606C0C2839D17B
:1053C000606B16281ED0606B10281BD0606B1128F4
:1053D00018D0606B122815D0606B132812D0606B48
:1053E0000E280FD0606B0F280CD0606B172809D0E7
:1053F000606B182806D0606B1A2803D0606B1628E3
:105400007FF42DAF002001900120009001230022A5
:105410001C21606BF9F704FA60630220F6F76BFF5A
:105420000028CDD10420F6F761FF0028C8D1002064
:105430006063C5E7606C02280BD0606C042808D05C
:10544000606C062805D0606C082802D0606C0A28C1
:1054500045D1606B10282AD0606B112827D0606B73
:10546000122824D0606B132821D0606B0E281ED028
:10547000606B0F281BD0606B172818D0606B182842
:1054800015D0606B1A2812D0606B16280FD0606B95
:1054900003280CD0606B022809D0606B062806D068
:1054A000606B052803D0606B16287FF4D8AE00200F
:1054B000019001200090012300221C21606BF9F76C
:1054C000AFF960630220F6F716FF0028C1D104206F
:1054D000F6F70CFF0028BCD100206063B9E7606BD1
:1054E00010281BD0606B112818D0606B122815D0C3
:1054F000606B132812D0606B1A280FD0606B1628CF
:105500000CD0606B032809D0606B022806D0606B5A
:10551000062803D0606B05287FF4A1AE002001901F
:1055200001200090012300221C21606BF9F778F91B
:1055300060630220F6F7DFFE0028D0D10420F6F7E2
:10554000D5FE0028CBD100206063C8E7F5F734FC16
:10555000012837D1606B022815D0606B032812D068
:10556000606B05280FD0606B06280CD0606B092893
:1055700009D0606B0D2806D0606B0B2803D0606BE0
:1055800019287FF46CAE00200190012000900123C7
:1055900000221C21606BF9F743F960630220F6F7E3
:1055A000AAFE0028D6D10420F6F7A0FE0028D1D10B
:1055B00000206063CEE70420F6F798FE002801D1B2
:1055C00000206063606B022809D0606B032806D05E
:1055D000606B052803D0606B06287FF440AE002086
:1055E000019001200090012300221C21606BF9F73B
:1055F00017F960630220F6F77EFE0028E2D1DAE7B1
:1056000080D403006CEF010078EF010030B58FB05B
:10561000040070200021F3F7ACF802A9606C00F0E0
:10562000A3F902ABDFF86424162108A8F6F78EFD73
:10563000606B002806D11622DFF8541402A8F6F792
:105640000DFC05E01622DFF84C1402A8F6F706FC64
:105650000420F7F718F90420F7F77CF908A90020CF
:10566000F7F753F902A90120F7F74FF9BCA102207F
:10567000F7F74BF9BAA10320F7F747F9B8A10420CF
:10568000F7F743F9B6A10520F7F73FF9B4A10620D3
:10569000F7F73BF9B2A10720F7F737F9B0A10820D7
:1056A000F7F733F90020F7F7F2F80820F6F728FEAD
:1056B00000286AD0606C00F0F5F90500606B216C81
:1056C000884207D0606B002802D135F0800501E0E8
:1056D00055F080052900606C00F02FFAF5F763FBA8
:1056E000012831D1A06B00282ED0606C012804D194
:1056F0002900022000F021FA26E0606C032804D182
:105700002900042000F019FA1EE0606C052804D17D
:105710002900062000F011FA16E0606C072804D179
:105720002900082000F009FA0EE0606C092804D175
:1057300029000A2000F001FA06E0606C0B2803D172
:1057400029000C2000F0F9F900200421F3F711F8EA
:10575000606C00F03BFA0C2801D00D2812D1606C6F
:1057600000F0A0F910F04000002802D00120606392
:1057700001E000206063606B206402214320F8F7A1
:1057800058FF43E0F8F7BEFF40E00120F6F7B8FD10
:10579000002802D0F8F7B6FF38E0F5F704FB01283F
:1057A00020D1606C00F012FA616C02290ED0616C9D
:1057B00004290BD0616C062908D0616C082905D03A
:1057C000616C0A2902D0616C0C290BD1172805D015
:1057D000182803D00E2801D00F2803D10120F7F795
:1057E000B9F813E00020019001200090012300226D
:1057F0000121606BF9F714F86063606C00F052F9F6
:1058000030F0C000172801D1002060630FB030BD18
:1058100058F2010010B58EB0040070200021F2F79C
:10582000A8FF02A9606C00F09FF802AB9A4A16210B
:1058300008A8F6F78BFC606B002805D11622974963
:1058400002A8F6F70BFB04E01622954902A8F6F72A
:1058500005FB0420F7F717F80420F7F77BF808A9F1
:105860000020F7F752F802A90120F7F74EF83CA103
:105870000220F7F74AF83AA10320F7F746F838A1D3
:105880000420F7F742F836A10520F7F73EF834A1D7
:105890000620F7F73AF832A10720F7F736F830A1DB
:1058A0000820F7F732F80020F6F7F1FF0820F6F7A6
:1058B00027FD002819D0606C00F0F4F80100606B3F
:1058C000226C904207D0606B002802D131F0400179
:1058D00001E051F04001606C00F02FF9002004213C
:1058E000F2F747FFF8F70EFF38E00120F6F708FD62
:1058F000002802D0F8F706FF30E0F5F754FA012847
:1059000021D1606C02280ED0606C04280BD0606C32
:10591000062808D0606C082805D0606C0A2802D0E0
:10592000606C0C280FD1606B172808D0606B1828AA
:1059300005D0606B0E2802D0606B0F2803D10120C8
:10594000F7F708F80AE000200190012000900123F9
:1059500000220121606BF8F763FF60630EB010BD99
:105960000000000084EF010010B50C00012805D1F3
:1059700039A204212000F6F7E9FB66E0022805D1F0
:1059800036A204212000F6F7E1FB5EE0032805D1F2
:1059900033A204212000F6F7D9FB56E0042805D1F4
:1059A00030A204212000F6F7D1FB4EE0092805D1F2
:1059B0002DA204212000F6F7C9FB46E00A2805D1F4
:1059C0002AA204212000F6F7C1FB3EE0052805D1FC
:1059D00027A204212000F6F7B9FB36E0062805D1FE
:1059E00024A204212000F6F7B1FB2EE0072805D100
:1059F00021A204212000F6F7A9FB26E008280FD1F8
:105A0000F5F7D1F9012805D11CA204212000F6F7F1
:105A10009DFB1AE017A204212000F6F797FB14E083
:105A20000B2805D116A204212000F6F78FFB0CE00D
:105A30000C2805D113A204212000F6F787FB04E00F
:105A400011A204212000F6F781FB10BD40D803000D
:105A500060F2010068F201004931000049320000A3
:105A60004933000049340000453100004532000050
:105A70005331000053320000533300005334000010
:105A800049000000450000004572000090EF010051
:105A900040D9030060D9030070F2010080E60300E2
:105AA000E0D9030080B5012803D12820F5F779FD5E
:105AB00042E0022803D12A20F5F773FD3CE00328D9
:105AC00003D12C20F5F76DFD36E0042803D12E20FC
:105AD000F5F767FD30E0052803D12020F5F761FDDB
:105AE0002AE0062803D12220F5F75BFD24E00728F1
:105AF00003D12420F5F755FD1EE0082803D1262008
:105B0000F5F74FFD18E0092803D13020F5F749FDDE
:105B100012E00A2803D13220F5F743FD0CE00B28F0
:105B200003D13420F5F73DFD06E00C2803D13620E3
:105B3000F5F737FD00E0002002BD80B5012803D154
:105B40002820F5F746FD40E0022803D12A20F5F78A
:105B500040FD3AE0032803D12C20F5F73AFD34E06C
:105B6000042803D12E20F5F734FD2EE0052803D1BB
:105B70002020F5F72EFD28E0062803D12220F5F796
:105B800028FD22E0072803D12420F5F722FD1CE0A0
:105B9000082803D12620F5F71CFD16E00B2803D1B9
:105BA0003420F5F716FD10E00C2803D13620F5F768
:105BB00010FD0AE0092803D13020F5F70AFD04E0C2
:105BC0000A2802D13220F5F704FD01BD80B5FFF7A8
:105BD00069FF30F0C000022801D101206CE02028CC
:105BE00001D1022068E0212801D1032064E00928C6
:105BF00001D1042060E01E2801D105205CE01F28AF
:105C000001D1062058E0042801D1072054E00528DE
:105C100001D1082050E0062801D109204CE00728D6
:105C200001D10A2048E0182801D10B2044E00828BF
:105C300001D10C2040E00E2801D10D203CE00B28C2
:105C400001D10E2038E00A2801D10F2034E01528B8
:105C500001D1102030E0142801D111202CE01328AC
:105C600001D1122028E0122801D1132024E00128BC
:105C700001D1142020E0032801D115201CE00F28B9
:105C800001D1162018E0102801D1172014E01128A6
:105C900001D1182010E00D2801D119200CE01628A0
:105CA00001D11A2008E00C2801D11B2004E017289C
:105CB00001D11C2000E00020C0B202BDC0B201280A
:105CC00001D1022087E0C0B2022801D11E2082E06B
:105CD000C0B2032801D121207DE0C0B2042801D147
:105CE000092078E0C0B2052801D11E2073E0C0B2BF
:105CF000062801D11F206EE0C0B2072801D1042080
:105D000069E0C0B2082801D1052064E0C0B20928CA
:105D100001D106205FE0C0B20A2801D107205AE075
:105D2000C0B20B2801D1182055E0C0B20C2801D117
:105D3000082050E0C0B20D2801D10E204BE0C0B2C7
:105D40000E2801D10B2046E0C0B20F2801D10A2055
:105D500041E0C0B2102801D115203CE0C0B21128AA
:105D600001D1142037E0C0B2122801D1132032E053
:105D7000C0B2132801D112202DE0C0B2142801D1E5
:105D8000012028E0C0B2152801D1032023E0C0B2D1
:105D9000162801D10F201EE0C0B2172801D1102013
:105DA00019E0C0B2182801D1112014E0C0B219289E
:105DB00001D10D200FE0C0B21A2801D116200AE04F
:105DC000C0B21B2801D10C2005E0C0B21C2801D1B3
:105DD000172000E000207047C0B2012801D1012047
:105DE00087E0C0B2022801D1022082E0C0B20328BD
:105DF00001D103207DE0C0B2042801D1042078E065
:105E0000C0B2052801D1052073E0C0B2062801D137
:105E100006206EE0C0B2072801D1072069E0C0B2B9
:105E2000082801D1082064E0C0B2092801D1092066
:105E30005FE0C0B20A2801D10A205AE0C0B20B28A4
:105E400001D10B2055E0C0B20C2801D1142050E044
:105E5000C0B20D2801D115204BE0C0B20E2801D1EF
:105E60001E2046E0C0B20F2801D11F2041E0C0B281
:105E7000102801D120203CE0C0B2112801D12120FE
:105E800037E0C0B2122801D1222032E0C0B213287C
:105E900001D123202DE0C0B2142801D1282028E010
:105EA000C0B2152801D1292023E0C0B2162801D1A3
:105EB0002A201EE0C0B2172801D12B2019E0C0B261
:105EC000182801D12C2014E0C0B2192801D12D20AE
:105ED0000FE0C0B21A2801D12E200AE0C0B21B2860
:105EE00001D13C2005E0C0B21C2801D13D2000E0DA
:105EF0000020704710B592B0040070200021F2F726
:105F000038FC0220F8F711FBDFF8A434DFF8A424F2
:105F100016216846F6F71AF98DA2162106A8F6F79B
:105F200015F98CA216210DF12E00F6F70FF90320BA
:105F3000F6F7A9FC0420F6F70DFD0020F8F73AFB70
:105F4000401CF6F7A4FC69460020F6F7DEFC06A923
:105F50000120F6F7DAFC0DF12E010220F6F7D5FC50
:105F6000C7A10320F6F7D1FCC5A10420F6F7CDFCAC
:105F70000120F6F7C5F9002802D0F8F7C3FB24E0AA
:105F80000820F6F7BDF900281CD00120F8F712FB15
:105F9000002808D10D2060644820F5F702FB30F09E
:105FA000C000606307E00E2060644920F5F7F9FA4D
:105FB00030F0C000606301214520F8F73AFB606BC8
:105FC000206402E00220F8F7B8FB12B010BD10B553
:105FD0008EB0040070200021F2F7CBFB606C0D281E
:105FE00008D1DFF8D433DFF8D423162108A8F6F758
:105FF000ADF807E0DFF8C033DFF8C423162108A8A6
:10600000F6F7A4F8616BC9B202A8F8F71AFE0420EB
:10601000F6F739FC0420F6F79DFC0020F6F737FC74
:1060200008A90020F6F771FC02A90120F6F76DFC23
:10603000626BDFF8901302A8F6F77DF890A10220BA
:10604000F6F763FC8EA10320F6F75FFC8CA1042019
:10605000F6F75BFC02A90520F6F757FC88A106209D
:10606000F6F753FC86A10720F6F74FFC84A1082021
:10607000F6F74BFC0820F6F743F9002853D0606B85
:10608000216C88421FD0606C0D2806D14820F5F79E
:1060900088FA010011F0800105E04920F5F781FA46
:1060A000010011F08001606B0143606C0D2803D189
:1060B0004820F5F78EFA02E04920F5F78AFA002029
:1060C0000821F2F756FB606B092810D10221472006
:1060D000F8F7AFFA606C0D2804D14A20F5F761FAA1
:1060E000606333E04B20F5F75CFA60632EE0022139
:1060F0004620F8F79EFA606C0D2805D14820F5F788
:1061000050FA10F0800004E04920F5F74AFA10F048
:106110008000002802D00120606301E0002060635D
:10612000606B206412E00120F6F7EAF8002802D044
:10613000F8F7E8FA0AE0002001900120009001231E
:1061400000220C21606BF8F76BFB60630EB010BD92
:106150004F3100004F32000010B58EB004007020A7
:106160000021F2F706FB606C0D2806D1964B934A8E
:10617000162108A8F5F7EAFF05E0934B904A16218F
:1061800008A8F5F7E3FF636B904A162102A8F5F71C
:10619000DDFF0420F6F777FB0420F6F7DBFB002099
:1061A000F6F775FB08A90020F6F7AFFB02A901205E
:1061B000F6F7ABFB32A10220F6F7A7FB30A10320D4
:1061C000F6F7A3FB2EA10420F6F79FFB2CA10520D8
:1061D000F6F79BFB2AA10620F6F797FB28A10720DC
:1061E000F6F793FB26A10820F6F78FFB0820F6F7B9
:1061F00087F800282FD0606B216C88420FD0606C2C
:106200000D2804D1616B4A20F5F7E3F903E0616BD7
:106210004B20F5F7DEF900200821F2F7AAFA022157
:106220004620F8F706FA606C0D2805D14820F5F7EE
:10623000B8F910F0800004E04920F5F7B2F910F049
:106240008000002802D00120606301E0002060632C
:10625000606B206412E00120F6F752F8002802D0AB
:10626000F8F750FA0AE00120019000200090012385
:106270000122F021606BF8F7D3FA60630EB010BD15
:106280000000000010B58EB0040070200021F2F76D
:1062900070FA606C0D2805D14D4A162108A8F5F753
:1062A00055FF04E04B4A162108A8F5F74FFF606B35
:1062B000002805D11622484902A8F5F7CFFD04E0D1
:1062C0001622464902A8F5F7C9FD0420F6F7DBFAC5
:1062D0000420F6F73FFB0020F6F7D9FA08A90020C2
:1062E000F6F713FB02A90120F6F70FFB2FA10220FE
:1062F000F6F70BFB2DA10320F6F707FB2BA10420DB
:10630000F6F703FB29A10520F6F7FFFA27A10620DF
:10631000F6F7FBFA25A10720F6F7F7FA23A10820E4
:10632000F6F7F3FA0120F5F7EBFF002802D0F8F7B3
:10633000E9F939E00820F5F7E3FF002829D0606B80
:10634000216C884222D0606C0D2806D14820F5F7D8
:1063500028F9010031F0800105E04920F5F721F925
:10636000010031F08001606B002801D051F0800104
:10637000606C0D2803D14820F5F72BF902E0492085
:10638000F5F727F900200821F2F7F3F9F8F7BAF941
:106390000AE0002001900120009001230022012149
:1063A000606BF8F73DFA60630EB010BD00000000AE
:1063B000A0D40300D8EF010040D8030068F3010027
:1063C00070F3010078F3010020D9030080F301008D
:1063D000E4EF0100F0EF010040D9030060D90300B1
:1063E00010B59CB0040070200021F2F7C2F904201F
:1063F000F8F79BF8DFF81439ACA216216846F5F7D8
:10640000A5FEDFF80C39DFF80C29162106A8F5F7F0
:106410009DFEDFF80439DFF8042916210DF12E0066
:10642000F5F794FEDFF8F838DFF8F828162111A800
:10643000F5F78CFEDFF8F02816210DF15A00F5F77C
:1064400085FE0320F6F71FFA0420F6F783FA0020F2
:10645000F8F7B0F8401CF6F71AFA69460020F6F78C
:1064600054FA06A90120F6F750FA0DF12E01022088
:10647000F6F74BFA11A90320F6F747FA0DF15A0186
:106480000420F6F742FA0820F5F73AFF002826D054
:106490000120F8F78FF8002804D101214920F8F7EE
:1064A000C8F819E0012804D101215120F8F7C1F8FA
:1064B00012E0022808D101215920F8F7BAF8542037
:1064C000F5F76FF8606307E001215A20F8F7B1F89B
:1064D0005C20F5F766F86063606B20640AE00120D9
:1064E000F5F70EFF002802D0F8F70CF902E00420BF
:1064F000F8F723F91CB010BD30B5A7B00400702028
:106500000021F2F736F90620F8F70FF8DFF8003827
:1065100066A216216846F5F719FEDFF81038DFF895
:10652000F427162106A8F5F711FEDFF80438DFF886
:10653000EC2716210DF12E00F5F708FEDFF8F437F1
:10654000DFF8E027162111A8F5F700FEDFF8E8379D
:10655000DFF8E82716210DF15A00F5F7F7FDDFF80F
:10656000E037DFF8E02716211CA8F5F7EFFDDFF88C
:10657000D837DFF8D82716210DF18600F5F7E6FDAC
:106580000320F6F780F90420F6F7E4F90020F8F785
:1065900011F8401CF6F77BF969460020F6F7B5F9CB
:1065A0000220F8F707F8050006A8162101FB05F1FF
:1065B00001440120F6F7A9F906A8162101FB05F10F
:1065C000084410F116010220F6F79FF906A81621DB
:1065D00001FB05F1084410F12C010320F6F795F9B1
:1065E00006A91620454301EB050010F142010420E5
:1065F000F6F78BF90820F5F783FE002848D0012034
:10660000F7F7D8FF002808D101214A20F8F711F840
:106610001620F4F7C6FF606345E0012808D1012188
:106620004B20F8F706F81020F4F7BBFF60633AE060
:10663000022808D101214D20F7F7FBFF0E20F4F7C7
:10664000B0FF60632FE0032808D101214E20F7F747
:10665000F0FF1C20F4F7A5FF606324E0042808D1B4
:1066600001214F20F7F7E5FF0420F4F79AFF60635C
:1066700019E0052808D101215020F7F7DAFF06209C
:10668000F4F78FFF60630EE00120F4F746FF0AE0A5
:106690000120F5F735FE002802D0F8F733F802E0C4
:1066A0000620F8F74AF827B030BD00002573000037
:1066B00010B58EB0040070200021F2F75AF81622AF
:1066C000DFF88C1608A8F5F7C9FB636B9BA21621AF
:1066D00002A8F5F73BFD0420F6F7D5F80420F6F7FD
:1066E00039F90020F6F7D3F808A90020F6F70DF9DC
:1066F00002A90120F6F709F9CFA10220F6F705F962
:10670000CDA10320F6F701F9CBA10420F6F7FDF89F
:10671000C9A10520F6F7F9F8C7A10620F6F7F5F8A4
:10672000C5A10720F6F7F1F8C3A10820F6F7EDF8A8
:106730000820F5F7E5FD002810D01620F4F731FF0A
:10674000616B814207D0616B1620F4F742FF002095
:106750000221F2F70EF8F7F7D5FF12E00120F5F766
:10676000CFFD002802D0F7F7CDFF0AE0002001900E
:1067700001200090012301220A21606BF8F750F8F4
:1067800060630EB010BD10B58EB004007020002103
:10679000F1F7EFFF1622DFF8BC1508A8F5F75EFB4E
:1067A000636BDFF8B425162102A8F5F7CFFC0420AF
:1067B000F6F769F808A90020F6F7A7F802A9012062
:1067C000F6F7A3F89CA10220F6F79FF89AA1032000
:1067D000F6F79BF898A10420F6F797F896A1052004
:1067E000F6F793F894A10620F6F78FF892A1072008
:1067F000F6F78BF890A10820F6F787F80020F6F757
:1068000046F80820F5F77CFD002816D01020F4F794
:10681000C8FE616B814207D0616B1020F4F7D9FE8E
:1068200000200221F1F7A5FF02214C20F7F701FF1C
:106830000020F4F7B6FE606312E00120F5F760FD7A
:10684000002802D0F7F75EFF0AE001200190002047
:10685000009001230022C821606BF7F7E1FF60631D
:106860000EB010BD10B58EB0040070200021F1F7FD
:1068700080FF1622DFF8E41408A8F5F7EFFA636B3F
:10688000B2A2162102A8F5F761FC0420F5F7FBFF80
:106890000420F6F75FF808A90020F6F736F802A9F9
:1068A0000120F6F732F864A10220F6F72EF862A173
:1068B0000320F6F72AF860A10420F6F726F85EA177
:1068C0000520F6F722F85CA10620F6F71EF85AA17B
:1068D0000720F6F71AF858A10820F6F716F8002056
:1068E000F5F7D5FF0820F5F70BFD002810D00020A4
:1068F000F4F757FE616B814207D0616B0020F4F71B
:1069000068FE00200221F1F734FFF7F7FBFE12E0EA
:106910000120F5F7F5FC002802D0F7F7F3FE0AE0B6
:106920000020019000200090012301220321606BD0
:10693000F7F776FF60630EB010BD000025326400EB
:1069400010B58EB0040070200021F1F712FF16225E
:10695000DFF80C1408A8F5F781FA636BB1A21621D1
:1069600002A8F5F7F3FB0420F5F78DFFF4F71BFA07
:10697000012803D10120F5F7EDFF02E00420F5F72F
:10698000E9FF08A90020F5F7C0FF02A90120F5F7EB
:10699000BCFF29A10220F5F7B8FF27A10320F5F7D6
:1069A000B4FF25A10420F5F7B0FF23A10520F5F7DA
:1069B000ACFF21A10620F5F7A8FF1FA10720F5F7DE
:1069C000A4FF1DA10820F5F7A0FF0020F5F75FFF49
:1069D0000820F5F795FC002810D00E20F4F7E1FD13
:1069E000616B814207D0616B0E20F4F7F2FD00204D
:1069F0000221F1F7BEFEF7F785FE1AE00120F5F758
:106A00007FFC002806D0F4F7CEF9012811D0F7F763
:106A100079FE0EE0F4F7C7F901280AD000200190B2
:106A200000200090012301220A21606BF7F7F8FE95
:106A300060630EB010BD00000000000010B590B003
:106A4000040070200021F1F794FE1622C54909A820
:106A5000F5F704FA636BC44A032102A8F5F776FB45
:106A60009DF808008DF80C002E208DF80D009DF883
:106A700009008DF80E0000208DF80F000420F5F7B6
:106A800002FFF4F790F9012803D10120F5F762FF26
:106A900002E00420F5F75EFF09A90020F5F735FFB5
:106AA00003A90120F5F731FF94A10220F5F72DFF8E
:106AB00093A10320F5F729FF91A10420F5F725FF05
:106AC0008FA10520F5F721FF8DA10620F5F71DFF09
:106AD0008BA10720F5F719FF89A10820F5F715FF0D
:106AE0000020F5F7D4FE0820F5F70AFC00280FD0A7
:106AF0001C20F4F756FD616B814207D0616B1C20AE
:106B0000F4F767FD00200221F1F733FEF7F7FAFDF5
:106B10000120F5F7F5FB002806D0F4F744F9012829
:106B200011D0F7F7EFFD0EE0F4F73DF901280AD098
:106B30000120019000200090012301221E21606BA2
:106B4000F7F76EFE606310B010BD00002564000012
:106B500010B58EB0040070200021F1F70AFE162255
:106B6000824908A8F5F77AF9636B66A2162102A894
:106B7000F5F7ECFA0420F5F786FE0420F5F7EAFEB7
:106B80000020F5F784FE08A90020F5F7BEFE02A953
:106B90000120F5F7BAFE5AA10220F5F7B6FE58A17A
:106BA0000320F5F7B2FE56A10420F5F7AEFE54A17E
:106BB0000520F5F7AAFE52A10620F5F7A6FE50A182
:106BC0000720F5F7A2FE4EA10820F5F79EFE08204B
:106BD000F5F796FB002810D00420F4F7E2FC616B77
:106BE000814207D0616B0420F4F7F3FC00200221FE
:106BF000F1F7BFFDF7F786FD12E00120F5F780FB06
:106C0000002802D0F7F77EFD0AE000200190002066
:106C10000090012301220A21606BF7F701FE6063F7
:106C20000EB010BD2532640010B58EB00400702087
:106C30000021F1F79EFD16224D4908A8F5F70EF93F
:106C4000636B31A2162102A8F5F780FA0420F5F74C
:106C50001AFE0420F5F77EFE0020F5F718FE08A9BD
:106C60000020F5F752FE02A90120F5F74EFE24A1FF
:106C70000220F5F74AFE22A10320F5F746FE20A1E7
:106C80000420F5F742FE1EA10520F5F73EFE1CA1EB
:106C90000620F5F73AFE1AA10720F5F736FE18A1EF
:106CA0000820F5F732FE0820F5F72AFB002810D05F
:106CB0000620F4F776FC616B814207D0616B0620F9
:106CC000F4F787FC00200221F1F753FDF7F71AFDD6
:106CD00012E00120F5F714FB002802D0F7F712FDAF
:106CE0000AE00020019000200090012301220A21E7
:106CF000606BF7F795FD60630EB010BD2073000068
:106D000000000000256400002532640060D3030009
:106D100080D50300E8F20100A0D50300F0F20100E5
:106D2000C0F50300F8F20100C0EF0100C0D5030078
:106D3000E0D5030000D6030020D6030000F30100D5
:106D400040D6030008F3010060D6030010F30100F1
:106D500080D60300A0D6030018F30100C0D60300BC
:106D6000E0D6030000D7030020F3010020D7030082
:106D700040D7030030B5A7B0040070200021F1F720
:106D8000F8FC0620F7F7D1FBDFF870399BA216213B
:106D90006846F5F7DBF9DFF86839DFF8682916216E
:106DA00006A8F5F7D3F9DFF86039DFF86029162176
:106DB0000DF12E00F5F7CAF9DFF85439DFF8542940
:106DC000162111A8F5F7C2F9DFF84C39DFF84C2984
:106DD00016210DF15A00F5F7B9F9DFF84439DFF85B
:106DE000442916211CA8F5F7B1F9DFF83C39DFF882
:106DF0003C2916210DF18600F5F7A8F90320F5F7D7
:106E000042FD0420F5F7A6FD0020F7F7D3FB401C58
:106E1000F5F73DFD69460020F5F777FD0220F7F70D
:106E2000C9FB050006A8162101FB05F1014401205C
:106E3000F5F76BFD06A8162101FB05F1084410F1DA
:106E400016010220F5F761FD06A8162101FB05F1E8
:106E5000084410F12C010320F5F757FD06A9162070
:106E6000454301EB050010F142010420F5F74DFD0B
:106E70000820F5F745FA002848D00120F7F79AFBDB
:106E8000002808D101215220F7F7D3FB1820F4F78E
:106E900088FB606345E0012808D101215320F7F702
:106EA000C8FB1220F4F77DFB60633AE0022808D1AA
:106EB00001215520F7F7BDFB0C20F4F772FB60634E
:106EC0002FE0032808D101215620F7F7B2FB1A2042
:106ED000F4F767FB606324E0042808D10121572000
:106EE000F7F7A7FB0820F4F75CFB606319E00528BF
:106EF00008D101215820F7F79CFB0A20F4F751FB39
:106F000060630EE00120F4F708FB0AE00120F5F7CA
:106F1000F7F9002802D0F7F7F5FB02E00620F7F7B3
:106F20000CFC27B030BD10B58EB0040070200021DD
:106F3000F1F71FFC1622DFF8F81708A8F4F78EFF08
:106F4000636B9EA2162102A8F5F700F90420F5F75D
:106F50009AFC0420F5F7FEFC0020F5F798FC08A940
:106F60000020F5F7D2FC02A90120F5F7CEFCCAA15A
:106F70000220F5F7CAFCC8A10320F5F7C6FCC6A19C
:106F80000420F5F7C2FCC4A10520F5F7BEFCC2A1A0
:106F90000620F5F7BAFCC0A10720F5F7B6FCBEA1A4
:106FA0000820F5F7B2FC0820F5F7AAF9002810D060
:106FB0001820F4F7F6FA616B814207D0616B182054
:106FC000F4F707FB00200221F1F7D3FBF7F79AFB58
:106FD00012E00120F5F794F9002802D0F7F792FBB0
:106FE0000AE00020019000200090012301220A21E4
:106FF000606BF7F715FC60630EB010BD25730000E1
:1070000010B58EB0040070200021F1F7B2FB1622FB
:10701000DFF8201708A8F4F721FF636BDFF81827C3
:10702000162102A8F5F792F80420F5F72CFC0420AD
:10703000F5F790FC08A90020F5F767FC02A90120EC
:10704000F5F763FC94A10220F5F75FFC92A1032001
:10705000F5F75BFC90A10420F5F757FC8EA1052005
:10706000F5F753FC8CA10620F5F74FFC8AA1072009
:10707000F5F74BFC88A10820F5F747FC0020F5F751
:1070800006FC0820F5F73CF9002816D01220F4F78A
:1070900088FA616B814207D0616B1220F4F799FA8C
:1070A00000200221F1F765FB02215420F7F7C1FA15
:1070B0000220F4F776FA606312E00120F5F720F978
:1070C000002802D0F7F71EFB0AE001200190002003
:1070D000009001230022C821606BF7F7A1FB6063D9
:1070E0000EB010BD10B58EB0040070200021F1F775
:1070F00040FB1622DFF8441608A8F4F7AFFE636BD6
:107100002EA2162102A8F5F721F80420F5F7BBFB03
:107110000420F5F71FFC08A90020F5F7F6FB02A9EB
:107120000120F5F7F2FB5CA10220F5F7EEFB5AA176
:107130000320F5F7EAFB58A10420F5F7E6FB56A17A
:107140000520F5F7E2FB54A10620F5F7DEFB52A17E
:107150000720F5F7DAFB50A10820F5F7D6FB002051
:10716000F5F795FB0820F5F7CBF8002810D00220A2
:10717000F4F717FA616B814207D0616B0220F4F7D4
:1071800028FA00200221F1F7F4FAF7F7BBFA12E02F
:107190000120F5F7B5F8002802D0F7F7B3FA0AE0B6
:1071A0000020019000200090012301220321606B48
:1071B000F7F736FB60630EB010BD000025640000D9
:1071C00010B58EB0040070200021F1F7D2FA16221B
:1071D000DFF86C1508A8F4F741FE636BA1A2162135
:1071E00002A8F4F7B3FF0420F5F74DFB0420F5F7F0
:1071F000B1FB08A90020F5F788FB02A90120F5F7EB
:1072000084FB25A10220F5F780FB23A10320F5F7DD
:107210007CFB21A10420F5F778FB1FA10520F5F7E1
:1072200074FB1DA10620F5F770FB1BA10720F5F7E5
:107230006CFB19A10820F5F768FB0020F5F727FB88
:107240000820F5F75DF8002810D00C20F4F7A9F914
:10725000616B814207D0616B0C20F4F7BAF9002012
:107260000221F1F786FAF7F74DFA12E00120F5F75F
:1072700047F8002802D0F7F745FA0AE0002001900D
:1072800000200090012301220A21606BF7F7C8FA61
:1072900060630EB010BD00000000000010B590B09B
:1072A000040070200021F1F764FA1622DFF894142C
:1072B00009A8F4F7D3FD636BDFF88C24032102A83F
:1072C000F4F744FF9DF808008DF80C002E208DF88F
:1072D0000D009DF809008DF80E0000208DF80F00BC
:1072E0000420F5F7D0FA0420F5F734FB09A90020B3
:1072F000F5F70BFB03A90120F5F707FBC4A102205A
:10730000F5F703FBC3A10320F5F7FFFAC1A10420A1
:10731000F5F7FBFABFA10520F5F7F7FABDA10620A6
:10732000F5F7F3FABBA10720F5F7EFFAB9A10820AA
:10733000F5F7EBFA0020F5F7AAFA0820F4F7E0FFDA
:1073400000280FD01A20F4F72CF9616B814207D086
:10735000616B1A20F4F73DF900200221F1F709FAD8
:10736000F7F7D0F90120F4F7CBFF002802D0F7F7A8
:10737000C9F90AE0002001900020009001230122B9
:107380001E21606BF7F74CFA606310B010BD10B5AA
:107390008EB0040070200021F1F7EBF91622DFF81F
:1073A000AC1308A8F4F75AFD636B9BA2162102A840
:1073B000F4F7CCFE0420F5F766FA0420F5F7CAFAD4
:1073C0000020F5F764FA08A90020F5F79EFA02A953
:1073D0000120F5F79AFA8FA10220F5F796FA8DA110
:1073E0000320F5F792FA8BA10420F5F78EFA89A114
:1073F0000520F5F78AFA87A10620F5F786FA85A118
:107400000720F5F782FA83A10820F5F77EFA082015
:10741000F4F776FF002810D00820F4F7C2F8616B6B
:10742000814207D0616B0820F4F7D3F800200221D5
:10743000F1F79FF9F7F766F912E00120F4F760FF22
:10744000002802D0F7F75EF90AE000200190002042
:107450000090012301220A21606BF7F7E1F96063D4
:107460000EB010BD2532640010B58EB0040070203F
:107470000021F1F77EF91622B54908A8F4F7EEFCD1
:10748000636B65A2162102A8F4F760FE0420F5F7ED
:10749000FAF90420F5F75EFA0020F5F7F8F908A9E3
:1074A0000020F5F732FA02A90120F5F72EFA59A1CA
:1074B0000220F5F72AFA57A10320F5F726FA55A17D
:1074C0000420F5F722FA53A10520F5F71EFA51A181
:1074D0000620F5F71AFA4FA10720F5F716FA4DA185
:1074E0000820F5F712FA0820F4F70AFF002810D058
:1074F0000A20F4F756F8616B814207D0616B0A20CD
:10750000F4F767F800200221F1F733F9F7F7FAF8FA
:1075100012E00120F4F7F4FE002802D0F7F7F2F8A9
:107520000AE00020019000200090012301220A219E
:10753000606BF7F775F960630EB010BD10B58EB0D3
:10754000040070200021F1F714F91622814908A8DF
:10755000F4F784FC636B30A2162102A8F4F7F6FD61
:107560000420F5F790F90420F5F7F4F90020F5F779
:107570008EF908A90020F5F7C8F902A90120F5F74E
:10758000C4F924A10220F5F7C0F922A10320F5F7E0
:10759000BCF920A10420F5F7B8F91EA10520F5F7E4
:1075A000B4F91CA10620F5F7B0F91AA10720F5F7E8
:1075B000ACF918A10820F5F7A8F90820F4F7A0FE07
:1075C000002810D05420F3F7ECFF616B814207D004
:1075D000616B5420F3F7FDFF00200821F1F7C9F893
:1075E000F7F790F812E00120F4F78AFE002802D0A5
:1075F000F7F788F80AE000200190002000900123AE
:1076000001220521606BF7F70BF960630EB010BD26
:1076100020730000000000002564000010B58EB04B
:10762000040070200021F1F7A4F84B4A162108A8A5
:10763000F4F78CFD636B2FA2162102A8F4F786FDE8
:107640000420F5F720F908A90020F5F75EF902A952
:107650000120F5F75AF928A10220F5F756F926A1DD
:107660000320F5F752F924A10420F5F74EF922A1E1
:107670000520F5F74AF920A10620F5F746F91EA1E5
:107680000720F5F742F91CA10820F5F73EF9002084
:10769000F5F7FDF80820F4F733FE00280ED0606BF4
:1076A000216C884207D0616B5C20F3F792FF0020C9
:1076B0000821F1F75EF8F7F725F819E00120F4F753
:1076C0001FFE002802D0F7F71DF811E0F3F76BFB5F
:1076D000012802D1002060630AE00020019001200F
:1076E0000090012300220A21606BF7F799F860638C
:1076F0000EB010BD2532640000000000A0D50300CC
:10770000C0D5030028F30100E0D5030030F30100E9
:1077100000D6030038F3010020D6030040F3010037
:1077200040D6030048F3010060D6030050F3010087
:1077300060D7030080D7030058F30100A0D70300EF
:10774000C0D70300E0D7030060F3010000D80300B6
:1077500020D80300C0F50300CCEF010010B598B0AD
:1077600070200021F1F705F80320F6F7DEFE16225F
:10777000DFF8C4136846F4F771FBDFF8C033DFF8B5
:10778000C023162106A8F4F7E1FCDFF8B833DFF8D0
:10779000B82316210DF12E00F4F7D8FCDFF8AC3336
:1077A000DFF8AC23162111A8F4F7D0FC0320F5F77D
:1077B0006AF80420F5F7CEF80020F6F7FBFE401C2F
:1077C000F5F765F80220F6F7F5FE0400694600209B
:1077D000F5F79BF806A8162101FB04F101440120EE
:1077E000F5F793F806A8162101FB04F1084410F1FF
:1077F00016010220F5F789F806A8162101FB04F10D
:10780000084410F12C010320F5F77FF806A9162093
:10781000444301EB040010F142010420F5F775F830
:107820000120F4F76DFD002802D0F6F76BFF32E07F
:107830000820F4F765FD00282AD00120F6F7BAFEEB
:10784000002809D101215C20F6F7F3FE3820F3F778
:10785000A8FEC04908601EE0012809D101215D2071
:10786000F6F7E7FE3920F3F79CFEBA49086012E00C
:10787000022809D101215E20F6F7DBFE3A20F3F75A
:1078800090FEB449086006E00120F3F746FE02E0EE
:107890000320F6F752FF18B010BD00B589B0702074
:1078A0000021F0F766FF1622A44902A8F4F7D6FAE1
:1078B00002A90020F5F729F80420F4F7E4FFA54811
:1078C0000368A54A162102A8F4F740FC02A901208A
:1078D000F5F71BF80420F5F73DF895A10220F5F720
:1078E00014F893A10320F5F710F891A10420F5F7FF
:1078F0000CF88FA10520F5F708F88DA10620F5F703
:1079000004F88BA10720F5F700F889A10820F4F707
:10791000FCFF0020F4F7BBFF0820F4F7F1FC00287F
:1079200012D03820F3F73DFE8A490968814208D019
:10793000884801683820F3F74CFE00200421F0F756
:1079400018FFF6F7DFFE14E00120F4F7D9FC002859
:1079500002D0F6F7D7FE0CE0012001900020009045
:10796000012300221E217B480068F6F759FF794960
:10797000086009B000BD00B58FB070200021F0F79D
:10798000F8FE0420F4F77FFF0420F4F7E3FF16224B
:107990006C4908A8F4F762FA08A90020F4F7B5FFCB
:1079A0006C4803686C4A162102A8F4F7CFFB02A9C1
:1079B0000120F4F7AAFF5EA10220F4F7A6FF5CA164
:1079C0000320F4F7A2FF5AA10420F4F79EFF58A168
:1079D0000520F4F79AFF56A10620F4F796FF54A16C
:1079E0000720F4F792FF52A10820F4F78EFF002041
:1079F000F4F74DFF0820F4F783FC002812D039205B
:107A0000F3F7CFFD53490968814208D05148016816
:107A10003920F3F7DEFD00200421F0F7AAFEF6F787
:107A200071FE14E00120F4F76BFC002802D0F6F799
:107A300069FE0CE00120019000200090012300224B
:107A4000F02144480068F6F7EBFE424908600FB0A9
:107A500000BD00B58FB070200021F0F78AFE3B4BCF
:107A600034A2162108A8F4F771FB3A4803683A4A91
:107A7000162102A8F4F76AFB0420F4F704FF04209F
:107A8000F4F768FF0020F4F702FF08A90020F4F7DC
:107A90003CFF02A90120F4F738FF25A10220F4F7EA
:107AA00034FF23A10320F4F730FF21A10420F4F7D1
:107AB0002CFF1FA10520F4F728FF1DA10620F4F7D5
:107AC00024FF1BA10720F4F720FF19A10820F4F7D9
:107AD0001CFF0120F4F714FC002802D0F6F712FE78
:107AE00024E00820F4F70CFC002812D03A20F3F729
:107AF00058FD18490968814208D0164801683A20A3
:107B0000F3F767FD00200421F0F733FEF6F7FAFDE6
:107B10000CE0012001900020009001230022F021C0
:107B20000C480068F6F77CFE0A4908600FB000BDFB
:107B3000000000002573000080F1030040D4030022
:107B400020F4010060D4030028F4010060D5030094
:107B500030F401003412002038F4010070B59EB0FA
:107B600004005720F3F71DFD012801D1042500E092
:107B7000022548200021F0F7FCFD1622DFF8EC1A60
:107B800017A8F4F76BF9DFF8E83ADFF8E82A1621CE
:107B900001A8F4F7DBFADFF8E00A0090DFF80C3C0C
:107BA000DFF80C2C16210DF11A00F4F7CFFA57204C
:107BB000F3F7F7FC012811D1DFF8F83BDFF8F82BD9
:107BC00016210CA8F4F7C2FADFF8F03BDFF8F02B2F
:107BD00016210DF14600F4F7B9FA0AE090A2162139
:107BE0000CA8F4F7B3FA8EA216210DF14600F4F7B3
:107BF000ADFA2800F6F799FC0320F4F744FE0420C0
:107C0000F4F7A8FE17A90020F4F77FFE0020F6F78E
:107C1000D1FC401CF4F73BFE0220F6F7CBFC06003B
:107C200001A8162101FB06F101440120F4F76DFEC5
:107C300001A8162101FB06F1084410F116010220EB
:107C4000F4F763FE01A8162101FB06F1084410F1C8
:107C50002C010320F4F759FE01A91620464301EB3D
:107C6000060010F142010420F4F74FFE0120F4F762
:107C700047FB002802D0F6F745FD2EE00820F4F778
:107C80003FFB002826D00120F6F794FC002808D1FD
:107C900001217920F6F7CDFC5620F3F782FC6063D2
:107CA00015E0012808D101217B20F6F7C2FC5720FE
:107CB000F3F777FC60630AE0022804D101217C20FD
:107CC000F6F7B7FC03E001217D20F6F7B2FC606B0C
:107CD000206402E02800F6F730FD1EB070BD10B53C
:107CE0008EB0040048200021F0F743FDDFF888093A
:107CF0000090DFF8B83ADFF8082C162108A8F4F74E
:107D000025FA606B01280AD1DFF8A00A0090636BA6
:107D1000DFF8F02B162102A8F4F718FA09E0DFF8D3
:107D200058090090636BDFF8DC2B162102A8F4F7EA
:107D30000DFA0420F4F7A7FD0420F4F70BFE08A9C0
:107D40000020F4F7E2FD02A90120F4F7DEFD34A1E2
:107D50000220F4F7DAFD32A10320F4F7D6FD30A1BA
:107D60000420F4F7D2FD2EA10520F4F7CEFD2CA1BE
:107D70000620F4F7CAFD2AA10720F4F7C6FD28A1C2
:107D80000820F4F7C2FD0020F4F781FD0820F4F785
:107D9000B7FA00280ED0606B216C884207D0616B67
:107DA0005720F3F716FC00200821F0F7E2FCF6F765
:107DB000A9FC33E00120F4F7A3FA002802D0F6F77B
:107DC000A1FC2BE05620F3F7ECFB02281BD1606BE3
:107DD000012805D0606B032802D0032060631DE0FA
:107DE0000220F4F788FA002804D10420F4F783FA7B
:107DF000002813D0606B012802D1032060630DE0DE
:107E0000012060630AE0002001900120009001231E
:107E100001220F21606BF6F703FD60630EB010BD09
:107E20000000000010B58EB0040048200021F0F7DB
:107E3000A0FC1622DFF8381808A8F4F70FF8606BDA
:107E4000012806D11622DFF8681B02A8F4F706F80D
:107E50000FE0606B022806D11622DFF8581B02A83B
:107E6000F3F7FCFF05E01622DFF84C1B02A8F3F73E
:107E7000F5FF0420F4F707FD0420F4F76BFD08A9D3
:107E80000020F4F742FD02A90120F4F73EFDC4A151
:107E90000220F4F73AFDC2A10320F4F736FDC0A199
:107EA0000420F4F732FDBEA10520F4F72EFDBCA19D
:107EB0000620F4F72AFDBAA10720F4F726FDB8A1A1
:107EC0000820F4F722FD0020F4F7E1FC0820F4F785
:107ED00017FA00281CD0606B216C884207D0616BB8
:107EE0005620F3F776FB00200821F0F742FC606B88
:107EF00002280AD15820F3F754FB6063606B2064BA
:107F000002217A20F6F795FB1BE0F6F7FBFB18E061
:107F10000120F4F7F5F9002802D0F6F7F3FB10E0A2
:107F2000F2F741FF012801D1012100E002210020E8
:107F300001900120009001230022606BF6F770FC95
:107F400060630EB010BD10B58CB004004820002155
:107F5000F0F70FFCDFF8643892A2162106A8F4F7B8
:107F6000F5F8DFF8B03B90A216216846F4F7EEF87A
:107F70000420F4F788FC0320F4F7ECFC0020F4F76D
:107F800086FC06A90020F4F7C0FC69460120F4F73E
:107F9000BCFC83A10220F4F7B8FC81A10320F4F714
:107FA000B4FC7FA10420F4F7B0FC7DA10520F4F718
:107FB000ACFC7BA10620F4F7A8FC79A10720F4F71C
:107FC000A4FC77A10820F4F7A0FC0820F4F798F9A6
:107FD00000280ED04020F3F7CCF800208021F0F7E5
:107FE000C8FB02218420F6F724FBF2F771FD6063E1
:107FF00006E00120F4F784F9002801D0F6F782FBAF
:108000000CB010BD10B58CB004001622DFF8AC1710
:1080100006A8F3F723FFDFF8002B16216846F4F7D4
:1080200095F80420F4F72FFC0020F4F793FC06A940
:108030000020F4F76AFC69460120F4F766FCD6A13B
:108040000220F4F762FCD4A10320F4F75EFCD2A175
:108050000420F4F75AFCD0A10520F4F756FCCEA179
:108060000620F4F752FCCCA10720F4F74EFCCAA17D
:108070000820F4F74AFC0020F4F709FCF2F728FD89
:10808000616B401A40F2D17188420CD35FF080706E
:108090000021F2F789FF00220023994203D1904288
:1080A00001D1F6F72FFB0CB010BD10B58EB0040057
:1080B00048200021F0F75DFB1622DFF8F81808A829
:1080C000F3F7CCFE606B012806D11622DFF84C1ABC
:1080D00002A8F3F7C3FE05E01622DFF8441A02A84F
:1080E000F3F7BCFE0420F4F7CEFB0420F4F732FCD7
:1080F00008A90020F4F709FC02A90120F4F705FC07
:10810000A5A10220F4F701FCA3A10320F4F7FDFBD5
:10811000A1A10420F4F7F9FB9FA10520F4F7F5FBDA
:108120009DA10620F4F7F1FB9BA10720F4F7EDFBDE
:1081300099A10820F4F7E9FB0020F4F7A8FB082038
:10814000F4F7DEF8002816D05820F3F72AFA606B0F
:10815000216C88420CD0606B012801D1012100E024
:1081600002215820F3F735FA00200821F0F701FB2F
:10817000F6F7C8FA12E00120F4F7C2F8002802D09E
:10818000F6F7C0FA0AE000200190012000900123D8
:1081900001220221606BF6F743FB60630EB010BD55
:1081A000000000002573000025733F002DE9F04713
:1081B000E6B0050048200021F0F7DBFA00240DE0CE
:1081C00075A216210BA8162303FB04F31844F3F73A
:1081D000BDFF002058A941F82400641C0E2CEFD3E9
:1081E000F3F7CEF88146F3F7BDF80600F3F7BDF8D4
:1081F0008046F3F710F90400F3F713F9044300275E
:108200005FF0020A0BE05046F3F7FEFC19EA000F9C
:1082100003D058A840F827A07F1C1AF1010ABAF130
:10822000100FF0D31622DFF88C1505A8F3F716FE11
:108230005FF0010922E059A20B2102A8F3F786FFA3
:1082400004E055A20A2102A8F3F780FF02A80190DA
:1082500058A800EB890050F8040C0090DFF818349F
:10826000DFF8C02816210BA85FF0160C0CFB09FCE8
:1082700060441638F3F76AFF19F101094F4527D317
:1082800058A800EB890050F8040CF3F7BDFC064237
:10829000D1D018EA000F13D0044208D0DFF8883894
:1082A000DFF888280D2102A8F3F750FFCEE7DFF8AA
:1082B0007838DFF87C280D2102A8F3F747FFC5E7DF
:1082C0000442BED0A0A20A2102A8F3F73FFFBDE7F7
:1082D0003800F6F72AF90320F4F7D5FA0420F4F76A
:1082E00039FB05A90020F4F710FB0020F6F762F92E
:1082F000401CF4F7CCFA0220F6F75CF904000BA856
:10830000162101FB04F101440120F4F7FEFA0BA849
:10831000162101FB04F1084410F116010220F4F7C4
:10832000F4FA0BA8162101FB04F1084410F12C010A
:108330000320F4F7EAFA0BA91620444301EB0400EA
:1083400010F142010420F4F7E0FA0120F3F7D8FF1E
:10835000002802D0F6F7D6F91BE00820F3F7D0FF8B
:10836000002813D00120F6F725F958A951F820006C
:108370006863686BF3F748FC064204D001217E2055
:10838000F6F757F905E0F6F7BDF902E03800F6F721
:10839000D4F966B0BDE8F08700000000282129006C
:1083A00030B5A3B00500686BF0F7FAF94FF48060C0
:1083B0000021F0F7DEF9686B0090AF4BDFF874270F
:1083C000162101A8F3F7C2FE0520F6F7AEF8DFF894
:1083D0006827162107A8F3F7B9FEDFF86037DFF842
:1083E000602716210DF13200F3F7B0FEDFF85437A5
:1083F000DFF8C423162112A8F3F7A8FEDFF84837E8
:10840000DFF8BC2316210DF15E00F3F79FFEDFF8C5
:108410003C37DFF83C2716211DA8F3F797FE032011
:10842000F4F731FA0420F4F795FA01A90020F4F7E3
:108430006CFA0220F6F7BEF8040007A8162101FB2B
:1084400004F101440120F4F760FA07A8162101FBAA
:1084500004F1084410F116010220F4F756FA07A8B7
:10846000162101FB04F1084410F12C010320F4F75C
:108470004CFA07A91620444301EB040010F1420115
:108480000420F4F742FA0020F6F794F8401CF4F7C1
:10849000FEF90120F3F734FF002802D0F6F732F995
:1084A0004FE00820F3F72CFF002847D00120F6F713
:1084B00081F80400686BF2F7B7FF002C04D10121AA
:1084C0007F20F6F7B6F83CE0012C06D1052804D051
:1084D00001218120F6F7ADF833E0022C06D1052802
:1084E00004D001218020F6F7A4F82AE0032C06D15D
:1084F000052804D001218220F6F79BF821E0042C06
:108500001FD105281DD0686BF3F77EFB0400F2F73E
:1085100088FF204202D00220A86308E0F2F77BFF28
:10852000204202D00120A86301E00020A863A86BCC
:10853000286401218320F6F77CF802E00520F6F795
:10854000FCF823B030BD0000282A290010B58CB0FB
:108550000400606BF0F724F94FF480600021F0F71D
:1085600008F9636BDFF8EC25162106A8F3F7EEFD9A
:10857000606BF2F759FFA063A06B052806D1DFF806
:10858000D82516216846F3F7E1FD38E0A06B0428F2
:1085900006D1DFF8C82516216846F3F7D7FD2EE08F
:1085A000A06B062806D1DFF8B82516216846F3F738
:1085B000CDFD24E0A06B072806D1DFF8A825162101
:1085C0006846F3F7C3FD1AE0A06B092806D1DFF86F
:1085D000982516216846F3F7B9FD10E0A06B08282E
:1085E00006D1DFF8882516216846F3F7AFFD06E0CF
:1085F000DFF87C35C0A216216846F3F7A7FD0420FA
:10860000F4F741F90120F4F7A5F90020F4F73FF958
:1086100006A90020F4F779F969460120F4F775F905
:10862000B6A10220F4F771F9B4A10320F4F76DF9B3
:10863000B2A10420F4F769F9B0A10520F4F765F9B7
:10864000AEA10620F4F761F9ACA10720F4F75DF9BB
:10865000AAA10820F4F759F90820F3F751FE0028E1
:1086600001D0F6F74FF80CB010BD00004CEA010045
:1086700040D80300C8F001002CEA010070B5B4B086
:108680000600706BF0F78CF84FF480600021F0F773
:1086900070F8DFF8B0040090736BDFF8D82416216F
:1086A00001A8F3F753FD01A90020F4F72EF90020EB
:1086B0000AE0002207AB162404FB00F423445A54BA
:1086C000491C1629F5D3401C082801D20021F8E7DF
:1086D00001240025706BF2F772FE06000CE02642C2
:1086E00009D02200002307A8162101FB05F1084448
:1086F000F9F753FE6D1C6400082D01D2002CEED159
:108700002800F5F712FF0320F4F7BDF80420F4F772
:1087100021F901A90020F4F7F8F8002E03D1002078
:10872000F4F7B5F805E00020F5F744FF401CF4F736
:10873000AEF80220F5F73EFF040007A8162101FB62
:1087400004F101440120F4F7E0F807A8162101FB29
:1087500004F1084410F116010220F4F7D6F807A836
:10876000162101FB04F1084410F12C010320F4F759
:10877000CCF807A91620444301EB040010F1420194
:108780000420F4F7C2F80820F3F7BAFD002804D15A
:108790000120F3F7B5FD002802D0F5F7B3FF02E0A2
:1087A0002800F5F7CAFF34B070BD00000CEA0100E4
:1087B000D0F0010020F60300D8F0010080E00300B3
:1087C000E0F00100F0B5B3B00400606BEFF7E8FF34
:1087D0004FF480600021EFF7CCFFD8480090636B26
:1087E000DFF89023162101A8F3F7B0FC01A90020BF
:1087F000F4F78BF80320F4F746F80420F4F7AAF80E
:1088000000200AE0002207AB162505FB00F52B44EB
:108810005A54491C1629F5D3401C082801D20021BE
:10882000F8E7606BF2F7B7FD0500606BF2F7FCFD4F
:10883000062801D1012700E00027012400260CE0D2
:10884000254209D03A00210007A8162303FB06F3AE
:108850001844F9F749FD761C6400082E01D2002C5B
:10886000EED13000F5F761FE002D03D10020F4F7C2
:108870000EF805E00020F5F79DFE401CF4F707F820
:108880000220F5F797FE040007A8162101FB04F16A
:1088900001440120F4F739F807A8162101FB04F17F
:1088A000084410F116010220F4F72FF807A816214A
:1088B00001FB04F1084410F12C010320F4F725F822
:1088C00007A91620444301EB040010F142010420E3
:1088D000F4F71BF80820F3F713FD002804D101205A
:1088E000F3F70EFD002802D0F5F70CFF02E0300090
:1088F000F5F723FF33B0F0BD257300000000000042
:10890000E8F00100F0F0010010B58EB00400606BDB
:10891000EFF746FF4FF480600021EFF72AFF636B0B
:10892000954A162107A8F3F711FC07A90020F3F7D1
:10893000ECFF0420F3F7A7FF0120F4F70BF80A235C
:10894000152207A98D48F5F7D9FF606BF2F74CFDAA
:10895000009007AB8A4A162101A8F3F7F7FB01A99B
:108960000120F3F7D2FF6AA10220F3F7CEFF68A13E
:108970000320F3F7CAFF66A10420F3F7C6FF64A142
:108980000620F3F7C2FF62A10720F3F7BEFF60A144
:108990000820F3F7BAFF0020F3F779FF0820F3F778
:1089A000AFFC002801D0F5F7ADFE0EB010BD000001
:1089B000ECE9010080F4030080E6030030B58FB0DD
:1089C000040008200021EFF7D4FE606BEFF7E8FE0B
:1089D0004FF480600021EFF7CCFE636B664A1621EE
:1089E00008A8F3F7B3FBA06B002805D11622654950
:1089F00002A8F3F733FA0EE0A06B012805D1162286
:108A0000614902A8F3F72AFA05E0604B604A162193
:108A100002A8F3F79BFB0420F3F735FF0420F3F7DC
:108A200099FF0020F3F733FF08A90020F3F76DFF4B
:108A300002A90120F3F769FF35A10220F3F765FFD2
:108A400033A10320F3F761FF31A10420F3F75DFFA9
:108A50002FA10520F3F759FF2DA10620F3F755FFAD
:108A60002BA10720F3F751FF29A10820F3F74DFFB1
:108A70000820F3F745FC002834D0206CA16B884215
:108A80002DD0606BF3F7C0F80500A06B002808D16B
:108A9000F2F7C1FC0400AC43F2F7C3FC30EA050571
:108AA00012E0A06B012808D1F2F7B5FC04002C43BA
:108AB000F2F7B7FC30EA050506E0F2F7ACFC04007B
:108AC000AC43F2F7AEFC05432000F2F7A1FC28000E
:108AD000F2F7A4FC5FF480100021EFF74AFEF5F7EF
:108AE00011FE12E00120F3F70BFC002802D0F5F78D
:108AF00009FE0AE0002001900120009001230022DD
:108B00000221A06BF5F78CFEA0630FB030BD000012
:108B100000000000E0DA0300ECED010040F6030085
:108B200060F60300F8ED010020E50300F8F0010015
:108B300000F1010008F1010010F1010060D2030012
:108B400018F1010080D2030000ED030020ED0300C6
:108B500020F101006CEC010004EE010028F101009D
:108B600010EE010030F1010038F1010040F1010088
:108B7000E0E003001CEE010028EE0100E0EC030041
:108B800048F1010080E6030060E40300E0F5030023
:108B900034EE010030B5A7B00500F2F704F9012862
:108BA00003D10520F5F7C1FC02E00620F5F7BDFC76
:108BB00078200021EFF7DDFD1622DFF8141A684651
:108BC000F3F74CF9F2F7EFF8012830D1DFF8043A67
:108BD000DFF8042A162106A8F3F7B8FADFF8FC3903
:108BE000DFF8FC2916210DF12E00F3F7AFFADFF8BC
:108BF000F439DFF8F429162111A8F3F7A7FADFF802
:108C0000EC39DFF8EC2916210DF15A00F3F79EFA42
:108C1000DFF8E039DFF8E02916211CA8F3F796FA0F
:108C20008AA216210DF18600F3F790FA32E0DFF800
:108C3000CC39DFF8A429162106A8F3F787FADFF864
:108C4000C039DFF89C2916210DF12E00F3F77EFACA
:108C5000DFF88839DFF89029162111A8F3F776FAA2
:108C6000DFF88039DFF8882916210DF15A00F3F773
:108C70006DFADFF87839DFF8802916211CA8F3F7A0
:108C800065FADFF87039DFF87C2916210DF18600CE
:108C9000F3F75CFA0320F3F7F6FD0420F3F75AFE2E
:108CA0000020F5F787FC401CF3F7F1FD6946002032
:108CB000F3F72BFE0220F5F77DFC040006A8162131
:108CC00001FB04F101440120F3F71FFE06A8162161
:108CD00001FB04F1084410F116010220F3F715FE20
:108CE00006A8162101FB04F1084410F12C01032011
:108CF000F3F70BFE06A91620444301EB040010F124
:108D000042010420F3F701FE0820F3F7F9FA0028E6
:108D100000F087800120F5F74DFC0400F2F743F8DE
:108D200001282AD1002C0ED101216020F5F781FC09
:108D30000220F2F725FC002802D1002068636DE0D4
:108D4000012068636AE0012C04D101216320F5F75A
:108D500070FC63E0022C04D101216420F5F769FC6A
:108D60005CE0032C04D101216520F5F762FC55E09D
:108D700001216620F5F75DFC50E0002C13D1F2F7DD
:108D800053F800284AD101216120F5F752FC5FF029
:108D90000040F2F7F5FB002802D1002068633DE0B7
:108DA000012068633AE0012C0FD101216220F5F720
:108DB00040FC4FF40070F2F7E3FB002802D00120E2
:108DC00068632BE00020686328E0022C08D1F2F7EA
:108DD0002BF8002822D101216320F5F72AFC1DE0A1
:108DE000032C08D1F2F720F8002817D101216420C4
:108DF000F5F71FFC12E0042C08D1F2F715F8002853
:108E00000CD101216520F5F714FC07E0F2F70CF80E
:108E1000002803D101216620F5F70BFC686B28645C
:108E200012E00120F3F76CFA002802D0F5F76AFC93
:108E30000AE0F1F7B8FF012803D10520F5F77DFC22
:108E400002E00620F5F779FC27B030BD00000000F5
:108E500010B58EB0040078200021EFF78AFC1622AE
:108E6000DFF8701708A8F2F7F9FF606B002806D149
:108E70001622DFF8941702A8F2F7F0FF05E0162299
:108E8000DFF8881702A8F2F7E9FF0420F3F7FBFCEC
:108E90000420F3F75FFD0020F3F7F9FC08A9002098
:108EA000F3F733FD02A90120F3F72FFDCFA1022034
:108EB000F3F72BFDCDA10320F3F727FDCBA1042071
:108EC000F3F723FDC9A10520F3F71FFDC7A1062075
:108ED000F3F71BFDC5A10720F3F717FDC3A1082079
:108EE000F3F713FD0820F3F70BFA002814D0206CD9
:108EF000616B88420DD0606B002803D00220F2F72E
:108F000043FB02E00220F2F745FB00200821EFF7C7
:108F100030FCF5F7F7FB12E00120F3F7F1F9002838
:108F200002D0F5F7EFFB0AE000200190012000904D
:108F3000012300220121606BF5F772FC60630EB023
:108F400010BD10B58EB0040070200021EFF711FCA9
:108F50001622DFF8AC1608A8F2F780FF606B002835
:108F600006D11622DFF8A81602A8F2F777FF05E06F
:108F70001622DFF8A01602A8F2F770FF0420F3F71C
:108F800082FC0420F3F7E6FC0020F3F780FC08A93C
:108F90000020F3F7BAFC02A90120F3F7B6FC93A175
:108FA0000220F3F7B2FC91A10320F3F7AEFC8FA1EE
:108FB0000420F3F7AAFC8DA10520F3F7A6FC8BA1F2
:108FC0000620F3F7A2FC89A10720F3F79EFC87A1F6
:108FD0000820F3F79AFC0820F3F792F9002816D03E
:108FE000606B216C88420FD0606B002804D14FF475
:108FF0000070F2F7CFFA03E04FF40070F2F7C4FA12
:1090000000200821EFF7B5FBF5F77CFB19E0012004
:10901000F3F776F9002802D0F5F774FB11E0F1F7C9
:10902000E7FE012802D1002060630AE000200190E1
:1090300001200090012300220121606BF5F7F0FB75
:1090400060630EB010BD10B58EB004007820002112
:10905000EFF78FFB1622DFF8A41508A8F2F7FEFE43
:10906000606B002806D11622DFF8AC1502A8F2F7D3
:10907000F5FE05E01622DFF8A41502A8F2F7EEFED1
:109080000420F3F700FC0420F3F764FC0020F3F75E
:10909000FEFB08A90020F3F738FC02A90120F3F732
:1090A00034FC52A10220F3F730FC50A10320F3F767
:1090B0002CFC4EA10420F3F728FC4CA10520F3F76B
:1090C00024FC4AA10620F3F720FC48A10720F3F76F
:1090D0001CFC46A10820F3F718FC0820F3F710F950
:1090E000002816D0206C616B88420FD0606B00287E
:1090F00004D05FF00040F2F747FA03E05FF0004071
:10910000F2F748FA00200821EFF733FBF5F7FAFAF7
:1091100012E00120F3F7F4F8002802D0F5F7F2FA94
:109120000AE000200190012000900123002201218B
:10913000606BF5F775FB60630EB010BD00B58DB0C8
:1091400078200021EFF715FB1622DFF8901406A80F
:10915000F2F784FEDFF8C83485A216216846F2F7DC
:10916000F5FF0420F3F78FFB0320F3F7F3FB002058
:10917000F3F78DFB06A90020F3F7C7FB6946012032
:10918000F3F7C3FB19A10220F3F7BFFB17A10320DC
:10919000F3F7BBFB15A10420F3F7B7FB13A10520E0
:1091A000F3F7B3FB11A10620F3F7AFFB0FA10720E4
:1091B000F3F7ABFB0DA10820F3F7A7FB0820F3F7AB
:1091C0009FF8002809D00220F1F7D3FF002080216A
:1091D000EFF7CFFAF5F796FA06E00120F3F790F8EB
:1091E000002801D0F5F78EFA0DB000BD0000000098
:1091F00030B587B078200021EFF7BBFA1622DFF8F0
:10920000E4136846F2F72AFE0025F1F7AAFF0400EE
:10921000E00701D555F01005F1F7C5FD01280CD187
:10922000A00701D555F02005600701D555F0400590
:10923000200706D555F0800503E0200701D555F03D
:109240002005E00601D555F00105A00601D555F031
:109250000205600601D555F00405200601D555F03C
:109260000805F1F7A0FD012809D114F4A04F01D0A1
:1092700055F4807514F4204F01D055F4007514F4A2
:10928000406F01D055F40045E00501D555F4005577
:10929000A00501D555F48045E00301D555F480556E
:1092A000F1F763FFC10701D555F48065800701D54B
:1092B00055F400650520F3F7E6FA0120F3F74AFBC1
:1092C00069460020F3F721FB2800F3F7E0FA0820B5
:1092D000F3F716F8002801D0F5F714FA07B030BDFF
:1092E00000B58DB078200021EFF743FA1622BF4970
:1092F00006A8F2F7B3FDF1F7F2FE0100C9B2684625
:10930000F5F72CFB0420F3F7BEFA0120F3F722FB5C
:109310000020F3F7BCFA06A90020F3F7F6FA694635
:109320000120F3F7F2FAA7A10220F3F7EEFAA5A1C4
:109330000320F3F7EAFAA3A10420F3F7E6FAA1A1C8
:109340000520F3F7E2FA9FA10620F3F7DEFA9DA1CC
:109350000720F3F7DAFA9BA10820F3F7D6FA0820E2
:10936000F2F7CEFF002801D0F5F7CCF90DB000BD23
:1093700025733F0010B5A4B078200021EFF7F9F96C
:1093800016229C4902A8F2F769FD0520F5F7CDF8F1
:10939000F1F7B9FE0300A34A06216846F2F7D6FEAC
:1093A0009DF802008DF803002C208DF802000020AB
:1093B0008DF804009DF80100202802D130208DF89E
:1093C00001009DF80300202802D130208DF8030011
:1093D0006B46954A162108A8F2F7B8FEF1F79BFEF6
:1093E000030079A206216846F2F7B0FE9DF802005C
:1093F0008DF803002C208DF8020000208DF8040069
:109400009DF80100202802D130208DF801009DF840
:109410000300202802D130208DF803006B46834AD8
:1094200016210DF13600F2F791FEF1F77CFE0300F4
:1094300065A206216846F2F789FE9DF802008DF8C4
:1094400003002C208DF8020000208DF804009DF808
:109450000100202802D130208DF801009DF8030082
:10946000202802D130208DF803006B46704A162167
:1094700013A8F2F76BFEF1F73EFE030052A206219D
:109480006846F2F763FE9DF802008DF803002C2079
:109490008DF8020000208DF804009DF801002028BE
:1094A00003D130208DF8010009E09DF801002D283E
:1094B00005D130208DF801002D208DF800009DF899
:1094C0000300202803D130208DF8030006E09DF82A
:1094D00003002D2802D130208DF803006B46554A39
:1094E00016210DF16200F2F731FEF1F765FC01285B
:1094F00008D1F1F72AFE03004F4A16211EA8F2F701
:1095000025FE0FE0F1F721FE0A2190FBF1F32FA2D7
:1095100005216846F2F71AFE6B46484A16211EA836
:10952000F2F714FE0320F3F7AEF90420F3F712FA72
:109530000020F5F73FF8401CF3F7A9F902A9002035
:10954000F3F7E3F90220F5F735F8040008A816212F
:1095500001FB04F101440120F3F7D7F908A8162113
:1095600001FB04F1084410F116010220F3F7CDF9D4
:1095700008A8162101FB04F1084410F12C01032076
:10958000F3F7C3F908A91620444301EB040010F1D6
:1095900042010420F3F7B9F90820F2F7B1FE0028E0
:1095A00002D0F5F7AFF80AE00120F2F7A9FE002893
:1095B00002D0F5F7A7F802E00520F5F7BEF824B0D1
:1095C00010BD000000000000253564002534640053
:1095D000E0D3030000DA030078F2010020DA030090
:1095E00080F2010040DA030088F2010060DA030033
:1095F00090F2010080DA030098F20100C0E003005D
:10960000A0DB0300A0F20100C0DA0300A0DA03002F
:1096100080E60300E0D903009CEF01005CED01004F
:10962000E0DA0300A8F201006CED01007CED01001E
:109630008CED01009CED0100ACED010080EC01001F
:1096400070B5C4B00500F1F7B7FB012801D10824BB
:109650000CE0F1F7A8FB012801D10B2406E0F1F79B
:10966000B9FB012801D10A2400E00B24702000215D
:10967000EFF77FF82000F4F758FF1622DFF8EC1A16
:109680003DA8F2F7EBFBF1F797FB012854D1DFF887
:10969000E03ADFF8E02A16216846F2F757FDDFF8D6
:1096A000D83ADFF8D82A16210DF11600F2F74EFD50
:1096B000DFF8183CDFF8182C16210BA8F2F746FD4E
:1096C000DFF8103CDFF8102C16210DF14200F2F704
:1096D0003DFDDFF8083CDFF8082C162116A8F2F74C
:1096E00035FDDFF8003CDFF8002C16210DF16E008F
:1096F000F2F72CFDDFF8F43BDFF8F42B162121A85C
:10970000F2F724FDDFF8EC3BDFF8EC2B16210DF12E
:109710009A00F2F71BFD43A216212CA8F2F716FDC2
:1097200040A216210DF1C600F2F710FD3DA2162150
:1097300037A8F2F70BFD88E0DFF8343ADFF8342A77
:1097400016216846F2F702FDDFF8B03BDFF82C2A5D
:1097500016210DF11600F2F7F9FCDFF81C3ADFF8DC
:10976000702B16210BA8F2F7F1FCDFF8603BDFF855
:10977000682B16210DF14200F2F7E8FCDFF8543BAC
:10978000DFF85C2B162116A8F2F7E0FCDFF8703B3F
:10979000DFF8542B16210DF16E00F2F7D7FCDFF83D
:1097A0003C3BDFF84C2B162121A8F2F7CFFCDFF869
:1097B000343BDFF8442B16210DF19A00F2F7C6FC7A
:1097C000DFF8283BDFF8202C16212CA8F2F7BEFC8E
:1097D000F1F7E9FA012811D1DFF8103CDFF8102C7D
:1097E00016210DF1C600F2F7B1FCDFF8083BDFF8F7
:1097F000DC2C162137A8F2F7A9FC26E0F1F7EAFAEB
:10980000012811D1DFF8EC3ADFF8E42B16210DF135
:10981000C600F2F79BFC03A2162137A8F2F796FCCC
:1098200013E000BF00000000DFF8C83ADFF8C02BEB
:1098300016210DF1C600F2F789FCDFF8B83BDFF81E
:109840008C2C162137A8F2F781FC0320F3F71BF8C4
:109850000420F3F77FF80020F4F7ACFE401CF3F788
:1098600016F83DA90020F3F750F80220F4F7A2FE05
:1098700006006846162101FB06F101440120F3F7BA
:1098800044F86846162101FB06F1084410F1160160
:109890000220F3F73AF86846162101FB06F1084466
:1098A00010F12C010320F3F730F8694616204643E7
:1098B00001EB060010F142010420F3F726F808201E
:1098C000F2F71EFD002800F059810120F4F772FE26
:1098D0000400F1F771FA012840F08280002C04D1D5
:1098E00001216820F4F7A5FE45E1012C0ED10121EC
:1098F0006C20F4F79EFE4020F1F742FE002802D1D2
:109900000020686337E10120686334E1022C0FD145
:1099100001216D20F4F78DFE4FF48060F1F730FEE9
:10992000002802D10020686325E10120686322E15C
:10993000032C1CD101216E20F4F77BFE0420F1F7EB
:109940001FFE002808D14FF48070F1F719FE00289F
:1099500002D1002068630EE10420F1F711FE002817
:1099600002D00120686306E10220686303E1042C51
:1099700007D101217020F4F75CFEF5F7E2F9686386
:10998000F9E0052C0AD101217120F4F752FE4F2095
:10999000F1F707FE10F00F006863ECE0062C0ED123
:1099A00001217320F4F745FE8020F1F7E9FD00283E
:1099B00002D001206863DEE000206863DBE0072C52
:1099C00040F0D98001217720F4F733FEF4F7A9FDA8
:1099D000002802D100206863CDE001206863CAE05E
:1099E000002C04D101216820F4F723FEC3E0012CF0
:1099F00008D101216A20F4F71CFE1420F1F7D1FDF3
:109A00006863B8E0022C0ED101216C20F4F711FE3E
:109A10004020F1F7B5FD002802D100206863AAE0DC
:109A200001206863A7E0032C0FD101216D20F4F71A
:109A300000FE4FF48060F1F7A3FD002802D1002062
:109A4000686398E00120686395E0042C1CD1012133
:109A50006E20F4F7EEFD0420F1F792FD002808D106
:109A60004FF48070F1F78CFD002802D1002068636C
:109A700081E00420F1F784FD002802D00120686312
:109A800079E00220686376E0052C08D101216F207F
:109A9000F4F7CFFD3D20F1F784FD68636BE0062C01
:109AA00007D101217020F4F7C4FDF5F74AF9686386
:109AB00061E0072C0AD101217120F4F7BAFD4F2093
:109AC000F1F76FFD10F00F00686354E0082C0ED121
:109AD00001217320F4F7ADFD8020F1F751FD00283E
:109AE00002D00120686346E00020686343E0092C4F
:109AF0000CD1F1F758F9012808D101216B20F4F7B6
:109B000098FD3C20F1F74DFD686334E0092C0DD140
:109B100001217720F4F78DFDF4F703FD002802D131
:109B20000020686327E00120686324E00A2C11D13B
:109B3000F1F739F901280DD101217720F4F779FDEA
:109B4000F4F7EFFC002802D10020686313E0012045
:109B5000686310E00A2C0ED101217520F4F769FD2D
:109B60004FF48050F1F70CFD002802D0012068630B
:109B700001E000206863686B28640AE00120F2F7C6
:109B8000BFFB002802D0F4F7BDFD02E02000F4F78F
:109B9000D4FD44B070BD10B58CB00400702000211D
:109BA000EEF7E7FD1622DFF8C81506A8F2F756F91A
:109BB0005FF000400021F1F7F7F9002200239942FD
:109BC00008D1904206D11622DFF8E41B6846F2F76E
:109BD00045F905E01622DFF8DC1B6846F2F73EF98E
:109BE0000420F2F750FE0320F2F7B4FE0020F2F753
:109BF0004EFE06A90020F2F788FE69460120F2F722
:109C000084FEA8A10220F2F780FEA6A10320F2F7AD
